:100000000C9445060C948B060C948B060C948B0672
:100010000C948B060C948B060C948B060C948B061C
:100020000C948B060C94C8180C948B060C948B06BD
:100030000C9446320C948B060C948B060C948B0615
:100040000C948B060C948B060C949C150C948B06CC
:100050000C94CB0B0C948B060C94950B0C948B0688
:100060000C94841B0C948B060C94CC2D0C948B0656
:100070000C9413780C948B060C947872AB1BB01B09
:10008000B51BBE1BD51BEC1BFC1B0C1C291C151E19
:10009000EC1BD71CE81C171D351D521DAC1D071E7F
:1000A0000E20B8204721C721FE21A122A824122515
:1000B0008C25D5251F264D267A26DD262727712754
:1000C0006A28EB2D1F2E622ED22EEA2E2B2FE22F26
:1000D000A930A930A930A930A930A930A930A93058
:1000E000A930A930A9305E30603065307D307F3076
:1000F0000A0D426174743A002025642043656C6CDB
:10010000732000204C6F77207761726E696E6720D4
:100110006C6576656C3A2025642E2564000A0D46D0
:100120006F756E6420424C2D4374726C3A2000252A
:1001300064000A0D0A0D2121204D495353494E47B1
:1001400020424C2D4354524C3A202564202121005A
:100150000A0D3D3D3D3D3D3D3D3D3D3D3D3D3D3D32
:100160003D3D3D3D3D3D3D3D3D3D3D3D3D3D3D3DBF
:100170003D3D3D3D3D000A0D43616C696272617415
:10018000696E672070726573737572652073656E32
:10019000736F722E2E004F4B0A0D000A0D466C69CC
:1001A0006768742D74696D65202575206D696E20F2
:1001B00020546F74616C3A2575206D696E000A0DCC
:1001C000436F6E74726F6C3A200048656164696EAB
:1001D00067486F6C64004E6F726D616C20284143FC
:1001E000432D4D6F646529000A0D3D3D3D3D3D3D6C
:1001F0003D3D3D3D3D3D3D3D3D3D3D3D3D3D3D3D2F
:100200003D3D3D3D3D3D3D3D3D3D3D3D3D0A0D00BE
:10021000416E676C654E69636B2020202020202092
:10022000416E676C65526F6C6C202020202020206E
:100230004163634E69636B20202020202020202012
:10024000416363526F6C6C202020202020202020EE
:100250005961774779726F202020202020202020AC
:100260004865696768742056616C75652020202098
:100270004163635A2020202020202020202020209D
:1002800047617320202020202020202020202020B3
:10029000436F6D706173732056616C75652020200B
:1002A000566F6C74616765205B302E31565D20207F
:1002B0005265636569766572204C6576656C2020B1
:1002C0004779726F20436F6D706173732020202017
:1002D0004D6F746F7220312020202020202020209C
:1002E0004D6F746F7220322020202020202020208B
:1002F0004D6F746F7220332020202020202020207A
:100300004D6F746F72203420202020202020202068
:1003100031362020202020202020202020202020B6
:1003200031372020202020202020202020202020A5
:100330003138202020202020202020202020202094
:100340003139202020202020202020202020202083
:10035000536572766F20202020202020202020202E
:10036000486F76657267617320202020202020204E
:1003700043757272656E74205B302E31415D2020B2
:100380004361706163697479205B6D41685D202011
:1003900048656967687420536574706F696E74206E
:1003A0003235202020202020202020202020202026
:1003B0003236202020202020202020202020202015
:1003C000436F6D7061737320536574706F696E74E1
:1003D0004932432D4572726F722020202020202048
:1003E000424C204C696D6974202020202020202060
:1003F0004750535F4E69636B20202020202020202F
:100400004750535F526F6C6C20202020202020200A
:1004100021212120494E434F4D50415449424C45E2
:1004200020212121002E000A0D20444143206F721B
:1004300020493243204552524F5221204368656380
:100440006B204932432C2033567265662C20444180
:100450004320616E6420424C2D4374726C005B2516
:10046000695D005B25695D002B204D696B726F4BE8
:100470006F70746572202B0048573A5625642E25FC
:10048000642053573A25642E256425630053657410
:1004900074696E673A2564202573004D697865722A
:1004A000204572726F7221004861726477617265D3
:1004B000204572726F7220313A2564202121004D4F
:1004C000697373696E6720424C2D4374726C3A25D0
:1004D0006421210021204E432D4552523A202532DD
:1004E0006420212000493243204552524F5221219D
:1004F00021004865696768743A20202535690053F2
:100500006574706F696E743A253569005072657351
:10051000737572653A253569004F66667365743A7E
:1005200020202535690048656967687420636F6E0F
:1005300074726F6C0044495341424C4544006163FE
:10054000742E2062656172696E67004E69636B3A52
:1005500020202020202025356900526F6C6C3A2025
:10056000202020202025356900436F6D7061737352
:100570003A202020253569004B25693A2534692029
:10058000204B25693A25346920004E693A253469A3
:100590002020526F3A253469200047733A25346988
:1005A000202047693A253469200050313A253469C2
:1005B000202050323A253469200050333A253469DE
:1005C000202050343A25346920004779726F202D5D
:1005D0002053656E736F72004E69636B253469201A
:1005E000282533692E25692900526F6C6C253469E2
:1005F00020282533692E256929004769657225342D
:1006000069202825336929004E69636B20253469E8
:1006100020282533692E25782900526F6C6C2025FF
:10062000346920282533692E2578290059617720DF
:1006300020253469202825336929004E69636B2001
:100640002534692028253369292825336929005252
:100650006F6C6C20253469202825336929282533BF
:1006600069290059617720202534692028253369BC
:1006700029282533692900414343202D2053656EE5
:10068000736F72004E69636B20253469202825330F
:10069000692900526F6C6C20253469202825336944
:1006A00029005A2020202025346920282533692953
:1006B00000566F6C746167653A2020202533692EDF
:1006C000253169560043757272656E743A20202098
:1006D0002533692E2531694100506F7765723A20C4
:1006E00020202020253469570044697363686172B3
:1006F00067653A202535696D416800526563656913
:100700007665720052432D525353493A20202020DF
:100710002534690052432D5175616C6974793A2012
:100720002534690052432D4368616E6E656C733ADF
:1007300025346900436F6D70617373004D61676E9E
:1007400065743A202020253569004779726F3A2078
:100750002020202025356900536574706F696E7400
:100760003A2025356900506F746925693A202025A3
:10077000336900506F746925693A20202533690078
:10078000536572766F202000536574706F696E74C4
:10079000202025336900506F736974696F6E3A20A9
:1007A0002533690052616E67653A2533692D25331B
:1007B0006900424C2D4374726C204572726F7273E3
:1007C000200025336420253364202533642025331D
:1007D000642000424C2054656D70657261747572BE
:1007E00065002533642025336420253364202533B8
:1007F000642000424C2D4374726C20666F756E64E9
:100800002000202563202020256320202025632030
:100810002020256320002025632020202563202020
:100820002025632020202563200020256320202010
:100830002D2020202D2020202D200031300031318E
:1008400000313200466C696768742D54696D65200B
:100850002000546F74616C3A2535756D696E0041E6
:1008600063743A20202535756D696E0028726573B2
:10087000657429000A0D47656E65726174696E675B
:100880002064656661756C7420506172616D657479
:10089000657220536574202564000A0D5573696ED6
:1008A0006720506172616D657465722053657420B4
:1008B0002564000A0D47656E65726174696E672074
:1008C00064656661756C74204D6978657220546149
:1008D000626C65000A0D4D697865722D436F6E6616
:1008E00069673A202725732720282575204D6F74C6
:1008F0006F727329000A0D3D3D3D3D3D3D3D3D3D3F
:100900003D3D3D3D3D3D3D3D3D3D3D3D3D3D3D3D17
:100910003D3D3D3D3D000A0D414343206E6F742037
:1009200063616C69627261746564210D0A00000084
:100930008F001E01AD013B02CA025803E603740496
:1009400002058F051B06A7063307BE074808D20815
:100950005B09E3096B0AF20A780BFD0B810C040DAD
:10096000860D070E870E060F840F00107B10F51002
:100970006E11E5115B12CF124213B31323149214BC
:10098000FE146A15D3153B16A11605176717C8176D
:1009900027188318DE1837198E19E319361A871AA3
:1009A000D61A231B6E1BB61BFD1B411C831CC31CCC
:1009B000001D3C1D751DAB1DE01D121E421E6F1E4D
:1009C0009A1EC31EE91E0D1F2E1F4D1F691F841F77
:1009D0009B1FB01FC31FD31FE11FEC1FF51FFB1F81
:1009E000FF1F002003010000C36B00020101B26C75
:1009F00001030202466D02000303A36D2532692E36
:100A00002531695600253364256320253033646D14
:100A1000256300537461747573004552524F523A06
:100A2000202532642000253469202532693A25309A
:100A30003269002534696D2563002533692025332B
:100A40006920253369202533690025336920253342
:100A50006920253369202533690054656D706572FE
:100A60006174757265732020202000256343202067
:100A7000202020002532692E25316956202025337B
:100A8000692E253169410025346957202536696D65
:100A90004168002532756D2F73205361743A2564C7
:100AA000200020203344004E6F46780044475053C6
:100AB00000486F6D653A2533646D202533642563E6
:100AC000202563004E6F204E6176694374726C215D
:100AD000000A0D7777772E4D696B726F4B6F7074CC
:100AE00065722E64652028632920486953797374E0
:100AF000656D7320476D6248000A0D746865207546
:100B00007365206F66207468697320736F667477ED
:100B1000617265206973206F6E6C79207065726DEB
:100B20006974746564200A0D6F6E206F726967695D
:100B30006E616C204D696B726F4B6F707465722DB6
:100B400048617264776172650047726175706E65A5
:100B50007220486F5454004143542044534C004A7F
:100B600065746920736174656C6C69740053706599
:100B70006B7472756D20736174656C6C6974202878
:100B80004C6F77207265736F6C7574696F6E290096
:100B90005370656B7472756D20736174656C6C69EC
:100BA0007420283230343829005370656B747275A4
:100BB0006D20736174656C6C6974004D756C74693B
:100BC0007369676E616C2050504D000A0D52656369
:100BD00065697665723A2000756E6B6E6F776E2E62
:100BE000205573696E672050504D2E2E2E006E6F6B
:100BF0007420737570706F727465642062792068F8
:100C00006172647761726521000A0D3D3D3D3D3D95
:100C10003D3D3D3D3D3D3D3D3D3D3D3D3D3D3D3D04
:100C20003D3D3D3D3D3D3D3D3D3D3D3D3D3D000A64
:100C30000D466C69676874436F6E74726F6C0A0D51
:100C400048617264776172653A25642E25640A0DE5
:100C5000536F6674776172653A5625642E25642554
:100C60006320000A0D3D3D3D3D3D3D3D3D3D3D3D4B
:100C70003D3D3D3D3D3D3D3D3D3D3D3D3D3D3D3DA4
:100C80003D3D3D3D3D3D3D3D000011241FBECFEFAC
:100C9000D0E1DEBFCDBF11E0A0E0B1E0E0ECF5EFC8
:100CA00002C005900D92A83AB107D9F718E0A8EA5A
:100CB000B1E001C01D92AD3DB107E1F76AEAE2E0A3
:100CC000F0E081E2809357007491AE014F5F5F4F77
:100CD00020EF37EFDA019FE0F9012F5F3F4F84915A
:100CE0008D93915097FFF8CF773911F40000FECF24
:100CF000FA019EE0819168276095915097FFFACFA5
:100D00008889681721F0773911F40000FECF0E941E
:100D10004C070C94DF7A0C94000080912306E82F96
:100D2000FF27EE0FFF1FEF5AF84F808191818D5EF4
:100D30009F4F14F010920301808191818A5B9F4F35
:100D4000CCF4809103018823A9F481E0809303010E
:100D5000809116048F5F80931604853038F088EEFA
:100D600093E09093DD018093DC0104C066E970E0BC
:100D70000E94C4358091160499279093A40580930E
:100D8000A30508951F93CF93DF93182F882389F02D
:100D900080EF90E09F938F9381E892E19F938F93F0
:100DA000E091E203F091E30309950F900F900F900B
:100DB0000F9080914606823308F044C084EF91E0A2
:100DC0000E948F16EC01112329F0CE010E94981683
:100DD0008823D9F3C2E0D0E026E530E080911E01FF
:100DE00090911F018217930730F02196255D3F4FA8
:100DF000C730D10598F3809146069927C89F900186
:100E0000C99F300DD89F300D11242093000111236C
:100E1000D9F068EC70E08C2F0E94C435DF93CF933B
:100E200088EF90E09F938F9381E892E19F938F9357
:100E3000E091E203F091E30309958DB79EB7069622
:100E40008DBF02C080930001112311F18091000138
:100E50006AE00E94327A892F99279F938F9380911D
:100E600000010E94327A99279F938F9383E091E04B
:100E70009F938F9381E892E19F938F93E091E20398
:100E8000F091E30309952DB73EB7285F3F4F2DBF83
:100E9000DF91CF911F910895CFEFD0E1DEBFCDBF9D
:100EA0008824992414B815B807EE13E002531040B3
:100EB00017FFFCCF189B06C0199B02C08DE007C02E
:100EC0008BE005C0199B02C084E101C08AE08093D9
:100ED000020181E887B93E9A8FEF88B98BE184B926
:100EE00081E085B98EE38AB987E48BB9469A84B7E5
:100EF000877F84BF8091600088618093600010923A
:100F0000600084EC99E09093DD018093DC01109205
:100F1000E5021092E40210925607109255071092C3
:100F2000E7021092E6021092E9021092E802209184
:100F30000201243128F084EC94E0A0E0B0E004C089
:100F40008BE095E0A0E0B0E08093430190934401F2
:100F5000A0934501B09346012A3011F0243110F0DE
:100F6000289801C0289A0E94F8160E94C9160E946B
:100F700089120E941D320E943C1A81E00E94802D3D
:100F80000E94E5620E94976E0E94CB7680910201DA
:100F90008C3010F4299A01C0299878940E94922CE0
:100FA00080912402826080932402109227020E9482
:100FB000EA4084EF91E00E948F168C018091240218
:100FC00080FD05C0C8010E9498168823B9F38DE101
:100FD00091E09F938F93C1E8AC2EC2E1BC2EBF92EB
:100FE000AF92E091E203F091E303099580EA9FE07C
:100FF0000E948F168C01C0E0D0E00F900F900F90F0
:101000000F90B3EFEB2EB6E0FB2EA7EACA2EA6E0B8
:10101000DA2E0E94EA408091240280FD05C0C801BA
:101020000E9498168823B9F3F60180811816ACF453
:101030000BC00E94EA408091240280FD05C0C801D7
:101040000E9498168823B9F3C8010E949816882335
:1010500021F4F7018081882364F7F701808187FFFD
:1010600018C02196DF93CF9321978FE291E09F9351
:101070008F93BF92AF92E091E203F091E303099561
:101080008091A9018F5F8093A9018DB79EB70696C5
:101090008DBF2196E4E0F0E0CE0EDF1E88E090E008
:1010A000E80EF91ECC30D10508F4B3CFC0E0D0E093
:1010B00000EF16E0F7EAEF2EF6E0FF2EF80183814D
:1010C00087FD1CC0F70180811816C4F42196DF93B8
:1010D000CF93219782E391E09F938F9381E892E1F0
:1010E0009F938F93E091E203F091E303099582E0EF
:1010F0008093DA018DB79EB706968DBFF801838184
:1011000080788383219684E090E0E80EF91E085FE2
:101110001F4FCC30D10590F280E591E09F938F93E3
:10112000C1E8D2E1DF93CF93E091E203F091E303D2
:101130000995909121068091A9010F900F900F9031
:101140000F90981728F48091FC0380618093FC0332
:1011500086E791E09F938F93DF93CF93E091E20333
:10116000F091E303099588EE93E00E948F168C01BD
:101170000E94421A0F900F900F900F90C8010E948A
:1011800098168823D9F386E991E09F938F93DF9394
:10119000CF93E091E203F091E303099580E00E9490
:1011A0008636809102010F900F900F900F908A3039
:1011B00011F0843110F0289801C0289A80ED97E052
:1011C0009093DD018093DC0185E5809318048EE027
:1011D00090E00E94C52A9927182F00278FE090E001
:1011E0000E94C52A080F111D1093AF010093AE0194
:1011F0008AE090E00E94C52A9927182F00278BE0EB
:1012000090E00E94C52A080F111D1093AD010093B4
:10121000AC010F5F1F4F39F08091AE019091AF018B
:101220008F5F9F4F41F41092AF011092AE01109268
:10123000AD011092AC018091AC019091AD019F93F2
:101240008F938091AE019091AF019F938F938BE923
:1012500091E09F938F93DF93CF93E091E203F0911E
:10126000E30309958DB79EB708968DBF8EEB91E08D
:101270009F938F93DF93CF93E091E203F091E30389
:10128000099580912F060F900F900F900F90E0918D
:10129000E203F091E30382FF07C08AEC91E09F93A1
:1012A0008F93DF93CF9308C086ED91E09F938F9348
:1012B00081E892E19F938F9309950F900F900F9083
:1012C0000F900E94801F88E893E190933E018093E5
:1012D0003D0161E0F62EF09217048F2D0E94C206A8
:1012E000809149060E94157688EE91E09F938F9336
:1012F000DF93CF93E091E203F091E303099580ED52
:1013000097E00E948F168C018AEF90E00E948F1662
:1013100083E080937B051092A80180918C060F904A
:101320000F900F900F9084FF02C0F092B001809157
:10133000B201882311F04798FECF8091E001882305
:1013400009F4EBC180911001882309F4E6C11092E1
:10135000E00180911604882319F00E948D0602C0D6
:101360000E9420440E94EA40209102012A3011F09C
:10137000243110F0289801C0289A8091D80288233F
:1013800031F08091D80281508093D8020EC08091B4
:101390006F00806280936F00109252071092510785
:1013A0008091FC0388608093FC0380913D019091C3
:1013B0003E01019790933E0180933D0180913D0154
:1013C00090913E01892B21F0809125028823C9F15B
:1013D00080913D0190913E01892BD9F40E94AA2D64
:1013E00085E090E090933E0180933D018091B505AA
:1013F0009091B60501969093B6058093B5058091BE
:10140000FC0381608093FC0380917C058260809363
:101410007C0580910801909109018F5F9F4FC1F475
:101420008091D7028823A1F088EA91E69093DD01AC
:101430008093DC0180E890E090930901809308019B
:1014400007C02A3011F0243110F0289801C0289AE2
:101450000E949D778091E001882309F05EC1809110
:101460000E01882311F00E940F170E94CC120E94D7
:101470001B0EC8010E949816882309F44AC10C5E0D
:101480001F4F80912502882349F08091FC038260E0
:101490008093FC0380917C0582600FC08091DC0109
:1014A0009091DD01892B59F480913D0190913E018D
:1014B000079728F080917C058D7F80937C05809133
:1014C000D802882361F08091B001882341F0109206
:1014D000B00188E893E19093DD018093DC01809175
:1014E0000501882321F08150809305012EC080934F
:1014F00022041092AE021092AD021092AC02109231
:10150000AB021092AA021092A9028091D8028823FD
:10151000E1F480910801909109018F5F9F4FA9F438
:101520002091B001223089F088E99AE39093DD019F
:101530008093DC0180E09CE0909309018093080196
:10154000222319F082E08093B00180919D01893CB3
:1015500048F0815080939D018091FC038B7F8093A4
:10156000FC033FC0809131088823F9F08091FC038F
:1015700084608093FC0389E08093AF03809108012D
:10158000909109018F5F9F4F81F48091D70288234A
:1015900061F088E99AE39093DD018093DC0180E0BB
:1015A00098EA90930901809308011092A603109283
:1015B000A5031092A4031092A3031092A203109209
:1015C0002408109263081092620810926508109225
:1015D00064088FEF9FEF90936108809360081092EA
:1015E0009D0180910001282F332780911E01909149
:1015F0001F0182179307CCF48091A202806280932E
:10160000A20280910801909109018F5F9F4FC1F460
:1016100080E797E19093DD018093DC0180E093E027
:1016200090930901809308010BC08091DC01909197
:10163000DD01892B29F48091A2028F7D8093A20283
:101640000E947E6784E08093DB018091A20281FD8D
:1016500005C05AEA852E55E0952E12C08091B10141
:101660008F5F8093B101813359F41092B101809161
:10167000AA019091AB0101969093AB018093AA01CE
:101680000894811C911CF2E78F16FBE09F0609F07D
:1016900040C0882499242091AE013091AF012F5F82
:1016A0003F4F3093AF012093AE018091AC019091F8
:1016B000AD0101969093AD018093AC01832F9927E2
:1016C000682F8EE090E00E94CD2A8091AE0190912B
:1016D000AF019070682F8FE090E00E94CD2A80913A
:1016E000AC019091AD01892F9927682F8AE090E095
:1016F0000E94CD2A8091AC019091AD019070682F2D
:101700008BE090E00E94CD2A84E190E00E948F1649
:101710008C010E94CE670E94AE6E8091DB0188230F
:1017200009F005CE0E94066302CE1F920F920FB6FB
:101730000F9211248F939F93EF93FF938091070152
:101740008823E1F48091CC019091CD010196909392
:10175000CD018093CC01FC01EF52FB4FE081ED30D5
:1017600019F08A3A910539F41092CD011092CC010A
:1017700081E080930701E093C60004C01092CD0180
:101780001092CC01FF91EF919F918F910F900FBE1E
:101790000F901F9018951F920F920FB60F92112461
:1017A0002F933F934F935F936F937F938F939F9369
:1017B000AF93BF93CF93EF93FF9390E08091B201EB
:1017C000813029F48091C6008093CE00CCC08091F6
:1017D000B201823029F48091C60080932504C3C0F1
:1017E0008091C6008093C4015091D2015A3A10F002
:1017F0009093D3018091C4018D3009F065C0809130
:10180000D301823009F060C09093D301852F9927CE
:101810008B5D9B4FFC01329740812091CE0130912E
:10182000CF01241B3109DC0111978C91281B310950
:10183000C9019F709093CF018093CE0146E09695A9
:1018400087954A95E1F7982F935C9093D0012F7379
:101850003070235C2093D1018081981729F48C91FA
:10186000281711F491E006C090E08091C1018F5FCC
:101870008093C101C091C301CC2309F074C09923A6
:1018800009F471C081E08093C301580F5093C001E7
:101890005150E52FFF27EB5DFB4F8DE0808380915A
:1018A0002704823509F05FC00E94801F88E190E024
:1018B0002CE00FB6F894A895809360000FBE20939B
:1018C0006000C093DA014FC02091D301822F992785
:1018D00081309105F9F0823091051CF4892B21F0BB
:1018E00040C0029711F13DC08091C401833239F4A8
:1018F0008091C301882319F481E08093D301809102
:10190000C4018093250481E08093D2018091C401B9
:10191000992722C02F5F2093D301E52FFF27EB5D8E
:10192000FB4F8091C401808309C0E52FFF27EB5D49
:10193000FB4F8091C40180835A3A20F45F5F50933B
:10194000D20102C01092D3012091C4018091CE0136
:101950009091CF01820F911D9093CF018093CE0182
:1019600002C01092D301FF91EF91CF91BF91AF913F
:101970009F918F917F916F915F914F913F912F91A7
:101980000F900FBE0F901F901895AC01A0E0B0E033
:101990009D01A817B90748F4E1EDF4E08191280F03
:1019A000311D1196A417B507C8F33F70FD01EF5222
:1019B000FB4FC90156E0969587955A95E1F7835CF0
:1019C00080831196FD01EF52FB4F2F733070822FF1
:1019D000835C8083AE52BB4F8DE08C9310920701E5
:1019E0008091D1048093C6000895A0E0B0E0EBEFB1
:1019F000FCE00C94AB7A2C859D850E85BB2483E29C
:101A00008093D1049F599093D2042093D30433E060
:101A1000E32EF12C002309F49EC0CF84D888BE01A8
:101A20006D5E7F4FA989BA890150109709F493C060
:101A30001097B9F0F601EB0DF11DB3949081119759
:101A400091F4002349F1FB016E5F7F4FDB01C08001
:101A5000D1806E5F7F4F0D90BC91A02DBB240150B3
:101A600002C090E019C01097B9F0F601EB0DF11D1E
:101A7000B3944081119791F4002341F1FB016E5F13
:101A80007F4FDB01C080D1806E5F7F4F0D90BC9196
:101A9000A02DBB24015002C040E018C01097B1F047
:101AA000F601EB0DF11DB3941081119781F4002321
:101AB00071F0FB013296DB01CD90DC90BF016E5FCF
:101AC0007F4FA081B181BB24015001C010E0F7011C
:101AD000EF52FB4F892F86958695835C808308940F
:101AE000E11CF11CF701EF52FB4F892F99278370FE
:101AF000907024E0880F991F2A95E1F755279A01E5
:101B000094E0369527959A95E1F7822B835C808344
:101B10000894E11CF11CF701EF52FB4F4F7050701D
:101B2000440F551F440F551F812F992726E0969586
:101B300087952A95E1F7842B835C80830894E11CC8
:101B4000F11CF701EF52FB4F1F73135C10830894D5
:101B5000E11CF11C6ACFC7010E94C50CE9E00C949E
:101B6000C77AA3E07A2F4091C0014650442309F47C
:101B700058C0E72FFF27EB5DFB4F80818D537F5FC0
:101B8000E72FFF27EB5DFB4F20812D537F5FE72F72
:101B9000FF27EB5DFB4F30813D537F5FE72FFF2732
:101BA000EB5DFB4F60816D537F5F9927880F991F15
:101BB000880F991F522F52955F70582B822F9927AB
:101BC0008F709070F4E0880F991FFA95E1F7232F3A
:101BD00026952695282B832F992783709070E6E011
:101BE000880F991FEA95E1F7682B41504F3FC9F0E4
:101BF000EA2FFF27EB5DFB4F5083AF5F41504F3F14
:101C000081F0EA2FFF27EB5DFB4F2083AF5F415050
:101C10004F3F39F0EA2FFF27EB5DFB4F6083AF5F4B
:101C2000A5CF88E294E09093BF018093BE01A350BA
:101C3000A093BD010895A2E0B0E0E1E2FEE00C94C3
:101C4000B17A8091C301882309F457C40E94B10D71
:101C500080912604823609F023C3809127049927B6
:101C60008037910509F4AFC081379105C4F48A36F5
:101C7000910509F480C28B36910544F48B349105AB
:101C800071F18636910509F45FC10AC38D3691055D
:101C900009F469C08E36910509F44DC001C384373B
:101CA000910541F1853791054CF48137910509F48F
:101CB00091C08337910509F4DFC0F2C287379105DF
:101CC00009F41BC2883791052CF48537910509F476
:101CD000D7C1E6C28937910509F46DC1E1C2E0912F
:101CE000BE01F091BF018081918190939101809319
:101CF0009001D6C28091C001A091BE01B091BF01F8
:101D0000853140F080E1E0E0F4E00D9001928A95A9
:101D1000E1F70DC08D919D910D90BC91A02D809308
:101D2000000490930104A0930204B093030480EF95
:101D30008093BB014BC0809107018823E1F38DE4C0
:101D400090E09F938F938AE996E09F938F9381E031
:101D50008F938F938EE48F930E94F50C8DB79EB76F
:101D600007968DBF9DC2A091BE01B091BF011C918D
:101D7000113081F48DE4EAE9F6E00D9001928A9544
:101D8000E1F70E94CF2B19838091FC038F7E809313
:101D9000FC0301C01982809107018823E1F381E0EF
:101DA00090E09F938F93CE0101969F938F9381E054
:101DB0008F938F938DE48F930E94F50CADB7BEB7D0
:101DC0001796ADBF6DC281E08093C6018FEF8093FF
:101DD000050166C2E091BE01F091BF01E0818E2F46
:101DE0008A508A3058F48983882311F481E003C033
:101DF000863010F085E0898361E00EC08E2F84511B
:101E00008A3070F48983882311F481E003C086301E
:101E100010F085E0898360E089810E944F2C12C018
:101E2000E983EF3F19F40E94322C8983898188234A
:101E300011F481E003C0863010F085E08983898148
:101E40000E94E32A809107018823E1F387E790E06D
:101E50009F938F9382E296E09F938F9381E090E02F
:101E60009F938F93CE0101969F938F9382E08F93E0
:101E700081E08F9381E577C12091BE013091BF0150
:101E8000D9018C918150853008F045C0F9018181DC
:101E9000883509F040C08091D7028823E1F52F5F93
:101EA0003F4F87E7E2E2F6E0D9010D9001928A9573
:101EB000E1F7F90182910E944C2B809163069927EA
:101EC000AA27BB27BC01CD0124EC39E040E050E05B
:101ED0000E94137ADC01CB018093880190938901E1
:101EE000A0938A01B0938B01809164069927AA2759
:101EF000BB27BC01CD010E94137ADC01CB0180938A
:101F0000840190938501A0938601B09387010E947C
:101F1000322C898301C01982809107018823E1F363
:101F200081E090E09F938F93CE0101969F938F93D2
:101F300081E08F938F9383E58F930E94F50C8DB78B
:101F40009EB707968DBF26C0E091BE01F091BF01FC
:101F5000E0818E2F8150853018F48E2F0E94E32A65
:101F60000E94322C8983809107018823E1F381E06C
:101F700090E09F938F93CE0101969F938F9381E082
:101F80008F938F9386E48F930E94F50CADB7BEB705
:101F90001796ADBF8091D702882329F46EE670E0D2
:101FA00089810E94C43580E00E94C2068091490662
:101FB0000E94157675C1E091BE01F091BF0180814C
:101FC000992787FD909590936C0780936B0781818B
:101FD000992787FD909590936E0780936D07828176
:101FE000992787FD90959093700780936F07838161
:101FF000992787FD9095909372078093710784814C
:10200000992787FD90959093740780937307858136
:10201000992787FD90959093760780937507868121
:10202000992787FD9095909378078093770787810C
:10203000992787FD909590937A07809379078085FB
:10204000992787FD909590937C0780937B078185E6
:10205000992787FD909590937E0780937D078285D1
:10206000992787FD90959093800780937F078385BC
:10207000992787FD9095909382078093810710C1DF
:10208000E091BE01F091BF0180810E9476318A8388
:10209000882319F481E0898301C0198280910701A6
:1020A0008823E1F388E090E09F938F9388EE96E099
:1020B0009F938F9321E030E03F932F938091BE0157
:1020C0009091BF019F938F933F932F93CE010296E0
:1020D0009F938F933F932F93CE01820F931F9F93D4
:1020E0008F9384E08F9381E08F9385E58F930E9497
:1020F000F50CEDB7FEB773963CC08091BD018930F9
:1021000008F4CEC02091BE013091BF012F5F3F4F38
:1021100088E0A8EEB6E0F90101900D928A95E1F70A
:10212000D9018E910E94CC308A83882319F481E0F2
:10213000898301C01982809107018823E1F321E09E
:1021400030E03F932F93CE0102969F938F933F935E
:102150002F93CE01820F931F9F938F9382E08F93D3
:1021600081E08F9387E58F930E94F50CEDB7FEB762
:102170003B96EDBF95C08091D702882309F090C0AF
:102180000E94C8758983823019F0843009F088C0B4
:1021900020E430E0F8948091C1008F738093C100F7
:1021A0008091C9008F738093C9008091C100877EA0
:1021B0008093C1008091C900877E8093C90080917F
:1021C000C80087FF03C08091CE00F9CF8091C00086
:1021D00087FF03C08091C600F9CFE091BE01F09166
:1021E000BF01E081E13021F482E08093B2012EC092
:1021F000E43611F421E830E081E08093B201832FCE
:1022000099278093CD002093CC008091CD008093BE
:10221000C5008091CC008093C4008091CA008F7D5E
:102220008093CA008091CA008F7E8093CA008091FB
:10223000C9008B7F8093C9008091CA00846080931D
:10224000CA008091CA0082608093CA008091CA004F
:10225000877F8093CA008091C200877F8093C200ED
:102260008091C9008E7F8093C9008091C1008861F0
:102270008093C1008091C90088618093C9008091DA
:10228000C10080688093C1008091C90080688093FC
:10229000C90010926E0010926F0010927000789436
:1022A0008091270499278436910509F4BBC08536AF
:1022B0009105ACF48136910509F46FC08236910521
:1022C0002CF48B34910509F45DC00FC18236910561
:1022D00009F470C08336910509F47FC006C18C36BD
:1022E000910509F4EDC08D3691054CF487369105C2
:1022F00009F4F8C08836910509F4B2C0F6C08437F5
:10230000910529F08637910509F4E8C0EEC0809167
:10231000C001A091BE01B091BF01803140F080E1C9
:10232000E0E0F4E00D9001928A95E1F70DC08D9107
:102330009D910D90BC91A02D809300049093010479
:10234000A0930204B0930304809107018823E1F372
:102350001F92809104018F9384E58F930E94F50C66
:102360008AEF8093BB018FEF8093050180EA9FE0A5
:102370000E948F169093B4018093B3010F900F9039
:102380000F90B3C0E091BE01F091BF0180819181B7
:102390009093910180939001A8C0E091BE01F091CB
:1023A000BF01808180930601803298F08FE1809395
:1023B00006010FC0A091BE01B091BF018BE0E8E122
:1023C000F4E00D9001928A95E1F7809121048093C9
:1023D000BD058FEF8093050188C08091B701909172
:1023E000B801892B89F4E091BE01F091BF01E08131
:1023F000EE2351F08AE0E89FC00111240E948F165D
:102400009093F3038093F203E091BE01F091BF013A
:1024100090818AE0989FC00111249093B801809325
:10242000B70115C08FEF80930501E091BE01F091D7
:10243000BF0190818AE0989FC00111249093BA0156
:102440008093B901892B19F081E08093C80180EA5B
:102450009FE00E948F169093B4018093B30145C012
:102460008FEF80930501E091BE01F091BF01908153
:1024700097FD08C082E08093C5011092B6011092CA
:10248000B5011AC0909580911D02892B80931D0281
:1024900091818AE0989FC00111249093B6018093A6
:1024A000B50184E08093C50180EA9FE00E948F1609
:1024B0009093B4018093B30181E08093C90115C06A
:1024C0008FEF80930501E091BE01F091BF01808103
:1024D00080931E0281E08093CA0107C081E080934F
:1024E000C70103C081E08093CB011092C301109219
:1024F000BF011092BE011092BD01E3E0CE5F0C94CB
:10250000CD7A982F8091C00085FFFCCF9093C600B4
:1025100008950F931F9388E18093C1008091C000BC
:1025200082608093C0008091C10080688093C10068
:102530008091C10080648093C10000E010E00093AE
:10254000C5008AE290E08093C4008091B901909127
:10255000BA010E948F169093F5038093F4038CEDDB
:1025600090E00E948F16909324048093230410928D
:10257000F60386E58093F7031092FA038BE08093CD
:10258000F8031092F9031093BF010093BE0110925B
:10259000BD011F910F910895A0E1B0E0E2EDF2E1DD
:1025A0000C94AE7A80910701882309F4C1C280910E
:1025B000B3019091B4010E949816882361F01092A3
:1025C000B6011092B5011092BA011092B9011092A1
:1025D000B8011092B7018091B5019091B601892B95
:1025E00041F08091CF049091D0040E9498168823E6
:1025F00029F48091C901882309F460C08091070102
:10260000882309F45BC08091C50101ED15E0843099
:10261000A8F00E94961F80E590E09F938F931F93F0
:102620000F9381E08F938F9388E48F930E94F50C32
:102630002DB73EB7295F3F4F2DBF34C010921F0208
:1026400080E194E09F938F9389E89FE19F938F931C
:10265000E091E203F091E303099584E190E09F9318
:102660008F931F930F9381E090E09F938F9385EC5E
:1026700091E09F938F9382E08F9381E08F9388E422
:102680008F930E94F50C8091C501982F8F5F8093E6
:10269000C5012DB73EB7215F3F4F2DBF943010F0DD
:1026A0001092C5018091B5019091B6010E948F16DC
:1026B0009093D0048093CF041092C9018091CA01F5
:1026C000882351F180910701882331F10E94961FE0
:1026D00080E590E09F938F9381ED95E09F938F939A
:1026E00021E030E03F932F9380E291E09F938F931E
:1026F0003F932F938EE192E09F938F9383E08F938C
:1027000081E08F938CE48F930E94F50C1092CA01A4
:102710008DB79EB70F968DBF8091C7018823D1F0EA
:10272000809107018823B1F08AE090E09F938F9316
:1027300086EF93E09F938F9381E08F938F9386E54D
:102740008F930E94F50C1092C7012DB73EB7295FF9
:102750003F4F2DBF8091CB018823D9F08091070195
:102760008823B9F08BE090E09F938F9388E194E009
:102770009F938F9381E08F93809104018F9387E4DF
:102780008F930E94F50C1092CB018DB79EB70796E0
:102790008DBF80912304909124040E949816882371
:1027A00009F461C080910701882309F45CC080911D
:1027B0003E069927880F991F880F991F7C010027D3
:1027C000F7FC0095102F8091320390913303A09174
:1027D0003403B0913503BC01CD01A80197010E94DB
:1027E000877A309311042093100480912A039091EA
:1027F0002B03A0912C03B0912D03BC01CD01A801A6
:1028000097010E94877A30931304209312048091D9
:10281000B702809314048091B6028093150488E077
:1028200090E09F938F9380E194E09F938F9381E05A
:102830008F9383E08F938BE68F930E94F50C8091AA
:1028400016042DB73EB7295F3F4F2DBF853018F0D6
:1028500086E08093160483E690E00E948F169093A2
:102860002404809323048091B9019091BA01892BAB
:1028700041F08091F4039091F5030E94981688230B
:1028800021F48091C801882339F1809107018823C0
:1028900019F10E94AE3482E490E09F938F938BE70E
:1028A00095E09F938F9381E08F938F9384E48F9330
:1028B0000E94F50C1092C8018DB79EB707968DBF88
:1028C0008091B9019091BA01009731F00E948F1662
:1028D0009093F5038093F4038091B7019091B80130
:1028E000892B09F4B8C08091F2039091F3030E9400
:1028F0009816882309F4AFC080910701882309F452
:10290000AAC080913E069927880F991F880F991FAA
:102910007C010027F7FC0095102F809132039091E5
:102920003303A0913403B0913503BC01CD01A8015C
:1029300097010E94877A3093E5032093E403809106
:102940002A0390912B03A0912C03B0912D03BC017D
:10295000CD01A80197010E94877A3093E703209365
:10296000E6032091190830911A0840911B085091F4
:102970001C08DA01C90163E0880F991FAA1FBB1F59
:102980006A95D1F7820F931FA41FB51F820F931F63
:10299000A41FB51F2091430130914401409145018E
:1029A00050914601BC01CD010E94877A3093E90322
:1029B0002093E8038091FA029091FB02A091FC021F
:1029C000B091FD0249E0B595A795979587954A95F1
:1029D000D1F78093EA038091F6029091F702A091DB
:1029E000F802B091F90239E0B595A79597958795CA
:1029F0003A95D1F78093EB03809102039091030302
:102A0000A0910403B091050329E0B595A79597958A
:102A100087952A95D1F78093EC038EE090E09F9301
:102A20008F9384EE93E09F938F9381E08F938F93A6
:102A300083E48F930E94F50C8091B7019091B801C7
:102A40000E948F169093F3038093F2032DB73EB745
:102A5000295F3F4F2DBF809106018F3F71F199276C
:102A600004E0880F991F0A95E1F7805F9D4F40E1D0
:102A700050E0BC01CE0101960E94667880E190E0B2
:102A80009F938F93CE0101969F938F9381E090E067
:102A90009F938F9386E091E09F938F9382E08F9333
:102AA00081E08F9381E48F930E94F50C8FEF8093E8
:102AB00006018DB79EB70B968DBF8091BD0588230B
:102AC000D1F0809107018823B1F081E090E09F93DD
:102AD0008F938DEB95E09F938F9381E08F938F93EE
:102AE00082E48F930E94F50C1092BD052DB73EB77E
:102AF000295F3F4F2DBF8091C6018823C9F0809187
:102B000007018823A9F084E390E09F938F9381E5E8
:102B100097E09F938F9381E08F938F9380E58F93BE
:102B20000E94F50C1092C6018DB79EB707968DBF17
:102B3000E6E0C05F0C94CA7A1F920F920FB60F9214
:102B400011242F933F935F936F937F938F939F9362
:102B5000AF93BF93EF93FF9320E08091DB01882335
:102B600029F08091DB0181508093DB018091C203C9
:102B7000882319F081508093C2038091E301815032
:102B80008093E3018F3F09F05BC089E08093E3010C
:102B90008091E1019091E20101969093E20180938E
:102BA000E10180910F018F5F817080930F01882375
:102BB00019F481E08093E001349903C081E08093AF
:102BC000E4018091DC019091DD01892B21F180915C
:102BD000DC019091DD010B9750F08091DC01909128
:102BE000DD010A979093DD018093DC0104C010920F
:102BF000DD011092DC018091DC019091DD012091DA
:102C000008013091090182239323892B11F021E0DF
:102C100008C020E006C08FEF9FEF909309018093DA
:102C2000080180910201222331F08A3011F45A9A6E
:102C300007C0479A05C08A3011F45A9801C04798D6
:102C40008091E401882309F45AC020919D01222338
:102C500009F055C08091090883FF51C086B19927BA
:102C6000FC01E071F07084FF13C08091DE0190914F
:102C7000DF0101969093DF018093DE018091DE01F8
:102C80009091DF01895E9340D0F12093E40137C039
:102C90008091DE019091DF01892B69F18091DE0145
:102CA0009091DF018A56914030F58091DE0190913C
:102CB000DF0169E270E00E943E7A8091DE0190912E
:102CC000DF01860F971F9093DF018093DE018091D3
:102CD000DE019091DF010B9750F08091DE01909121
:102CE000DF010A97909391018093900104C0F093C3
:102CF0009101E09390011092DF011092DE01FF91AB
:102D0000EF91BF91AF919F918F917F916F915F9163
:102D10003F912F910F900FBE0F901F90189520910B
:102D2000E1013091E201280F391FC9010196089590
:102D30002091E1013091E201821B930B892F9927A9
:102D40008695807490700895CF93DF930E948F16BC
:102D5000EC01CE010E9498168823D9F3DF91CF9120
:102D60000895CF93DF930E948F16EC0109C08091E4
:102D70001001882329F0909310018FEC80937A0042
:102D8000CE010E949816982F882389F3DF91CF9166
:102D900008959FB7F8945F983E9A469A8091B00044
:102DA0008F708093B0008091B00083608093B000FA
:102DB0008091B1008B738093B1008091B1008B60E2
:102DC0008093B1001092B2008FEF8093B300809196
:102DD000B00080688093B000809170008A7F8093FB
:102DE0007000809170008260809370009FBF089592
:102DF0008AE090E00E948F169093EA018093E901A7
:102E000082E085BD83EA84BD17BC84EB88BD86E083
:102E100086BD80916E00816080936E000895A0E071
:102E2000B0E0E5E1F7E10C94AD7A80915906E82F26
:102E3000FF27E75BFE4F9681D08080910E01A92F7E
:102E4000BB27A7FDB095CB2FDB2F813009F0DDC06C
:102E50002091320330913303409134035091350374
:102E6000BD01CE010E94137A97FF04C061587F4FC5
:102E70008F4F9F4F7B018C01F7E015950795F794D5
:102E8000E794FA95D1F78D2D992787FD9095A92F75
:102E9000B92F20912A0330912B0340912C0350919C
:102EA0002D03BC01CD010E94137A97FF04C0615825
:102EB0007F4F8F4F9F4FE7E0959587957795679563
:102EC000EA95D1F7F801E701C61BD70BE80BF90B20
:102ED0002091AD033091AE03C90153E0880F991FD3
:102EE0005A95E1F7821B930BAA2797FDA095BA2F5D
:102EF000C81BD90BEA0BFB0B809150069927AA2718
:102F0000BB27BC01CD019E01AF010E94137A97FF40
:102F100004C061507E4F8F4F9F4FFC01EB0149E091
:102F2000F595E795D795C7954A95D1F780916F01AB
:102F3000992736E0880F991F3A95E1F740910C01E7
:102F400050910D01209158063327841B950BB90130
:102F50000E94527A80910C0190910D01860F971F6B
:102F600090930D0180930C0180910C0190910D01C3
:102F700097FD0F9624E0959587952A95E1F7909314
:102F8000D7018093D60180918B0680FF07C0809186
:102F9000D6019091D7018C0F9D1F06C08091D6015C
:102FA0009091D7018C1B9D0B9093D7018093D601F4
:102FB00080915106282F3327220F331F220F331FF2
:102FC0008091D6019091D701821793077CF0809170
:102FD0005206282F3327220F331F220F331F8091D1
:102FE000D6019091D7012817390724F43093D701DF
:102FF0002093D60180910201843108F4C2C08091EF
:103000000E018F5F80930E01BEC020912A03309184
:103010002B0340912C0350912D03BD01CE010E9442
:10302000137A97FF04C061587F4F8F4F9F4F7B01EA
:103030008C01C7E015950795F794E794CA95D1F7E9
:103040008D2D992787FD9095A92FB92F20913203B7
:10305000309133034091340350913503BC01CD01CD
:103060000E94137A9B01AC0197FF04C021583F4F87
:103070004F4F5F4FB7E05595479537952795BA95D0
:10308000D1F72E0D3F1D401F511F809154069927E7
:10309000AA27BB27BC01CD010E94137A97FF04C069
:1030A00061507E4F8F4F9F4FFC01EB01A9E0F595DA
:1030B000E795D795C795AA95D1F780916E01992785
:1030C00076E0880F991F7A95E1F740910A015091B7
:1030D0000B01209158063327841B950BB9010E94E0
:1030E000527A80910A0190910B01860F971F90935D
:1030F0000B0180930A0180910A0190910B0197FDC9
:103100000F9664E0959587956A95E1F79093D501C0
:103110008093D40180918B0681FF07C08091D401F8
:103120009091D5018C0F9D1F06C08091D401909184
:10313000D5018C1B9D0B9093D5018093D401809178
:103140005506282F3327220F331F220F331F80915C
:10315000D4019091D501821793077CF08091560697
:10316000282F3327220F331F220F331F8091D401C2
:103170009091D5012817390724F43093D501209375
:10318000D40110920E01E7E0CDB7DEB70C94C97AF6
:103190001F920F920FB60F9211242F933F934F93CC
:1031A0005F938F939F93EF93FF9380910201909190
:1031B000E501843108F04CC0992309F01CC18091CD
:1031C000B00086FF24C08091B0008F7B8093B00058
:1031D0008091D6019091D70187559E4F9093D90148
:1031E0008093D80125E08D3D920718F08CED95E095
:1031F00005C08757914030F487E791E09093D9015B
:103200008093D8018091D8019091D901BAC0809162
:10321000B00080648093B00080915706282F332738
:103220008DED96E0289FA001299F500D389F500DED
:103230001124CA012091E6013091E701821B930B12
:103240009093D9018093D80181E080930E01D0C082
:10325000992309F0D0C08091B00086FF97C080917B
:10326000B0008F7B8093B000E091E801EE23F1F491
:1032700080915706282F33278DED96E0289FA001D7
:10328000299F500D389F500D1124CA012091E6014D
:103290003091E701821B930B9093D9018093D80161
:1032A0001092E7011092E601469AA2C089EA93E0E3
:1032B0009093D9018093D8018E2F9927833091055F
:1032C000D9F08430910534F48130910549F00297AA
:1032D00061F020C08430910591F0059799F01AC0F3
:1032E0008091D6019091D70104C08091D401909132
:1032F000D50187559E4F1DC08091E50705C080917F
:10330000BF0702C08091EE079927880F991F880F89
:10331000991FEFCFFF27EE0FFF1FEF5AF84F2081C5
:103320003181220F331F8091D8019091D901820FF2
:10333000931F9093D9018093D8018091D8019091E7
:10334000D90155E08D3D950718F08CED95E005C04D
:103350008757914030F487E791E09093D9018093AB
:10336000D8012091D8013091D9012C5B30403093A5
:10337000D9012093D8018091E6019091E701820F55
:10338000931F9093E7018093E60132C08091B000D3
:1033900080648093B0008CEB90E09093D90180938F
:1033A000D8018091E6019091E70184549F4F90935A
:1033B000E7018093E6018091DA01882321F0809172
:1033C000D802882321F48091DA01823011F44698E2
:1033D00001C0469A8091E8018F5F8093E801909147
:1033E0005706981728F481E080930E011092E801A7
:1033F00081E08093E5012091D8013091D90141E02D
:103400002F37340730F08FEF8093B3002F5F3040B9
:103410000FC02F3F3105C9F0C0F0A9014F5F5040E8
:103420004F37510550F480E88093B3002058304066
:103430003093D9012093D80112C08FEF8093B3004D
:103440005093D9014093D8010AC08091D80180934C
:10345000B3001092D9011092D8011092E501FF91AA
:10346000EF919F918F915F914F913F912F910F908D
:103470000FBE0F901F90189510927C008FEC8093D8
:103480007A000895CF93DF931092EF0183E090E0EC
:103490000E94C52AC82FDD27C531D10508F02A971B
:1034A000C7BD84E690E00E94B1168091140190910E
:1034B00015018052934010F4C0E0D0E0CA3FD1051E
:1034C000F8F4C7BD82E390E00E94B11685E294E073
:1034D0009F938F9381E892E19F938F93E091E20312
:1034E000F091E303099580911401909115010F90DB
:1034F0000F900F900F908052934010F02196DECFE6
:10350000C093CE056C2F83E090E00E94CD2A80917D
:103510002F0680FF0AC08091CE058A508B3E28F08E
:103520008091FB0380648093FB03C7BD8CE291E034
:103530000E94B116DF91CF910895EF92FF921F93F1
:10354000CF9310E080ED97E00E948F167C01CCE8CD
:10355000133019F4CB3008F0C9E010E08091FF017E
:10356000909100028C5F934024F48091130181506C
:103570000AC08091FF01909100028750944034F07E
:10358000809113018F5F8093130101C011E080913E
:10359000FD019091FE018C5F934024F48091120113
:1035A00081500AC08091FD019091FE0187509440A6
:1035B00034F0809112018F5F8093120101C01F5F70
:1035C0008091FB019091FC018C5F934024F48091E9
:1035D000110181500AC08091FB019091FC0187503C
:1035E0009440C4F0809111018F5F8093110113C04A
:1035F00087E294E09F938F9381E892E19F938F936A
:10360000E091E203F091E30309950F900F900F9082
:103610000F905FC01F5F82E180932A028091240295
:103620008E7F8093240285EA8093BC0080911301F1
:103630008A3040F48091FB0381608093FB038AE031
:103640008093130180911301863F40F08091FB032A
:1036500081608093FB0385EF8093130180911201B9
:103660008A3040F48091FB0382608093FB038AE000
:103670008093120180911201863F40F08091FB03FC
:1036800082608093FB0385EF80931201809111018A
:103690008A3040F48091FB0384608093FB038AE0CE
:1036A0008093110180911101863F40F08091FB03CE
:1036B00084608093FB0385EF8093110180912A023F
:1036C000882339F0C7010E949816882309F090CF0B
:1036D000F5CF109210018FEC80937A008091100149
:1036E0008823E1F3CA3020F48AE090E00E94B1160A
:1036F000C15009F02DCF86E490E00E94B116CF9121
:103700001F91FF90EF9008951F920F920FB60F92A6
:103710001124EF92FF920F931F932F933F934F9398
:103720005F936F937F938F939F93AF93BF93EF9329
:10373000FF9380910802282F3327442755278F5F56
:1037400080930802F9012231310508F0B4C3E25C2C
:10375000FF4F0C94D97A809178009091790046C0FF
:1037600080917800909179002CC18091780090919F
:10377000790090930B0280930A0257C180913B031A
:1037800090913C032091780030917900821B930B3B
:103790009093BF058093BE058091BE059091BF05B3
:1037A00090931502809314025EC1809178009091ED
:1037B000790020913D0330913E03821B930B90933F
:1037C000CD058093CC058091CC059091CD0590934B
:1037D00017028093160271C380910E0290910F021E
:1037E0002091780030917900820F931F90930F02FF
:1037F00080930E0281E062C380910C0290910D02D1
:103800002091780030917900820F931F90930D02E0
:1038100080930C0284E052C380911E0190911F019D
:103820009C01220F331F280F391F8091780090913F
:10383000790063E070E00E943E7A260F371F3695CC
:1038400027953695279530931F0120931E0185E01B
:1038500035C3809178009091790040913703509161
:103860003803841B950B9093F6018093F5018091AA
:10387000F5019091F601029704F122E04E3E5207C5
:1038800084F4209109022B5F209309022550809136
:10389000A3029091A402845F914018F4215F2093C9
:1038A000090280910902853684F14F5F5F4F509382
:1038B000380340933703845626C08091F5019091D8
:1038C000F6018F5F9F4F0CF532E047325307ECF063
:1038D000209109022550209309022B5F8091A302B9
:1038E0009091A402845F914018F42F502093090214
:1038F000809109028C394CF4415050405093380368
:10390000409337038C598093090281E08093F4013E
:1039100080917800909179009093C5058093C405BB
:103920008091F5019091F6019C01442737FD409567
:10393000542F8091F2029091F302A091F402B09181
:10394000F502820F931FA41FB51F8093F20290937C
:10395000F302A093F402B093F5022091F2023091A9
:10396000F3024091F4025091F50257FF04C0215038
:103970003C4F4F4F5F4F6AE05595479537952795D8
:103980006A95D1F78091F2029091F302A091F4022E
:10399000B091F502821B930BA40BB50B8093F2023E
:1039A0009093F302A093F402B093F5022EC180919C
:1039B0000C0290910D022091780030917900820FD5
:1039C000931F90930D0280930C021092070278C20D
:1039D000809102018A3071F4809178009091790091
:1039E00020910A0230910B02820F931F0196969547
:1039F000879517C040910A0250910B02843158F00C
:103A00002091780030917900240F351F8FEF97E0D7
:103A1000821B930B06C08091780090917900840FEF
:103A2000951F9093FC018093FB0186E047C2809133
:103A30003B0390913C032091780030917900821BE8
:103A4000930B9093BF058093BE058091BE05909126
:103A5000BF052091140230911502820F931F90939D
:103A6000FA018093F90187E029C280917800909152
:103A7000790020913D0330913E03821B930B90937C
:103A8000CD058093CC058091CC059091CD052091FA
:103A9000160230911702820F931F9093F8018093C2
:103AA000F7010BC220910E0230910F028091780035
:103AB00090917900280F391F30930F0220930E0246
:103AC000809102018A3019F4220F331F04C0220FA3
:103AD000331F220F331F30930F0220930E022091C9
:103AE0000E0230910F02C90137FD079603E095954C
:103AF00087950A95E1F7909300028093FF018091EA
:103B0000100290911102820F931F97FD01969595D7
:103B10008795909311028093100220914703309172
:103B20004803821B930B90931D0180931C012091ED
:103B300005023091060280911C0190911D01280F11
:103B4000391F37FF02C02F5F3F4F359527953093C0
:103B50000602209305024ECE20910C0230910D02F8
:103B60008091780090917900280F391F30930D02D1
:103B700020930C02809102018A3019F4220F331F26
:103B800004C0220F331F220F331F30930D022093E6
:103B90000C0220910C0230910D02C90137FD0796ED
:103BA000F3E095958795FA95E1F79093FE01809360
:103BB000FD018091120290911302820F931F97FDD5
:103BC0000196959587959093130280931202209108
:103BD000450330914603821B930B90931B01809306
:103BE0001A01209103023091040280911A019091F0
:103BF0001B01280F391F37FF02C02F5F3F4F35953C
:103C00002795309304022093030283E057C110925A
:103C1000080281E0809310018091EB019091EC010A
:103C200001969093EC018093EB0180917800909144
:103C30007900909315018093140180911401909163
:103C40001501AA27BB272091180230911902409133
:103C50001A0250911B02280F391F4A1F5B1F209325
:103C600018023093190240931A0250931B0280915C
:103C70001C028F5F80931C02823108F41EC1809168
:103C8000160190911701A0911801B09119017C01C2
:103C90008D0163E0EE0CFF1C001F111F6A95D1F728
:103CA000E81AF90A0A0B1B0BE20EF31E041F151F7C
:103CB0008091EF01992787FD9095A92FB92FBC011D
:103CC000CD0126EC34E240E050E00E94137ADC01A2
:103CD000CB01E81AF90A0A0B1B0BD801C70104969D
:103CE000A11DB11DB7FF05C0D801C7010B96A11DCD
:103CF000B11D23E0B595A795979587952A95D1F79E
:103D00008093160190931701A0931801B0931901A5
:103D10008091C6059091C7057C010027F7FC0095AE
:103D2000102F8091160190911701A0911801B09168
:103D30001901E81AF90A0A0B1B0BE092D202F09261
:103D4000D3020093D4021093D5022091F001309158
:103D5000F1014091F2015091F30157FF04C0215F3E
:103D60003F4F4F4F5F4F84E05595479537952795C7
:103D70008A95D1F78091F0019091F101A091F20123
:103D8000B091F301821B930BA40BB50B8093F00150
:103D90009093F101A093F201B093F3018091F001AF
:103DA0009091F101A091F201B091F3018E0D9F1D50
:103DB000A01FB11F8093F0019093F101A093F20135
:103DC000B093F3018091F0019091F101A091F20183
:103DD000B091F301B7FF03C00F96A11DB11D14E010
:103DE000B595A795979587951A95D1F72091D20209
:103DF0003091D302281B390BC90137FF03C030951E
:103E000021953F4FAC01F3E0440F551FFA95E1F7C0
:103E100021383105C4F08091ED019091EE019C01B3
:103E2000E3E0220F331FEA95E1F7281B390B240F3B
:103E3000351F37FF02C0295F3F4F73E03595279547
:103E40007A95E1F717C08091ED019091EE019C0108
:103E500065E0220F331F6A95E1F7281B390B240F09
:103E6000351F37FF02C0215E3F4F45E0359527954E
:103E70004A95E1F73093EE012093ED01809118020D
:103E800090911902A0911A02B0911B02B7FF03C0D2
:103E90000196A11DB11DB595A7959795879580931E
:103EA000180290931902A0931A02B0931B0289E0A2
:103EB00080931C0202C01092080282E080930702E5
:103EC0008091070280937C0080910802882319F07A
:103ED0008FEC80937A00FF91EF91BF91AF919F910A
:103EE0008F917F916F915F914F913F912F911F9192
:103EF0000F91FF90EF900F900FBE0F901F901895AD
:103F000090E2E1EDF5E08FE49193815087FFFCCFE3
:103F1000089590911F02903540F4E92FFF27EF524A
:103F2000FA4F80839F5F90931F020895AF92BF92D4
:103F3000CF92DF92FF920F931F93CF93DF93209145
:103F40001D0220FF0AC080911E02882311F08150BB
:103F500002C08091200180931E0221FF0CC090912D
:103F60001E0280912001981719F410921E0203C0BE
:103F70009F5F90931E02822F992780FF04C081FFCC
:103F800002C010921E020E94801F80911E02282FE4
:103F90003327C9E8CC2ECFE1DC2EC091E203D091CB
:103FA000E3038A3098F481E180931F023F932F93BB
:103FB0008EE594E09F938F93DF92CF92FE01099557
:103FC0002DB73EB72A5F3F4F2DBF11C080E18093D0
:103FD0001F023F932F9383E694E09F938F93DF928A
:103FE000CF92FE0109958DB79EB706968DBF2091A1
:103FF0001E02822F9927AA27BB27FC01419710F0A8
:104000000C94CA28E05BFF4FB9E8CB2EBFE1DB2E52
:10401000C091E203D091E3030C94D97A10921F026D
:1040200088E694E09F938F9309E81FE1DF92CF9297
:10403000FE01099584E180931F020F900F900F906D
:104040000F9081E690E09F938F9386E590E09F9399
:104050008F931F921F92809102016AE00E94327A30
:10406000892F99279F938F93809102010E94327A22
:1040700099279F938F9388E794E09F938F93DF9284
:10408000CF92E091E203F091E303099588E28093F7
:104090001F02EDB7FEB73E96EDBF8BE996E09F930A
:1040A0008F930E94322C99279F938F938DE894E0F1
:1040B0009F938F93DF92CF92E091E203F091E3031D
:1040C00009958091FC032DB73EB7285F3F4F2DBF68
:1040D00084FF06C08CE380931F028BE994E0D2C07A
:1040E0009091FB03992351F08CE380931F02892F59
:1040F00099279F938F9388EA94E03BC19091250282
:104100009923B1F08CE380931F02892F99279F9305
:104110008F938FEB94E09F938F931F930F93E09176
:10412000E203F091E3030995EDB7FEB7369678C444
:104130009091AF03992371F08CE380931F02892F34
:1041400099279F938F9384ED94E09F938F931F9370
:104150000F93D8C480913D0190913E01069710F0D5
:104160000C94D3288CE380931F0285EE94E0A4C7BF
:1041700080910908A9E8CA2EAFE1DA2EC091E203C6
:10418000D091E30380FF6BC010921F028091D20296
:104190009091D302A091D402B091D502BC01CD017F
:1041A00025E030E040E050E00E94877A3F932F9373
:1041B00082EF94E09F938F93DF92CF92FE01099557
:1041C00084E180931F028DB79EB706968DBF8091C4
:1041D000CE029091CF02A091D002B091D102BC0149
:1041E000CD0125E030E040E050E00E94877A3F9327
:1041F0002F938FEF94E09F938F93DF92CF92E09174
:10420000E203F091E303099588E280931F02EDB782
:10421000FEB73696EDBF80911401909115019F93E2
:104220008F938CE095E09F938F93DF92CF92E091F4
:10423000E203F091E30309958CE380931F022DB70D
:104240003EB72A5F3F4F2DBF87B599279F938F9326
:1042500089E195E09F938F93DF92CF928EC0109269
:104260001F0286E295E09F938F93DF92CF92FE012B
:10427000099584E180931F020F900F900F900F908B
:1042800085E395E09F938F93DF92CF9219C71092A9
:104290001F028EE395E09F938F9309E81FE1DF9261
:1042A000CF92FE01099584E180931F020F900F9039
:1042B0000F900F908091320390913303A0913403BB
:1042C000B0913503B7FF04C081509C4FAF4FBF4F33
:1042D000FAE0B595A79597958795FA95D1F7BF938D
:1042E000AF939F938F938BE495E09F938F931F934E
:1042F0000F93E091E203F091E303099588E2809344
:104300001F02EDB7FEB73896EDBF80912A0390915A
:104310002B03A0912C03B0912D03B7FF04C0815053
:104320009C4FAF4FBF4FEAE0B595A79597958795FE
:10433000EA95D1F7BF93AF939F938F938AE595E06A
:104340009F938F931F930F93E091E203F091E30308
:1043500009958CE380931F022DB73EB7285F3F4F2E
:104360002DBF8091C7079091C8079F938F9389E6CF
:1043700095E09F938F931F930F93E091E203F09149
:10438000E30309958DB79EB706968DBF0CC7FF2432
:10439000C0E0D0E001E517E09F2D969584E1989F5D
:1043A000C001112480931F02F801848195819F939D
:1043B0008F932196DF93CF932197828193819F934F
:1043C0008F93DF93CF9388E795E09F938F9389E84E
:1043D0009FE19F938F93E091E203F091E3030995AE
:1043E0002DB73EB7245F3F4F2DBF32E0F30E22962C
:1043F0000C5F1F4F87E08F1578F6D5C610921F020D
:1044000080912406E82FFF27EE0FFF1FEF5AF84F89
:10441000808191819F938F9380912306E82FFF27BE
:10442000EE0FFF1FEF5AF84F808191819F938F937A
:104430008AE895E09F938F93DF92CF92FE010995D2
:1044400084E180931F02EDB7FEB73896EDBF8091EF
:104450002606E82FFF27EE0FFF1FEF5AF84F808147
:1044600091819F938F9380912506E82FFF27EE0F70
:10447000FF1FEF5AF84F8081918181589F4F9F9382
:104480008F938AE995E09F938F93DF92CF92E0918B
:10449000E203F091E303099588E280931F022DB7B0
:1044A0003EB7285F3F4F2DBF80912806E82FFF279A
:1044B000EE0FFF1FEF5AF84F8081918181589F4F77
:1044C0009F938F9380912706E82FFF27EE0FFF1F02
:1044D000EF5AF84F8081918181589F4F9F938F931E
:1044E0008AEA95E09F938F93DF92CF92E091E20367
:1044F000F091E30309958CE380931F028DB79EB77B
:1045000008968DBF80912A06E82FFF27EE0FFF1F28
:10451000EF5AF84F8081918181589F4F9F938F93DD
:1045200080912906E82FFF27EE0FFF1FEF5AF84F63
:104530008081918181589F4F9F938F938AEB95E063
:1045400063C210921F028AEC95E09F938F9309E853
:104550001FE1DF92CF92FE010995809102010F9039
:104560000F900F900F908A3009F09DC084E18093E6
:104570001F0280914703909148039C0197FF02C05E
:10458000295F3F4F287F821B930B9F938F938091CE
:1045900047039091480397FD079673E0959587959B
:1045A0007A95E1F79F938F932091470330914803C9
:1045B00037FF02C0295F3F4F63E0359527956A9525
:1045C000E1F78091FF0190910002821B930B9F9372
:1045D0008F9388ED95E09F938F931F930F93E091B6
:1045E000E203F091E303099588E280931F022DB75F
:1045F0003EB7265F3F4F2DBF809145039091460304
:104600009C0197FF02C0295F3F4F287F821B930BBD
:104610009F938F93809145039091460397FD079652
:1046200053E0959587955A95E1F79F938F93209145
:1046300045033091460337FF02C0295F3F4F43E0F7
:10464000359527954A95E1F78091FD019091FE01FE
:10465000821B930B9F938F9389EE95E09F938F938B
:104660001F930F93E091E203F091E30309958CE32C
:1046700080931F028DB79EB70A968DBF809143032A
:10468000909144039F938F938091430390914403AF
:104690002091FB013091FC01821B930B9F938F9320
:1046A0008AEF95E0ADC08B3019F0843108F4ADC0CD
:1046B00084E180931F0280914703909148039C01FD
:1046C00097FF02C0215F3F4F207F821B930B97FD16
:1046D0000196959587959F938F938091470390912D
:1046E000480397FD0F9624E0959587952A95E1F765
:1046F0009F938F93209147033091480337FF02C067
:10470000295F3F4FC3E035952795CA95E1F7809122
:10471000FF0190910002821B930B9F938F9388E07F
:1047200096E09F938F931F930F93E091E203F09194
:10473000E303099588E280931F022DB73EB7265FF9
:104740003F4F2DBF80914503909146039C0197FFF9
:1047500002C0215F3F4F207F821B930B97FD019684
:10476000959587959F938F938091450390914603EC
:1047700097FD0F96A4E095958795AA95E1F79F93ED
:104780008F93209145033091460337FF02C0295F84
:104790003F4FF3E035952795FA95E1F78091FD01BC
:1047A0009091FE01821B930B9F938F938AE196E079
:1047B0009F938F931F930F93E091E203F091E30394
:1047C00009958CE380931F028DB79EB70A968DBF23
:1047D000809143039091440397FD019695958795A9
:1047E0009F938F9380914303909144032091FB0109
:1047F0003091FC01821B930B9F938F938CE296E088
:104800009F938F931F930F9303C18D3009F0CBC4F7
:1048100084E180931F028091130199279F938F93C6
:10482000809147039091480397FD0F9674E095950A
:1048300087957A95E1F79F938F9320914703309165
:10484000480337FF02C0295F3F4F63E03595279546
:104850006A95E1F78091FF0190910002821B930B12
:104860009F938F938BE396E09F938F931F930F9368
:10487000E091E203F091E303099588E280931F023F
:104880002DB73EB7265F3F4F2DBF8091120199276C
:104890009F938F93809145039091460397FD0F96C8
:1048A00054E0959587955A95E1F79F938F932091C2
:1048B00045033091460337FF02C0295F3F4F43E075
:1048C000359527954A95E1F78091FD019091FE017C
:1048D000821B930B9F938F938FE496E09F938F930C
:1048E0001F930F93E091E203F091E30309958CE3AA
:1048F00080931F028DB79EB70A968DBF80911101DC
:1049000099279F938F93809143039091440397FD40
:104910000196959587959F938F93809143039091EE
:1049200044032091FB013091FC01821B930B9F9368
:104930008F9383E696E09F938F931F930F93E0915D
:10494000E203F091E3030995EDB7FEB73A9668C02C
:1049500010921F0287E796E09F938F93DF92CF928A
:10496000FE01099584E180931F020F900F900F9034
:104970000F9080913D0390913E039F938F93809180
:10498000F7019091F8019F938F9384E896E09F93AD
:104990008F93DF92CF92E091E203F091E3030995C8
:1049A00088E280931F022DB73EB7285F3F4F2DBF8F
:1049B00080913B0390913C039F938F938091F901E9
:1049C0009091FA019F938F9383E996E09F938F9341
:1049D000DF92CF92E091E203F091E30309958CE33B
:1049E00080931F028DB79EB708968DBF80913703C5
:1049F000909138039F938F938091F5019091F601E8
:104A00009F938F9382EA96E09F938F93DF92CF924A
:104A1000E091E203F091E3030995EDB7FEB7389614
:104A2000EDBFC1C310921F0280911E0190911F0122
:104A30006AE070E00E94527A9F938F9380911E01EA
:104A400090911F016AE070E00E94527A7F936F9309
:104A500081EB96E09F938F93DF92CF92FE010995B1
:104A600084E180931F022DB73EB7285F3F4F2DBFD3
:104A70008091A9089091AA086AE070E00E943E7AAD
:104A80009F938F938091A9089091AA086AE070E0A3
:104A90000E943E7A7F936F9385EC96E09F938F936D
:104AA000DF92CF92E091E203F091E303099588E26F
:104AB00080931F028DB79EB708968DBF8091AB087B
:104AC0009091AC089F938F9389ED96E09F938F937D
:104AD000DF92CF92E091E203F091E30309958CE33A
:104AE00080931F02EDB7FEB73696EDBF8091AD08FB
:104AF0009091AE089F938F9389EE96E09F938F934A
:104B0000DF92CF92E091E203F091E30309952DB794
:104B10003EB72A5F3F4F4FC110921F028BEF96E0C6
:104B20009F938F93DF92CF92FE01099584E180934A
:104B30001F020F900F900F900F908091510790914E
:104B400052079F938F9384E097E09F938F93DF9218
:104B5000CF92E091E203F091E303099588E280931C
:104B60001F028DB79EB706968DBF8091D8029927F8
:104B70009F938F9384E197E09F938F93DF92CF92DF
:104B8000E091E203F091E30309958CE380931F0227
:104B9000EDB7FEB73696EDBF809150079927019784
:104BA0009F938F9384E297E0A9CF10921F0284E332
:104BB00097E09F938F93DF92CF92FE01099584E156
:104BC00080931F020F900F900F900F908091900193
:104BD000909191019F938F938CE397E09F938F9394
:104BE000DF92CF92E091E203F091E303099588E22E
:104BF00080931F028DB79EB706968DBF8091C70721
:104C00009091C8079F938F938AE497E09F938F9327
:104C1000DF92CF92E091E203F091E30309958CE3F8
:104C200080931F02EDB7FEB73696EDBF8091F0027C
:104C30009091F1029F938F9388E597E05FCFC9ED44
:104C4000CC2EC2E0DC2E20E030E0E901B3E0FB2E08
:104C5000C0931F02F60181916F0199279F938F9353
:104C600089010F5F1F4F1F930F9386E697E09F9375
:104C70008F9389E89FE19F938F93E091E203F091F6
:104C8000E30309952DB73EB7285F3F4F2DBFFA9438
:104C900064969801F7FEDCCF86C2ADEDCA2EA2E085
:104CA000DA2EC0E0D0E08E01F3E0FF2E00931F0269
:104CB000F60181916F0199279F938F932596DF933A
:104CC000CF9383E797E09F938F9389E89FE19F932A
:104CD0008F93E091E203F091E30309952DB73EB77E
:104CE000285F3F4F2DBFFA940C5E1F4F2497F7FEAD
:104CF000DDCF59C210921F0280E897E09F938F93F7
:104D000009E81FE1DF92CF92FE01099584E18093CB
:104D10001F020F900F900F900F9080916F019927B5
:104D20009F938F9388E897E09F938F93DF92CF9222
:104D3000E091E203F091E303099588E280931F027A
:104D40008DB79EB706968DBF8091D6019091D70101
:104D500097FD039695958795959587959F938F9346
:104D600086E997E09F938F931F930F93E091E2035F
:104D7000F091E30309958CE380931F02EDB7FEB732
:104D80003696EDBF8091520699279F938F9380911D
:104D9000510699279F938F9384EA97E09F938F936F
:104DA0001F930F93E091E203F091E30309952DB770
:104DB0003EB7285F3F4F2DBFF6C110921F0282EB16
:104DC00097E09F938F9379E8A72E7FE1B72EDF922C
:104DD000CF92FE0109950F900F900F900F90C0EFAA
:104DE000D6E000E010E062E0F62E802F8C5E80932B
:104DF0001F028B8D99278F7790709F938F938B894C
:104E000099278F7790709F938F938B8599278F77B2
:104E100090709F938F938B8199278F7790709F933A
:104E20008F9382EC97E09F938F93BF92AF92E09124
:104E3000E203F091E30309958DB79EB70C968DBF01
:104E4000FA940C5E1F4FA096F7FECFCFACC1109224
:104E50001F0283ED97E09F938F9359E8A52E5FE1A2
:104E6000B52EDF92CF92FE0109950F900F900F9013
:104E70000F90C0EFD6E000E010E042E0F42E802F6B
:104E80008C5E80931F028F8D992787FD90959F934D
:104E90008F938F89992787FD90959F938F938F8507
:104EA000992787FD90959F938F938F81992787FDF1
:104EB00090959F938F9382EE97E09F938F93BF92ED
:104EC000AF92E091E203F091E3030995EDB7FEB7ED
:104ED0003C96EDBFFA940C5E1F4FA096F7FECFCF25
:104EE00062C110921F0283EF97E09F938F9309E8AE
:104EF0001FE1DF92CF92FE01099584E180931F02AA
:104F00000F900F900F900F9080910B07881F8827AC
:104F1000881F97E0899FC00111248D969F938F93DE
:104F200080910307881F8827881F96E0899FC0010A
:104F300011248D969F938F938091FB06881F88275D
:104F4000881F95E0899FC00111248D969F938F93B0
:104F50008091F306881F8827881F9927880F991F3B
:104F6000880F991F8D969F938F9382E098E09F936F
:104F70008F93DF92CF92E091E203F091E3030995E2
:104F800088E280931F022DB73EB7245F3F4F2DBFAD
:104F900080912B07881F8827881F9BE0899FC0016D
:104FA00011248D969F938F9380912307881F8827C4
:104FB000881F9AE0899FC00111248D969F938F933B
:104FC00080911B07881F8827881F99E0899FC0014F
:104FD00011248D969F938F9380911307881F8827A4
:104FE000881F992723E0880F991F2A95E1F78D964E
:104FF0009F938F9386E198E09F938F93DF92CF9258
:10500000E091E203F091E30309958CE380931F02A2
:105010008DB79EB70C968DBF80913307881F882768
:10502000881F9CE0899FC00111248D969F938F93C8
:105030008AE298E09F938F93DF92CF92E091E20310
:10504000F091E303099580913B07EDB7FEB73696E3
:10505000EDBF87FF12C080E480931F028BE398E0CE
:105060009F938F93DF92CF92E091E203F091E3035D
:1050700009950F900F900F900F908091430787FF35
:1050800012C084E480931F028EE398E09F938F9375
:105090001F930F93E091E203F091E30309950F90C2
:1050A0000F900F900F9080914B0787FF7CC088E492
:1050B00080931F0281E498E09F938F931F930F9337
:1050C000E091E203F091E30309950F900F900F90A8
:1050D0000F9069C010921F0284E498E09F938F9311
:1050E000DF92CF92FE01099584E180931F020F9019
:1050F0000F900F900F908091AC019091AD019F9314
:105100008F9382E598E09F938F93DF92CF92E09107
:10511000E203F091E303099588E280931F022DB723
:105120003EB72A5F3F4F2DBF8091AE019091AF01F6
:105130009F938F938FE598E09F938F93DF92CF9209
:10514000E091E203F091E303099589E480931F0263
:105150008DB79EB706968DBF8CE698E09F938F9390
:10516000DF92CF92E091E203F091E3030995809101
:105170001D020F900F900F900F9083FF14C010929C
:10518000AF011092AE0160E070E08EE090E00E940E
:10519000DE2A09C080912001281719F4215020939C
:1051A000200110921E0210921D02DF91CF911F91DB
:1051B0000F91FF90DF90CF90BF90AF900895F99935
:1051C000FECF92BD81BDF89A80B599270895F999CF
:1051D000FECF1FBA92BD81BD60BD0FB6F894FA9A9A
:1051E000F99A0FBE08954AEA20E030E02617370703
:1051F00040F4FC018191480F2F5F3F4F261737077E
:10520000C8F3842F99270895EAEA40E050E0461752
:10521000570778F49C01F999FECF32BD21BDF89A69
:1052200080B5E80F4F5F5F4F2F5F3F4F461757071F
:1052300090F38E2F9927089581E08093250682E0D0
:105240008093240683E08093230684E080932606DF
:1052500085E08093270686E08093280687E0809388
:10526000290688E080932A0689E080932B068AE04D
:1052700080932C068BE080932D068CE080932E0685
:10528000089588E58093220680910201843150F0D0
:105290008AE080934206109266068BE180933E0678
:1052A0008EE40AC083E08093420680E28093660623
:1052B0008EE180933E0685E58093630680936406C5
:1052C00080E2809365068AE680932F0682E28093CF
:1052D0008C0664E06093490610928506109282065F
:1052E00048E040933C0656EE50933D0630E4309340
:1052F0003F069EE1909330068FEF809332062FE0B9
:10530000209333069093310610923506409336066B
:1053100030933706109238062093340610924B06CD
:1053200010924C0610924D0610924E06109268068E
:105330001092690610926A0610926B0690E890939C
:105340004F0632E33093500682E080938B06209321
:10535000510650935206609357068DE780935A0684
:1053600080935B0680935C069093530625E520931B
:10537000540686E4809355068CED809356068CE3A4
:1053800080935806109259068FE580936C0683EF40
:1053900080936E068AEA809370068093710684E19A
:1053A00080936D0680936F0630935D069AE5909327
:1053B0005E0630935F0610928A068EEF8093720627
:1053C00084E6809373069093740690937506909389
:1053D00076068BE48093770620937806809379068F
:1053E00010927A0686E080937B0640937C06909329
:1053F0007D068AE280937E0685EF80937F068CE8A7
:105400008093800685E08093810610928306109237
:10541000840681E2809346068DE28093470690934E
:10542000480610928606109287061092880686E932
:10543000809389069093600687E3809361060895C0
:10544000CF93DF930E9441298AE08093390680E15F
:1054500080933A0626E020933B069AE59093400617
:1054600088E78093410690934306809344062093F7
:10547000450680E280934A068CE3809362068BE4C3
:1054800080936706ADE8B6E08CE0E1E2F1E0ED0183
:10549000019009928A95E1F767E770E0CD018B569C
:1054A00090400E94F32880939906DF91CF91089550
:1054B000CF93DF930E94412988E08093390630E141
:1054C00030933A0626E020933B0694E690934006FC
:1054D00088E7809341069093430680934406209387
:1054E000450630934A0686E48093620680936706F9
:1054F000ADE8B6E08CE0E7E2F1E0ED010190099261
:105500008A95E1F767E770E0CD018B5690400E94E5
:10551000F32880939906DF91CF910895CF93DF937D
:105520000E94412926E0209339068AE080933A06BA
:1055300084E080933B0694E69093400688E780934E
:10554000410690934306809344062093450680E1EC
:1055500080934A0686E48093620680936706ADE8EE
:10556000B6E08CE0EFE2F1E0ED01019009928A955E
:10557000E1F767E770E0CD018B5690400E94F32879
:1055800080939906DF91CF910895F999FECF92BD4E
:1055900081BDF89A80B599270895F999FECF1FBA71
:1055A00092BD81BD60BD0FB6F894FA9AF99A0FBE0C
:1055B00008956FED78E20E94A178089547EE58E2D1
:1055C0000E94DB780895EF92FF920F931F93CF9381
:1055D000C82F8150853008F0C3E088E7C89F80015C
:1055E00011248CEEE82E8FEFF82EE00EF11E67E707
:1055F00070E0C7010E940429682F98012D593F4F80
:105600008FB39927AC014270507081FDF9CF32BD44
:1056100021BDF89A80B5861711F0CA0121C08FB359
:1056200099279C012270307081FDF9CFF2BCE1BC5A
:10563000F89A80B5883511F0C90112C088E7C89F73
:10564000C001112444972FED38E248E750E0BC0137
:1056500082E296E00E947C780E94BF6781E090E041
:10566000CF911F910F91FF90EF900895282F8630D2
:1056700010F025E003C0882309F421E0F999FECF5A
:105680001FBA82E090E092BD81BD20BD0FB6F894B4
:10569000FA9AF99A0FBE0895CF93C82F80912206E7
:1056A000883509F044C0C63010F0C5E003C0CC23F3
:1056B00009F43DC00E94877767E770E082E296E0D8
:1056C0000E94F3288093990688E7C89FC00111249F
:1056D00027EE38E248E750E062E276E044970E9425
:1056E000B97827EE38E24CE050E063E276E080E5FE
:1056F00090E00E94B9786CE070E083E296E00E944E
:10570000F328282FF999FECF1FBA8CE590E092BDBF
:1057100081BD20BD0FB6F894FA9AF99A0FBE8C2F6E
:105720000E94362B0E94BF6781E090E002C080E0BB
:1057300090E0CF9108956DE470E088EE93E00E94D0
:105740000429482F8FB399279C012270307081FD66
:10575000F9CF85E394E092BD81BDF89A80B58417B6
:1057600079F48FB399279C012270307081FDF9CFB5
:1057700088EE93E092BD81BDF89A80B5813011F03A
:10578000C90108952FED38E24EE450E068EE73E071
:105790008AE996E00E947C7881E090E0089580910B
:1057A0009A068130A9F46DE470E08AE996E00E94DF
:1057B000F3288093E70627EE38E24EE450E06AE9EA
:1057C00076E088EE93E00E94B97881E090E0089559
:1057D00080E090E00895CF93DF9381E080939A0674
:1057E000EAE9F6E08FE0158616861786108A815062
:1057F000349687FFF8CF80E48093A7068093A806AD
:105800001092A9068093AA068093AB0690EC909321
:10581000AC061092AD068093AE068093AF06109250
:10582000B0069093B1069093B2068093B30610929F
:10583000B4068093B5069093B606ABE9B6E087E070
:10584000E5E3F1E0ED01019009928A95E1F76DE45D
:1058500070E0CD0101970E94F3288093E706DF9165
:10586000CF910895F999FECF82E090E092BD81BD7D
:10587000F89A80B5282F863078F023E0322FF999F6
:10588000FECF1FBA82E090E092BD81BD30BD0FB661
:10589000F894FA9AF99A0FBE822F992708951F93C8
:1058A000CF93C82F162F863010F0C5E003C0882391
:1058B00009F4C1E08C2F99278230910541F08330A3
:1058C000910544F4019731F40E94202A05C00E94FA
:1058D000582A02C00E948E2A1123E1F06CE070E089
:1058E00080E590E00E940429282FF999FECF8CE5ED
:1058F00090E092BD81BDF89A80B5821759F42FEDE2
:1059000038E24CE050E060E570E083E296E00E940F
:105910007C7802C00E941C298C2F0E944C2BCF91B6
:105920001F910895DF92EF92FF920F931F93CF93F1
:10593000FF24DF2CEF2C81E090E00E94C52A8835FF
:1059400011F031E0E32E6CE070E080E590E00E9421
:105950000429C82FF999FECF8CE590E092BD81BD56
:10596000F89A80B58C1711F421E0D22EC1E001E045
:1059700010E0EE2029F48C2F0E94E32A8823C9F539
:1059800091E0F92E1F930F9384E798E09F938F93F4
:1059900081E892E19F938F93E091E203F091E3031A
:1059A00009952DB73EB72A5F3F4F2DBF0230110535
:1059B00049F0033011054CF40130110531F40E9417
:1059C000202A05C00E94582A02C00E948E2ADD208B
:1059D00059F02FED38E24CE050E060E570E083E2F2
:1059E00096E00E947C7802C00E941C298C2F0E94A5
:1059F0004C2BCF5F0F5F1F4FC63008F4BACFFF208C
:105A000019F083E00E94362B0E94322CC82F0E948E
:105A1000E32A8C2F99279F938F938AE998E09F938D
:105A20008F9301E812E11F930F93E091E203F0914D
:105A3000E303099581E090E00E94C52A2DB73EB7A7
:105A40002A5F3F4F2DBF8F3F21F00E949B2B882361
:105A500099F483EB98E09F938F931F930F93E091BA
:105A6000E203F091E30309950E94EB2B0E94CF2BF8
:105A70000F900F900F900F90EE2029F068E581E0D5
:105A800090E00E94CD2A1092210690E0E7EAF6E02D
:105A9000CFE08081349618160CF49F5FC150C7FF89
:105AA000F8CF90932106892F99279F938F938BE9A5
:105AB00096E09F938F9384ED98E09F938F931F932D
:105AC0000F93E091E203F091E30309958DB79EB740
:105AD00008968DBF85EF98E09F938F931F930F9348
:105AE000E091E203F091E30309950F900F900F907E
:105AF0000F90CF911F910F91FF90EF90DF9008953D
:105B0000982F2FB7F8943998389A88B1836088B95C
:105B10008091B9008C7F8093B9008AE28093B800AD
:105B200010922A021092280210922702992379F0EB
:105B3000E0EFF6E08BE01082118212821382148271
:105B40001582168217828150389687FFF4CF789499
:105B50002FBF089510922A0284E98093BC0080E848
:105B60008093BC001092BD001092BA001092BB004E
:105B70001092B9001092B8001092260280E00E94A4
:105B8000802D1092BB0085E88093BC008091240298
:105B900082608093240208951F920F920FB60F9295
:105BA00011242F933F934F935F938F939F93EF9382
:105BB000FF9380912A02282F3327442755278F5F90
:105BC00080932A02F9012731310508F0C2C2EF594A
:105BD000FF4F0C94D97A81E08093260209C080910E
:105BE00028028C3090F4809128028F5F80932802E5
:105BF00080912802E82FFF27EE0FFF1FEE0FFF1FF7
:105C0000E656F94F8585181654F7809128028C3096
:105C100070F010922302109222021092280285E066
:105C200080932A0280912702880F8D5A04C08091A8
:105C30002802880F8E5A8093BB0085E87FC280912E
:105C40002802E82FFF2783E0EE0FFF1F8A95E1F778
:105C5000E051F94F81818093BB0085E88093BC00BF
:105C600080912802E82FFF27EE0FFF1FEE0FFF1F86
:105C7000EE0FFF1FE051F94F808180FF91C08091AE
:105C80002802E82FFF27EE0FFF1FEE0FFF1FEE0F7A
:105C9000FF1FE051F94F8281882329F0809121066E
:105CA000873008F46CC28091220290912302892BE4
:105CB00009F065C28091200290912102892B09F0A0
:105CC0005EC26EC08091280221E030E002C0220F47
:105CD000331F8A95E2F780912002909121022823B8
:105CE0003923232B79F080912802E82FFF27EE0F2C
:105CF000FF1FEE0FFF1FEE0FFF1FE051F94F80E176
:105D000084830DC080912802E82FFF27EE0FFF1F2C
:105D1000EE0FFF1FEE0FFF1FE051F94F148280912D
:105D20002802E82FFF2753E0EE0FFF1F5A95E1F7F7
:105D3000E051F94F8481282F332743E0220F331F8E
:105D40004A95E1F780912802E82FFF2793E0EE0FB4
:105D5000FF1F9A95E1F7E051F94F82818770822BFE
:105D60008093BB0085E88093BC002091280281E0ED
:105D700090E002C0880F991F2A95E2F72091220235
:105D80003091230282239323892B51F088EE96E0F1
:105D900090932E0280932D0288E080932F02EFC112
:105DA00084E089C1E0912D02F0912E0281918093CF
:105DB000BB0085E88093BC00F0932E02E0932D0297
:105DC00080912F02815080932F02882309F4D7C13C
:105DD00083E071C18091B900803351F580912B022D
:105DE000882329F4809128028F5F80932B02809171
:105DF0002802E82FFF2783E0EE0FFF1F8A95E1F7C7
:105E0000E051F94F838199278F7790708F379105F3
:105E10007CF480912802E82FFF27EE0FFF1FEE0F82
:105E2000FF1FEE0FFF1FE051F94F83818F5F8383C8
:105E300010922A0284E98093BC008AE090E090935B
:105E40003E0180933D01809128028F5F809328025C
:105E500010922A026DC18091B9008034C9F18091FD
:105E60002702E82FFF27EE0FFF1FEE0FFF1FEE0F99
:105E7000FF1FE051F94F83818F7783838091270241
:105E80008F5F80932702809127028C30A0F01092C0
:105E90002702109221021092200280912C028F5F23
:105EA00080932C028C3038F010922C0280912402C6
:105EB0008D7F80932402809124028160809324024C
:105EC00010922A0284E98093BC001092260273C0CB
:105ED00080912702E82FFF27EE0FFF1FEE0FFF1F15
:105EE000EE0FFF1FE051F94F83818068838380911B
:105EF0002702E82FFF27EE0FFF1FEE0FFF1FEE0F09
:105F0000FF1FE051F94F808180FF2FC08091270251
:105F1000E82FFF2753E0EE0FFF1F5A95E1F7E051FE
:105F2000F94F84819927009751F04097D9F588EE71
:105F300096E090932E0280932D0288E031C08091EC
:105F40002702992743E0880F991F4A95E1F78B5064
:105F5000994F90932E0280932D0290912702809169
:105F60002C029817E1F483E01BC080912702992747
:105F700033E0880F991F3A95E1F78B50994F909332
:105F80002E0280932D028091240281FD06C0909103
:105F9000270280912C02981711F482E001C081E061
:105FA00080932F0280912F02813011F485E801C087
:105FB00085EC8093BC0080912B0280932502109287
:105FC0002B02DDC0E0912D02F0912E028091BB00EA
:105FD000808380912D0290912E02019690932E0243
:105FE00080932D0280912F02815080932F02823066
:105FF00010F085EC5DC0813011F485E859C08091C6
:10600000240281FF2DC08091A20280FD1DC08091DD
:106010002702E82FFF2723E0EE0FFF1F2A95E1F765
:10602000E051F94F86818A3F79F480912702E82F69
:10603000FF2793E0EE0FFF1F9A95E1F7E051F94F2C
:106040008081816080830CC080912702E82FFF2728
:1060500083E0EE0FFF1F8A95E1F7E051F94F1082C0
:10606000809127028F5F80932702809127028C30D6
:10607000A0F010922702109221021092200280912B
:106080002C028F5F80932C028C3038F010922C02FF
:10609000809124028D7F8093240210922A0284E949
:1060A0008093BC008091240281608093240265C0AB
:1060B0008093BC0086E080932A0261C088E9BBCD52
:1060C00080912902880F805FB6CD8091290299279F
:1060D0008130910561F0823091051CF4892B21F00B
:1060E0004EC0029739F04BC080911301A4CD80912E
:1060F0001201A1CD809111019ECD80E89CCD10921E
:106100002A0284E98093BC00109226028AE090E083
:1061100090933E0180933D0180912902823088F462
:10612000809129028F5F8093290282E180932A0265
:10613000809124028E7F8093240285EA8093BC00A4
:106140001EC0109229028091240281608093240253
:1061500016C010922A0284E98093BC008091240228
:106160008160809324028AE090E090933E018093C6
:106170003D01109228021092270210922602FF91F0
:10618000EF919F918F915F914F913F912F910F9040
:106190000FBE0F901F9018951F93CF93DF93182F6A
:1061A0008091D702882321F48091BB01882319F0C4
:1061B00081E090E097C01D3008F092C01123B1F04B
:1061C000E12FFF2723E0EE0FFF1F2A95E1F7E051B3
:1061D000F94F35978081359688230CF081C0389728
:1061E000808180FD03C083E090E07CC08091E80660
:1061F000823019F084E090E075C067E070E088EECE
:1062000096E00E94F3289091EF06891719F085E037
:1062100090E068C080ED97E00E948F16EC018091BD
:10622000240280FD05C0CE010E9498168823B9F390
:10623000112319F48FEF90E00BC0212F3327215049
:10624000304081E090E002C0880F991F2A95E2F764
:106250009093230280932202A1E0B0E0E0EFF6E009
:1062600040E050E06BE0CD01042E02C0880F991F82
:106270000A94E2F720912202309123028223932391
:10628000892B11F01182128261504F5F5F4F389657
:1062900067FFE9CF1092280210922A02809124020F
:1062A0008E7F8093240285EA8093BC008091240233
:1062B00080FD05C0CE010E9498168823B9F3809115
:1062C000220290912302892B29F0CE010E94981678
:1062D000882311F38091220290912302009711F0FC
:1062E00082E090E0DF91CF911F9108950F931F936B
:1062F000CF93DF93982F8091D702882321F4809148
:10630000BB01882319F081E090E092C09D30A0F499
:10631000992319F486E090E08BC0C92FDD27FE0198
:1063200033E0EE0FFF1F3A95E1F7E051F94F359753
:106330008081359687FD03C082E090E079C0389770
:10634000808180FD03C083E090E072C080ED97E023
:106350000E948F168C018091240280FD05C0C80127
:106360000E9498168823B9F3219721E030E0C901F3
:1063700002C0880F991FCA95E2F79093210280937B
:106380002002D901E0EFF6E040E050E06BE0CD0103
:10639000042E02C0880F991F0A94E2F72091200270
:1063A0003091210282239323892B11F011821282D2
:1063B00061504F5F5F4F389667FFE9CF1092270219
:1063C0001092E8061092EF0610922A0280912402A1
:1063D0008E7F8093240285EA8093BC008091240202
:1063E00080FD05C0C8010E9498168823B9F38091EA
:1063F000200290912102892B29F0C8010E94981651
:10640000882311F38091E806823019F084E090E04F
:106410000FC067E070E088EE96E00E94F32890914C
:10642000EF06891719F085E090E002C080E090E067
:10643000DF91CF911F910F910895CF93DF9380E06B
:1064400022E83FEFC5E8D7E0E1E5F7E0DF0185307E
:1064500020F411961C921E9202C03183208319826F
:10646000188222968F5F129632968A3180F31092AC
:106470004403109243031092460310924503109276
:10648000480310924703DF91CF9108951F920F9216
:106490000FB60F9211240F931F932F933F934F9397
:1064A0005F936F937F938F939F93AF93BF93CF939C
:1064B000DF93EF93FF9380918C0682FDD3C04091D0
:1064C0008600509187008091310290913202481BE2
:1064D000590B8091860090918700909332028093AF
:1064E0003102CA018D549440A0913302B09134021C
:1064F000835F9A4178F48091330280935007149718
:1065000014F01092410181E090E090933402809366
:1065100033020FC2AD30B1050CF00BC2CA018B5F64
:106520009040845B914008F078C080913F01909149
:106530004001481B590BFD01EA0FFB1FEF5AF84FB2
:1065400080819181FA01E81BF90BCF01F7FF03C0AD
:10655000909581959F4F06975CF48091D802883C76
:1065600020F48091D802865F01C088EC8093D80225
:10657000FD01EA0FFB1FEF5AF84F808191819C01CA
:10658000220F331F280F391F240F351F37FF02C07A
:106590002D5F3F4FE901D595C795D595C795CA01A0
:1065A00001968C179D0714F4219706C04150504066
:1065B000C417D5070CF421968091D802833CE0F0F3
:1065C0008D010A0F1B1FF801EF5AF84F808191814E
:1065D0009E01281B390BC90163E070E00E94527ACA
:1065E000CB01880F991F860F971F0B57184FD801A3
:1065F00011969C938E9307C0AA0FBB1FAB57B84F41
:1066000011961C921E92E0913302F0913402EE0F2B
:10661000FF1FEF5AF84FD183C0832091330230918E
:1066200034022F5F3F4F3093340220933302809126
:106630000201843108F07DC12530310511F45D9AE5
:1066400001C05D98809133029091340286309105AB
:1066500011F45C9A01C05C98079711F45B9A69C1C8
:106660005B9867C140918600509187008091350208
:1066700090913602481B590B8091860090918700BB
:106680009093360280933502CA018D5494406091F4
:106690009F02835F9A4108F07AC060933002809134
:1066A0003002843008F453C090915007809130023A
:1066B000981709F04CC05091A0025B3008F43FC01D
:1066C0001092410110929F0240E05F31C0F0E42F30
:1066D000FF27EE0FFF1F9F0125593D4FDF01AF5AE6
:1066E000B84F8D919C91D9018D939C93DF01AB574D
:1066F000B84F8D919C91EB57FD4F91838083E42F90
:10670000FF27EE0FFF1F9F012F5A384FDF01A95CB3
:10671000BD4F8D919C91D90111969C938E93DF0171
:10672000AF5ABD4F8D919C91EB57F84F9183808369
:10673000842F8F5F482F8D3040F280939F0280918D
:10674000A0028F3FB9F08F5F8093A00213C08091A9
:10675000A002853620F08AE08093A00202C0109249
:10676000A002809102018A3011F0843110F0289A41
:1067700001C0289881E080939F028091D7028823EE
:1067800009F0D7C08091300280935007D2C06D309D
:1067900008F0A7C0CA018B5F9040845B914008F06D
:1067A00082C080913F0190914001481B590BE62F18
:1067B000FF27EE0FFF1FE95CFD4F80819181FA01F9
:1067C000E81BF90BCF0105960B97B0F48091A0025E
:1067D0008A3120F08091D802865F05C08B3028F086
:1067E0008091D8028E5F8093D8028091D802893C34
:1067F00018F088EC8093D802E62FFF27EE0FFF1FDA
:10680000E95CFD4F808191819C01220F331F280F8D
:10681000391F240F351F37FF02C02D5F3F4FE9019D
:10682000D595C795D595C795CA0101968C179D0733
:1068300014F4219706C041505040C417D5070CF4FA
:1068400021968091D8028E3BD8F0E62FFF27EE0FDD
:10685000FF1FDF01A95CBD4F8D919C919E01281BFC
:10686000390BC90163E070E00E94527ACB01880FB6
:10687000991F860F971FEF5AFD4F9183808308C0A1
:10688000E62FFF27EE0FFF1FEF5AFD4F11821082F8
:1068900080919F02E82FFF27EE0FFF1FE95CFD4F5D
:1068A000D183C08309C0809102018A3011F0843104
:1068B00010F0289A01C0289880910201843188F450
:1068C00080919F02853011F45D9A05C05D988630F5
:1068D00011F45C9A05C05C98873011F45B9A01C092
:1068E0005B9880919F02843120F48F5F80939F0298
:1068F00020C08431F1F4809102018A3011F084319A
:1069000010F0289A01C028988EE180939F022CE015
:10691000C5E8D7E0ABE6B2E0E1E5F7E08D919D9107
:10692000918380833296198218822296215027FF04
:10693000F5CFFF91EF91DF91CF91BF91AF919F91F3
:106940008F917F916F915F914F913F912F911F9107
:106950000F910F900FBE0F901F901895EF92FF921E
:106960000F931F9380913E069927880F991F880FD8
:10697000991F7C010027F7FC0095102F80913203AE
:1069800090913303A0913403B0913503BC01CD0144
:10699000A80197010E94877A30937E0520937D0598
:1069A00080912A0390912B03A0912C03B0912D0389
:1069B000BC01CD01A80197010E94877A3093800520
:1069C00020937F0580910D0890910E0897FD039606
:1069D00095958795959587959093820580938105E8
:1069E00080911D0890911E0897FD039695958795B7
:1069F00095958795909384058093830580914303B3
:106A0000909144032091FB013091FC01821B930B78
:106A100090938605809385058091D2029091D30250
:106A2000A091D402B091D502BC01CD0125E030E0A7
:106A300040E050E00E94877A3093880520938705D4
:106A40008091F5019091F60190938A0580938905D4
:106A5000809190019091910190938E0580938D0586
:106A600080911E0190911F019093900580938F0556
:106A70008091D802992790939205809391058091F7
:106A8000C7079091C80790939405809393058091D0
:106A9000F106992790939605809395058091F906C4
:106AA00099279093980580939705809101079927DE
:106AB00090939A058093990580910907992790935F
:106AC0009C0580939B058091D6019091D70190936E
:106AD000A6058093A5058091A9089091AA08909396
:106AE000AA058093A9058091AD089091AE08909376
:106AF000AC058093AB058091CE029091CF02A0911E
:106B0000D002B091D102BC01CD0125E030E040E0DF
:106B100050E00E94877A3093AE052093AD058091B6
:106B2000F0029091F1029093B4058093B3058091A7
:106B3000AF0899279093B8058093B7058091A50376
:106B40009091A6039093BA058093B9058091A30311
:106B50009091A4039093BC058093BB058091FB03A7
:106B6000882321F48091FC03882321F080917C0507
:106B7000816003C080917C058E7F80937C051F918E
:106B80000F91FF90EF9008951F93CF93DF93182FED
:106B9000EB018091D7028823A1F411501F3F89F0A7
:106BA000D093DD01C093DC018091DC019091DD0187
:106BB000892BD1F7CE018C0F9D1F0E94A416115076
:106BC00078F7DF91CF911F910895CF93DF93809154
:106BD00002018D3011F40E949D1A10927A0080916A
:106BE000FF01909100029093D2078093D10780918A
:106BF000FD019091FE019093C3078093C20780919D
:106C0000FB019091FC01909313088093120820914E
:106C1000F7013091F801C901880F991F880F991F5A
:106C2000820F931F820F931F90930E0880930D087D
:106C30002091F9013091FA01C901880F991F880F3D
:106C4000991F820F931F820F931F90931E088093AA
:106C50001D088FEC80937A00A9EDB2E0C7E2D6E080
:106C600097E08991E82FFF27EE0FFF1FEF5AF84FAB
:106C70000190F081E02DE158FF4F1E161F061CF019
:106C8000E0E0F0E005C0EF3FF10514F0EFEFF0E0D9
:106C90008C91282F3327E217F30714F4815004C096
:106CA0002E173F0714F48F5F8C939150119697FF26
:106CB000D8CF809163069927AA27BB27BC01CD01B5
:106CC00024EC39E040E050E00E94137ADC01CB0173
:106CD0008093880190938901A0938A01B0938B01DE
:106CE000809164069927AA27BB27BC01CD010E9489
:106CF000137ADC01CB018093840190938501A093EA
:106D00008601B0938701DF91CF910895A0E0B0E0B4
:106D1000ECE8F6E30C94A87A882EC0E0D0E07E017F
:106D20006E011092FB03469AD0933E03C0933D033D
:106D3000D0933C03C0933B03D0933803C0933703F5
:106D4000D0934803C0934703D0934603C0934503B1
:106D5000D0934403C093430310926C0110926B01D3
:106D60001092EF010E94E53584E690E00E94B11692
:106D70000E94E53580912F0680FF10C0809114019C
:106D800090911501875B934038F4809114019091A4
:106D900015018E5E924010F40E94421A0FE18AE0C3
:106DA00090E00E94B1168091FB019091FC01C80F08
:106DB000D91F8091FF0190910002E80EF91E809189
:106DC000FD019091FE01C80ED91E015007FFE7CFCB
:106DD0009701205F3F4F369527953695279530933D
:106DE000480320934703C60140969695879596954C
:106DF000879590934603809345036096F5E0D6957A
:106E0000C795FA95E1F7D0934403C0934303909359
:106E10004203809341033093400320933F03882033
:106E200009F441C080910D0890910E0897FF03C0AE
:106E3000909581959F4F6CE070E00E94527A9B0183
:106E400070933E0360933D0380911D0890911E084E
:106E500097FF03C0909581959F4F6CE070E00E9472
:106E6000527A70933C0360933B038091C4059091E8
:106E7000C5059093380380933703B90184E090E00F
:106E80000E94DE2A60913B0370913C0386E090E013
:106E90000E94DE2A609137037091380388E090E009
:106EA0000E94DE2A65C084E090E00E94D92A909377
:106EB0003E0380933D0386E090E00E94D92A9093A0
:106EC0003C0380933B0388E090E00E94D92A9C0118
:106ED000909338038093370380913D0390913E0354
:106EE0008150984050F480913B0390913C03815035
:106EF000984018F421503440D8F186E199E09F93EE
:106F00008F9381E892E19F938F93E091E203F09158
:106F1000E303099580910D0890910E0897FF03C037
:106F2000909581959F4F6CE070E00E94527A70932B
:106F30003E0360933D0380911D0890911E0897FFCA
:106F400003C0909581959F4F6CE070E00E94527A4B
:106F500070933C0360933B038091C4059091C505F9
:106F600090933803809337030F900F900F900F90FA
:106F70001092D2071092D1071092C3071092C20745
:106F8000109213081092120884E690E00E94B11645
:106F90008091F7019091F8019C01220F331F220F7D
:106FA000331F280F391F280F391F30930E082093E5
:106FB0000D088091F9019091FA018C01000F111FC9
:106FC000000F111F080F191F080F191F10931E081B
:106FD00000931D0880913E06C82EDD24EE24FF2478
:106FE000442737FD4095542FC701B6010E94137AFC
:106FF0004B015C016093320370933303809334033D
:10700000909335039801442737FD4095542FC701CD
:10701000B6010E94137ADC01CB0180932A0390937E
:107020002B03A0932C03B0932D0380920E03909218
:107030000F03A0921003B092110380930603909364
:107040000703A0930803B093090310920203109260
:10705000030310920403109205038091160190918E
:107060001701A0911801B09119019093C705809361
:10707000C6051092EE011092ED011092F2021092EC
:10708000F3021092F4021092F50200919001109117
:1070900091011093F1020093F00284E690E0909346
:1070A0008D0180938C0182E390E09093DD018093C9
:1070B000DC01809163069927AA27BB27BC01CD017B
:1070C00024EC39E040E050E00E94137ADC01CB016F
:1070D0008856954CAF4FBF4F80938801909389019C
:1070E000A0938A01B0938B01809164069927AA2707
:1070F000BB27BC01CD010E94137ADC01CB0188566D
:10710000954CAF4FBF4F8093840190938501A0931E
:107110008601B09387011092480110924701C8017F
:10712000AA2797FDA095BA2F2091430130914401E1
:107130004091450150914601BC01CD010E94137A56
:10714000DC01CB018093190890931A08A0931B08C7
:10715000B0931C081092ED021092EC0281E0809333
:1071600001010E94BF678091A20284608093A20205
:107170008FEF8093990810929A0880E280939B0881
:10718000C9EDD2E0A7E2B6E007E08D91E82FFF2736
:10719000EE0FFF1FEF5AF84F80819181815889933C
:1071A000015007FFF2CF84E68093D8028091DA0184
:1071B000882311F0469A579A80914703909148038B
:1071C00080569940815C9B4228F08091FB0381604E
:1071D0008093FB038091450390914603805699402C
:1071E000815C9B4228F08091FB0382608093FB03CB
:1071F00080914303909144038C529140895795406C
:1072000028F08091FB0384608093FB0380913D0311
:1072100090913E038C529140835C914028F0809184
:10722000FB0388608093FB0380913B0390913C03B8
:107230008C529140835C914028F08091FB038061E7
:107240008093FB03809137039091380380509240E4
:107250008355914028F08091FB0380628093FB036B
:1072600086E480937F01ECE0CDB7DEB70C94C47A5E
:10727000A3E1B0E0EEE3F9E30C94A27A809143033A
:10728000909144032091FB013091FC01821B930BF0
:107290009093130880931208809105029091060242
:1072A00097FD07969C0113E0359527951A95E1F710
:1072B0003093D2072093D10780910302909104026A
:1072C00097FD0796B3E095958795BA95E1F790936A
:1072D000C3078093C2073093DD072093DC079093A8
:1072E000D5078093D40780910D0890910E08AC01CA
:1072F000440F551F480F591F2091F7013091F80195
:10730000C901880F991F880F991F820F931F820F41
:10731000931F480F591F57FF02C04D5F5F4F559590
:1073200047955595479550930E0840930D088091C9
:107330001D0890911E08AC01440F551F480F591F9E
:107340002091F9013091FA01C901880F991F880F26
:10735000991F820F931F820F931F480F591F57FFCA
:1073600002C04D5F5F4F5595479555954795509392
:107370001E0840931D082091F7013091F801C901C2
:10738000880F991F880F991F820F931F820F931FD9
:107390009C01442737FD4095542F80912203909102
:1073A0002303A0912403B0912503820F931FA41FF0
:1073B000B51F8093220390932303A0932403B093DB
:1073C00025032091F9013091FA01C901880F991F15
:1073D000880F991F820F931F820F931F9C014427D0
:1073E00037FD4095542F80911E0390911F03A0916B
:1073F0002003B0912103820F931FA41FB51F809318
:107400001E0390931F03A0932003B0932103809148
:10741000E6079091E7072091F7013091F801820F7C
:10742000931F9093E7078093E6078091150890914A
:1074300016082091F9013091FA01820F931F909361
:107440001608809315088091390390913A030196AC
:1074500090933A03809339038091C4059091C505B8
:107460002091370330913803821B930B9C014427F2
:1074700037FD4095542F80911A0390911B03A091E2
:107480001C03B0911D03820F931FA41FB51F80938F
:107490001A0390931B03A0931C03B0931D038FEC5E
:1074A00080937A001092100120910A0330910B030F
:1074B00040910C0350910D0329873A874B875C87D5
:1074C00029543B46414050402CF028E43BE641E043
:1074D00050E00DC089859A85AB85BC85885B944951
:1074E000AE4FBF4F4CF428EB34E94EEF5FEF2D83E6
:1074F0003E834F83588708C089859A85AB85BC85B4
:107500008D839E83AF83B88720911203309113033C
:1075100040911403509115032D873E874F87588B58
:1075200029543B46414050402CF028E43BE641E0E2
:1075300050E00DC08D859E85AF85B889885B9449E4
:10754000AE4FBF4F4CF428EB34E94EEF5FEF298389
:107550003A834B835C8308C08D859E85AF85B8894F
:1075600089839A83AB83BC83A0911208B0911308DE
:10757000BB8BAA8BFD01CF01AA2797FDA095BA2F3F
:10758000A0900203B0900303C0900403D0900503C1
:10759000A80EB91ECA1EDB1EA0920203B0920303FE
:1075A000C0920403D0920503E0901908F0901A08E5
:1075B00000911B0810911C08E80EF91E0A1F1B1FE2
:1075C000E0921908F0921A0800931B0810931C0807
:1075D000F091BD02F98BFF2309F098C18091BC02A4
:1075E000882309F093C18091090886FF8FC180919B
:1075F000C2079091C307AA2797FDA095BA2FBC0197
:10760000CD0129813A814B815C810E94137A9B01D3
:10761000AC0197FF04C02150384F4F4F5F4FBBE084
:107620005595479537952795BA95D1F780916B0178
:10763000682E772488249924CA01B901A4019301F2
:107640000E94137ADC01CB0180935303909354037F
:10765000A0935503B0935603B7FF04C08150904FD9
:10766000AF4FBF4F1C012D01ACE0559447943794A8
:107670002794AA95D1F72092530330925403409255
:107680005503509256038091D1079091D207AA27B3
:1076900097FDA095BA2FBC01CD012D813E814F8170
:1076A00058850E94137A97FF04C06150784F8F4F1E
:1076B0009F4FFBE09595879577956795FA95D1F75C
:1076C000A40193010E94137ADC01CB01809357033C
:1076D00090935803A0935903B0935A03B7FF04C083
:1076E0008150904FAF4FBF4F9C01AD01ECE05595DD
:1076F000479537952795EA95D1F72093570330930F
:1077000058034093590350935A0380915303909127
:1077100054039093BA078093B907809157039091CF
:1077200058039093BE078093BD072219330944097B
:1077300055092093570330935803409359035093AE
:107740005A03E20EF31E041F151FE0921908F0926F
:107750001A0800931B0810931C0880916A01882363
:10776000B1F457FF04C02F5F3F4F4F4F5F4F559508
:10777000479537952795A21AB30AC40AD50AA0924D
:107780000203B0920303C0920403D09205032A8936
:107790003B8979010027F7FC0095102F8091570352
:1077A00090915803A0915903B0915A03E80EF91E25
:1077B0000A1F1B1FC801B70129813A814B815C81D7
:1077C0000E94137A9B01AC0197FF04C02150384FEF
:1077D0004F4F5F4F6BE055954795379527956A95C5
:1077E000D1F780916C01A82EBB24CC24DD24CA01E2
:1077F000B901A60195010E94137ADC01CB018093A7
:107800004B0390934C03A0934D03B0934E03B7FFEB
:1078100004C08150904FAF4FBF4F3C014D013CE041
:1078200095948794779467943A95D1F760924B0337
:1078300070924C0380924D0390924E03C801B701A1
:107840002D813E814F8158850E94137A97FF04C095
:107850006150784F8F4F9F4F2BE095958795779587
:1078600067952A95D1F7A60195010E94137ADC014C
:10787000CB0180934F0390935003A0935103B09397
:107880005203B7FF04C08150904FAF4FBF4FAC01C0
:10789000BD018CE075956795579547958A95D1F709
:1078A00040934F03509350036093510370935203DE
:1078B0002A893B8937FF03C0309521953F4F2134FA
:1078C0003105E4F1D401C30197FE07C0B095A0953E
:1078D000909581959F4FAF4FBF4F81389105A1057E
:1078E000B10584F4DB01CA0177FF07C0B095A0950C
:1078F000909581959F4FAF4FBF4F81389105A1055E
:10790000B105E4F081E08093EE0218C01092BE074A
:107910001092BD071092BA071092B90710924F0348
:1079200010925003109251031092520310924B0385
:1079300010924C0310924D0310924E0380914F030E
:1079400090915003A0915103B0915203BC01CD011D
:1079500024E630E040E050E00E94877AE0904B035C
:10796000F0904C03E21AF30AF092D007E092CF07AE
:1079700080914B0390914C03A0914D03B0914E0325
:10798000BC01CD0124E630E040E050E00E94877A5F
:10799000DA01C90120914F03309150038C01021B81
:1079A000130B1093C5070093C40780914301909176
:1079B0004401A0914501B0914601BC01CD0128E6EA
:1079C00031E040E050E00E94137A20911908309194
:1079D0001A0840911B0850911C08261737074807C2
:1079E000590764F0261B370B480B590B20931908D5
:1079F00030931A0840931B0850931C0820911908D3
:107A000030911A0840911B0850911C0857FF0CC078
:107A1000260F371F481F591F2093190830931A0843
:107A200040931B0850931C086091C2077091C307D4
:107A30006E0D7F1D9B01442737FD4095542F80918B
:107A4000060390910703A0910803B0910903820FE8
:107A5000931FA41FB51F8093060390930703A09361
:107A60000803B09309038091C2029091C302681B7E
:107A7000790BCB01AA2797FDA095BA2F29853A85C6
:107A80004B855C85820F931FA41FB51F80930A034B
:107A900090930B03A0930C03B0930D03C09084014B
:107AA000D0908501E0908601F0908701C816D90634
:107AB000EA06FB06C4F488EA91E6A0E0B0E08C197F
:107AC0009D09AE09BF0980930A0390930B03A0930D
:107AD0000C03B0930D038093060390930703A093C8
:107AE0000803B093090322273327A9012C193D0964
:107AF0004E095F0980910A0390910B03A0910C033A
:107B0000B0910D0382179307A407B507B4F4D7010A
:107B1000C601885A9146A040B04080930A039093D2
:107B20000B03A0930C03B0930D0380930603909373
:107B30000703A0930803B09309036091D1077091E4
:107B4000D207600F711F9B01442737FD4095542FCA
:107B500080910E0390910F03A0911003B091110337
:107B6000820F931FA41FB51F80930E0390930F03E2
:107B7000A0931003B09311038091C0029091C102B1
:107B8000681B790BCB01AA2797FDA095BA2F2D85ED
:107B90003E854F855889820F931FA41FB51F809380
:107BA000120390931303A0931403B0931503E09072
:107BB0008801F090890100918A0110918B01E816EB
:107BC000F9060A071B07C4F488EA91E6A0E0B0E0D2
:107BD0008E199F09A00BB10B80931203909313038E
:107BE000A0931403B093150380930E0390930F0397
:107BF000A0931003B093110322273327A9012E1954
:107C00003F09400B510B8091120390911303A091F7
:107C10001403B091150382179307A407B507B4F4B2
:107C2000D801C701885A9146A040B0408093120302
:107C300090931303A0931403B093150380930E0342
:107C400090930F03A0931003B0931103809102034C
:107C500090910303A0910403B09105038093160350
:107C600090931703A0931803B09319038091120304
:107C700090911303A0911403B091150380933203E4
:107C800090933303A0933403B093350380910A0398
:107C900090910B03A0910C03B0910D0380932A03E4
:107CA00090932B03A0932C03B0932D0380910E038C
:107CB00090910F03A0911003B091110380932E03B4
:107CC00090932F03A0933003B09331038091060368
:107CD00090910703A0910803B091090380932603B4
:107CE00090932703A0932803B093290380911C014C
:107CF00090911D0197FD079603E0959587950A954C
:107D0000E1F79093D2078093D10780911A01909167
:107D10001B0197FD079613E0959587951A95E1F756
:107D20009093C3078093C2078091FF019091000256
:107D30000F9734F488E19CEF9093D2078093D1079A
:107D40008091FF0190910002079734F480E398EF4F
:107D50009093D2078093D107209102012A30A9F491
:107D60008091FF0190910002835F934034F088EE90
:107D700093E09093D2078093D1078091FF01909177
:107D800000028A5F9340DCF014C08091FF01909163
:107D90000002815D974034F088EE93E09093D20723
:107DA0008093D1078091FF0190910002805E9740FF
:107DB00034F080ED97E09093D2078093D1078091C3
:107DC000FD019091FE010F9734F488E19CEF9093B0
:107DD000C3078093C2078091FD019091FE01079730
:107DE00034F480E398EF9093C3078093C2072A305E
:107DF000A9F48091FD019091FE01835F934034F0DE
:107E000088EE93E09093C3078093C2078091FD01B1
:107E10009091FE018A5F9340DCF014C08091FD01D7
:107E20009091FE01815D974034F088EE93E090934D
:107E3000C3078093C2078091FD019091FE01805E8F
:107E4000974034F080ED97E09093C3078093C2078A
:107E500060917601662309F4AFC040911C015091F6
:107E60001D0180915B0390915C03481B590B50935B
:107E700062034093610320911C0130911D01280F82
:107E8000391F37FF02C02F5F3F4F3595279530933D
:107E90005C0320935B03413851051CF080E890E0BF
:107EA00005C040585F4F34F480E89FEF9093620321
:107EB0008093610340911A0150911B0180915D03F1
:107EC00090915E03481B590B5093600340935F03EE
:107ED00020911A0130911B01280F391F37FF02C072
:107EE0002F5F3F4F3595279530935E0320935D03B9
:107EF000413851051CF080E890E005C040585F4FC4
:107F000034F480E89FEF9093600380935F03462FE3
:107F100055278091610390916203849FB001859FF2
:107F2000700D949F700D11249B0177FF02C0215F9B
:107F30003F4FF4E035952795FA95E1F78091D10709
:107F40009091D207820F931F9093D2078093D1070D
:107F500080915F0390916003849FD001859FB00D55
:107F6000949FB00D1124AD019D01B7FF02C0215FA8
:107F70003F4FE4E035952795EA95E1F78091C207F8
:107F80009091C307820F931F9093C3078093C207FA
:107F900080911C0190911D01860F971F90931D01E8
:107FA00080931C0180911A0190911B01840F951FF1
:107FB00090931B0180931A010091D4071091D5076B
:107FC0008091B9079091BA07101611065CF59C01D3
:107FD00097FF04C022273327281B390BC901AA2782
:107FE00097FDA095BA2F20916A0133274427552782
:107FF000BC01CD010E94137A9B01AC0197FF04C024
:10800000215C3F4F4F4F5F4F76E055954795379531
:1080100027957A95D1F78091CF079091D007820F5D
:10802000931F27C097FF03C0909581959F4FAA2764
:1080300097FDA095BA2F20916A0133274427552731
:10804000BC01CD010E94137A9B01AC0197FF04C0D3
:10805000215C3F4F4F4F5F4F66E0559547953795F1
:1080600027956A95D1F78091CF079091D007821B11
:10807000930B9093D0078093CF07E090DC07F090AC
:10808000DD078091BD079091BE071E141F045CF5AB
:108090009C0197FF04C022273327281B390BC901F5
:1080A000AA2797FDA095BA2F20916A01332744276C
:1080B0005527BC01CD010E94137A9B01AC0197FFAB
:1080C00004C0215C3F4F4F4F5F4F96E05595479559
:1080D000379527959A95D1F78091C4079091C50758
:1080E000820F931F27C097FF03C0909581959F4FE4
:1080F000AA2797FDA095BA2F20916A01332744271C
:108100005527BC01CD010E94137A9B01AC0197FF5A
:1081100004C0215C3F4F4F4F5F4F86E05595479518
:10812000379527958A95D1F78091C4079091C50717
:10813000821B930B9093C5078093C4078091090815
:1081400087FF44C0B989BB2309F040C08091BC02BD
:108150008823E1F5E1E0EE16E1E0FE064CF08091C7
:10816000D1079091D2078E0D9F1D805091400DC078
:10817000F0E0EF16FFEFFF0664F48091D1079091D5
:10818000D2078E0D9F1D80509F4F9093D2078093F2
:10819000D10721E0013012074CF08091C207909185
:1081A000C307800F911F805091400CC03FEF0030FB
:1081B000130764F48091C2079091C307800F911F49
:1081C00080509F4F9093C3078093C207E2E1CD5E3A
:1081D0000C94BE7A8091D702882301F58091A20287
:1081E0008C7F8093A202A0E0B4E0E0EFF6E09BE099
:1081F0008091BB01882309F48C938D918183128235
:108200009150389697FFF4CF8091BB01882359F0A5
:108210008091BB0181508093BB0105C08091A20277
:1082200081608093A20280912602882319F0109227
:10823000260208958093280280932A0280912402C6
:108240008E7F8093240285EA8093BC000895CF93AB
:10825000DF93A9EDB2E0C7E2D6E057E09991E92FAC
:10826000FF27EE0FFF1FEF5AF84F0190F081E02D2E
:10827000E158FF4FEF3FF10521F01CF0EFEFF0E088
:1082800004C0F7FF02C0E0E0F0E0993111F4EC9394
:108290001BC04C91242F3327E217F307A9F0CF011D
:1082A000821B930B97FD03969595879595958795DA
:1082B000242F280F2C93822F9927E817F90714F4FD
:1082C000215001C02F5F2C935150119657FFC6CFFC
:1082D00080913106883F38F0EFEFF0E0E81BF109BC
:1082E000E752FD4F808180937C0180917C0188233F
:1082F00029F0843618F084E680937C01809133065F
:10830000883F38F0EFEFF0E0E81BF109E752FD4F4E
:10831000808180937A0180917A01882329F08436C4
:1083200018F084E680937A0180914006883F38F007
:10833000EFEFF0E0E81BF109E752FD4F80818093F9
:108340007501809175018B3010F48AE002C08F3F77
:1083500011F48093750180916D06883F38F0EFEF3E
:10836000F0E0E81BF109E752FD4F80818093E807B8
:108370008091E807863010F485E002C08F3F11F449
:108380008093E80780916F06883F38F0EFEFF0E0C8
:10839000E81BF109E752FD4F80818093100880911E
:1083A0001008863010F485E002C08F3F11F48093EE
:1083B000100880915A06883F38F0EFEFF0E0E81B94
:1083C000F109E752FD4F80818093E50780915B06BC
:1083D000883F38F0EFEFF0E0E81BF109E752FD4F7E
:1083E00080818093BF0780915C06883F38F0EFEF73
:1083F000F0E0E81BF109E752FD4F80818093EE0722
:1084000080913206883F38F0EFEFF0E0E81BF10989
:10841000E752FD4F808180937B0180913506883F34
:1084200038F0EFEFF0E0E81BF109E752FD4F8081F3
:108430008093790180913706883F38F0EFEFF0E0C4
:10844000E81BF109E752FD4F80818093770180910D
:108450003F06883F38F0EFEFF0E0E81BF109E75204
:10846000FD4F80818093780180914106883F38F0EC
:10847000EFEFF0E0E81BF109E752FD4F80818093B8
:10848000740180914206883F38F0EFEFF0E0E81B7E
:10849000F109E752FD4F8081809376018091430678
:1084A000883F38F0EFEFF0E0E81BF109E752FD4FAD
:1084B00080818093730180914406883F38F0EFEF0C
:1084C000F0E0E81BF109E752FD4F808180937201D3
:1084D00080914A06883F38F0EFEFF0E0E81BF109A1
:1084E000E752FD4F80818093700180914B06883F59
:1084F00038F0EFEFF0E0E81BF109E752FD4F808123
:108500008093B70280914C06883F38F0EFEFF0E09F
:10851000E81BF109E752FD4F80818093B6028091FC
:108520004D06883F38F0EFEFF0E0E81BF109E75225
:10853000FD4F80818093B50280914E06883F38F0D0
:10854000EFEFF0E0E81BF109E752FD4F80818093E7
:10855000B40280916806883F38F0EFEFF0E0E81B46
:10856000F109E752FD4F80818093B3028091690643
:10857000883F38F0EFEFF0E0E81BF109E752FD4FDC
:1085800080818093B20280916A06883F38F0EFEFD5
:10859000F0E0E81BF109E752FD4F80818093B102C2
:1085A00080916B06883F38F0EFEFF0E0E81BF109AF
:1085B000E752FD4F80818093B00280914F06883F43
:1085C00038F0EFEFF0E0E81BF109E752FD4F808152
:1085D00080936F0180915306883F38F0EFEFF0E011
:1085E000E81BF109E752FD4F808180936E01809175
:1085F0005D06883F38F0EFEFF0E0E81BF109E75245
:10860000FD4F808180936D0180916006883F38F036
:10861000EFEFF0E0E81BF109E752FD4F8081809316
:108620006C0180916106883F38F0EFEFF0E0E81BC5
:10863000F109E752FD4F808180936B0180916206C2
:10864000883F38F0EFEFF0E0E81BF109E752FD4F0B
:10865000808180936A0180918906883F38F0EFEF2E
:10866000F0E0E81BF109E752FD4F8081809368013B
:1086700080912F068093090880918C068093ED07E6
:1086800080916706883F38F0EFEFF0E0E81BF109D2
:10869000E752FD4F80818093690180918206883F77
:1086A00038F0EFEFF0E0E81BF109E752FD4F808171
:1086B0008093200880917001282F33272F5F3F4F30
:1086C0008CE398E2B9010E94527A70937E01609324
:1086D0007D0180913D068093110880913C06809336
:1086E000D607909184069333C8F181E08093AF025E
:1086F000983F58F0EFEFF0E0E91BF109E752FD4F2A
:108700008081823310F41092AF0280917F0120911A
:10871000AF02821799F0833070F4222319F08CEDA8
:1087200095E002C088EC90E09093DD018093DC013D
:1087300020937F0103C0815080937F018091600866
:108740009091610897FF0FC08091AF02882359F084
:108750008091FB0380688093FB0305C01092AF02F9
:108760008AE080937F01809160089091610897FF73
:108770001DC08091D7028823C9F08091AF02882361
:10878000A9F080910801909109018F5F9F4F71F4CA
:1087900088E99AE39093DD018093DC0180E094EA1C
:1087A00090930901809308011092AF028091AF026B
:1087B000882369F08091A10281608093A102809159
:1087C0006C01823D48F4825E80936C0105C080910B
:1087D000A1028E7F8093A102C0916801CC2369F130
:1087E0008091CE029091CF02A091D002B091D1029F
:1087F000BC01CD0124E630E040E050E00E94877AE1
:10880000DA01C9012C2F33274427552728173907A8
:108810004A075B0794F4CA01B90124E630E040E05E
:1088200050E00E94137ADC01CB018093CE0290933A
:10883000CF02A093D002B093D102DF91CF910895DF
:10884000ABE1B0E0E6E2F4E40C94A27A0E9438399D
:10885000E090E202F090E302FA82E9828091D6078A
:1088600099270A96E816F90614F49A838983809169
:10887000D802843608F066C08091A10282FD62C0F1
:108880008091770390917803009731F0019790934E
:108890007803809377030BC01092D7029093A402C1
:1088A0008093A3028091A2028D7E8093A202809188
:1088B00002018A3011F0843110F0289A01C0289802
:1088C0008091A3029091A402895E9340C0F18091AF
:1088D0004706282F33273A8329838091A20280619B
:1088E0008093A20280912306A82FBB27AA0FBB1F4B
:1088F000FD01EB57F84F1182108280912406282F3A
:108900003327220F331FC9018B57984FFC01118267
:108910001082AF5AB84F11961C921E922F5A384FA0
:10892000D90111961C921E9280912606E82FFF27EE
:10893000EE0FFF1FEF5AF84F11821082B9C210924A
:10894000D702B6C28091D8028D3808F4B1C28091A6
:10895000A2028F7E8093A2029091480682E3989FA4
:10896000C00111249093780380937703E981FA8101
:10897000B9978CF08091D702882369F08091A30287
:108980009091A402FFEF8F3F9F0729F001969093EB
:10899000A4028093A3028091A3029091A4028F3F2E
:1089A000910509F008F51092FA021092FB0210925C
:1089B000FC021092FD021092F6021092F702109241
:1089C000F8021092F902109263031092640310925D
:1089D0006503109266031092020310920303109233
:1089E00004031092050305C08091A2028260809367
:1089F000A20280912506E82FFF27EE0FFF1FEF5AF6
:108A0000F84F80819181813591050CF445C1209109
:108A1000D702222309F040C180912606E82FFF27C4
:108A2000EE0FFF1FEF5AF84F808191818C34910532
:108A30000CF408C1809179038F5F80937903893C9E
:108A400008F42AC1809102018C3010F4299801C0E9
:108A5000299A1092D702109279031092A4021092D0
:108A6000A30230912306E32FFF27EE0FFF1FEF5ADB
:108A7000F84F8081918187349105B4F48091240668
:108A8000E82FFF27EE0FFF1FEF5AF84F80819181EB
:108A90000190F081E02DF7FF03C0F095E195FF4FC5
:108AA000E734F1050CF478C041E020912406A22FB0
:108AB000BB27AA0FBB1FAF5AB84F8D919C9111973E
:108AC0008734910544F0E32FFF27EE0FFF1FEF5A85
:108AD000F84F808191818D919C918734910574F03C
:108AE00080912306E82FFF27EE0FFF1FEF5AF84F64
:108AF00080819181873491050CF042E0E22FFF27BD
:108B0000EE0FFF1FEF5AF84F808191818634910557
:108B100074F480912306E82FFF27EE0FFF1FEF5A12
:108B2000F84F80819181873491050CF043E0E22F6A
:108B3000FF27EE0FFF1FEF5AF84F808191818A5B6C
:108B40009F4F74F480912306E82FFF27EE0FFF1F3D
:108B5000EF5AF84F80819181873491050CF044E001
:108B6000E22FFF27EE0FFF1FEF5AF84F8081918110
:108B70008A5B9F4F74F480912306E82FFF27EE0F46
:108B8000FF1FEF5AF84F80819181863491050CF4D4
:108B900045E0842F0E94362B80912406E82FFF2782
:108BA000EE0FFF1FEF5AF84F808191810190F08105
:108BB000E02DF7FF03C0F095E195FF4F7E97BCF4E1
:108BC00080912306E82FFF27EE0FFF1FEF5AF84F83
:108BD000808191818A5B9F4F54F481E080931604D9
:108BE00088EE93E09093DD018093DC0155C00E94F4
:108BF000322C0E94E32A80E00E94C206809149063E
:108C00000E9415768091090880FF10C080911401A0
:108C100090911501875B934038F4809114019091F5
:108C200015018E5E924010F40E94421A1092DA01F1
:108C300080E00E94863681E080937C038093DA0195
:108C4000579A21C080819181855B9F4F1CF580914F
:108C500079038F5F80937903893CF0F08091020162
:108C60008C3010F4299801C0299A1092D7021092E2
:108C700079031092A4021092A30281E00E9486362A
:108C800081E080937C030E94322C68E770E00E94B0
:108C9000C43502C02093790380912506E82FFF2771
:108CA000EE0FFF1FEF5AF84F808191818B5A9F4F33
:108CB0000CF0FEC03091D702E0912606332309F074
:108CC000CCC0FF27EE0FFF1FEF5AF84F8081918134
:108CD000855B9F4F0CF0BEC020918506E22FFF27D9
:108CE000EE0FFF1FEF5AF84F80819181855B9F4FF8
:108CF0001CF0222309F0AEC080917A038F5F80932D
:108D00007A03893C08F4D4C030937A038091FB0342
:108D1000882309F098C080917C03882309F493C0CC
:108D20008091AF03882309F08EC081E090E090939A
:108D3000A4028093A30281E08093D7021092630380
:108D4000109264031092650310926603109202035E
:108D50001092030310920403109205031092FE0276
:108D60001092FF02109200031092010380913E06C0
:108D7000E82EFF240027112780910D0890910E08FE
:108D80009C01442737FD4095542FC801B7010E942C
:108D9000137ADC01CB018093120390931303A09309
:108DA0001403B093150380911D0890911E089C0137
:108DB000442737FD4095542FC801B7010E94137A0C
:108DC000DC01CB0180930A0390930B03A0930C0367
:108DD000B0930D038091320390913303A09134033B
:108DE000B091350380930E0390930F03A09310036B
:108DF000B093110380912A0390912B03A0912C032F
:108E0000B0912D038093060390930703A09308036A
:108E1000B09309031092FA021092FB021092FC0226
:108E20001092FD021092F6021092F7021092F802D0
:108E30001092F9028091A20288608093A20284E6D7
:108E400080937D0335C08CED95E09093DD01809398
:108E5000DC012EC010927A032BC0FF27EE0FFF1FFC
:108E6000EF5AF84F808191818C349105FCF020916C
:108E70008506E22FFF27EE0FFF1FEF5AF84F808184
:108E80009181855B9F4F14F0222381F480917B03B5
:108E90008F5F80937B03893C58F01092D702109229
:108EA0007B031092A4021092A30202C010927B03D3
:108EB00080914101815080934101809141018F3F18
:108EC00021F08091A20284FFA9C30E942741B090A3
:108ED000390680918603909187039C01220F331FEE
:108EE000280F391FC0902306AC2DBB27AA0FBB1F2C
:108EF000FD01EF5AF84F4B2D552780819181849FBA
:108F0000F001859FF00D949FF00D11242E0F3F1F4F
:108F100037FF02C02D5F3F4FB90175956795759575
:108F20006795AB57B84F80913A06082F11278D915E
:108F30009C91809F7001819FF00C909FF00C1124F8
:108F40006E0D7F1D70938703609386038091880365
:108F5000909189039C01220F331F280F391FD09055
:108F60002406AD2DBB27AA0FBB1FFD01EF5AF84FFA
:108F700080819181849FF001859FF00D949FF00D79
:108F800011242E0F3F1F37FF02C02D5F3F4FA90155
:108F90005595479555954795AB57B84F8D919C91F1
:108FA000809F7001819FF00C909FF00C11244E0D5A
:108FB0005F1D50938903409388038091AF028823FB
:108FC00009F448C0CB0177FD0396DC01B595A79560
:108FD000B595A795CA0157FD0396FC01F595E79550
:108FE000F595E79580919E01682F772767FD70952D
:108FF0006A9F90016B9F300D7A9F300D11248091F4
:10900000B103482F552747FD50954E9FC0014F9FF4
:10901000900D5E9F900D1124280F391F37FF02C05D
:10902000295F3F4F93E0359527959A95E1F7309367
:10903000E9022093E8026E9F90016F9F300D7E9FA2
:10904000300D11244A9FC0014B9F900D5A9F900DE7
:1090500011243FC080918306E82FFF27E75BFE4F76
:10906000868180939E0190819093B103A82FBB27A6
:10907000A7FDB095A69F9001A79F300DB69F300D1C
:109080001124E92FFF27E7FDF095E49FC001E59F3C
:10909000900DF49F900D1124280F391F37FF02C047
:1090A000295F3F4F83E0359527958A95E1F7309307
:1090B000E9022093E802A49F9001A59F300DB49F80
:1090C000300D1124E69FC001E79F900DF69F900D93
:1090D0001124281B390B37FF02C0295F3F4F03E0E3
:1090E000359527950A95E1F73093E7022093E6023C
:1090F00080912606E82FFF27EE0FFF1FEF5AF84F4B
:1091000080819181909581959F4F9093E502809306
:10911000E4028530910514F0049705C00FEF8C3FF1
:10912000900734F404969093E5028093E40204C01F
:109130001092E5021092E4028091A203882309F4C0
:109140003EC0282F33278091E8029091E90297FDD5
:10915000079613E0959587951A95E1F7289FA0014A
:10916000299F500D389F500D1124CA0157FD0F96AD
:10917000B4E095958795BA95E1F79093E9028093CD
:10918000E8028091E6029091E70297FD0796A3E03E
:1091900095958795AA95E1F7289FB001299F700DB5
:1091A000389F700D1124CB0177FD0F96F4E0959553
:1091B0008795FA95E1F79093E7028093E602809015
:1091C000E8029090E9028091A5039091A603881A85
:1091D000990A9092E9028092E8020091E6021091C9
:1091E000E7028091A3039091A403081B190B10932D
:1091F000E7020093E60280912506E82FFF27EE0F95
:10920000FF1FEF5AF84FE080F1808FE790E0E80E03
:10921000F91EF092E302E092E20280917501992733
:10922000AA2797FDA095BA2FBC01CD010E9487798E
:10923000DC01CB0120E030E040E251E4BC01CD0193
:109240000E94F578DC01CB01BC01CD010E94597967
:10925000DC01CB0180931708809174018093EF07A4
:10926000809173019927AA2797FDA095BA2FBC0179
:10927000CD010E948779DC01CB0120E030E040E2A3
:1092800051E4BC01CD010E94F578DC01CB01BC01A9
:10929000CD010E945979DC01CB018093C9078091EF
:1092A00072018093DE078091220480FF59C0809173
:1092B0002008813808F454C080911B04992787FD49
:1092C00090952B2D3327829FD001839FB00D929FC5
:1092D000B00D11248A0E9B1E9092E9028092E80242
:1092E00080911C04992787FD9095829FF001839FB0
:1092F000F00D929FF00D11240E0F1F1F1093E70227
:109300000093E60280911D04282F332727FD309516
:109310008091E4029091E502820F931F9093E50201
:109320008093E40280911F04282F332727FD309576
:10933000809134069927289F8001299F100D389F1E
:10934000100D1124109348010093470180911E04D1
:1093500099278E159F0524F49093E3028093E202EF
:109360008091E2029091E30297FF04C01092E30221
:109370001092E2028091090882FF02C01092EF076A
:109380004091E8025091E902CA0157FD03969C0101
:10939000359527953595279537FF03C0309521954D
:1093A0003F4F8091A7029091A80282179307B4F4CF
:1093B000CA0157FF03C0909581959F4F97FD039673
:1093C00095958795959587959093A8028093A70288
:1093D0008536910544F084E690E001C001979093B2
:1093E000A8028093A7024091E6025091E702CA01C9
:1093F00057FD03969C01359527953595279537FFA1
:1094000003C0309521953F4F8091A5029091A6020F
:1094100082179307B4F4CA0157FF03C09095819552
:109420009F4F97FD03969595879595958795909372
:10943000A6028093A5028536910544F084E690E06B
:1094400001C001979093A6028093A5028091A20289
:1094500084FF08C01092A8021092A7021092A602E0
:109460001092A502ED2DFF27EE0FFF1FEF5AF84FC8
:1094700040915E06242F3327808191812817390778
:1094800044F480918A0682FF04C081E08093BB028D
:1094900013C0ED2DFF27EE0FFF1FEF5AF84F842F5B
:1094A000992720915F06821B91092081318128171D
:1094B000390714F41092BB0240912406E42FFF27D1
:1094C000EE0FFF1FEF5AF84F50915E06852F992738
:1094D00022273327281B390B80819181821793071C
:1094E00044F480918A0683FF04C081E08093BA022D
:1094F00016C08091BA02882391F0E42FFF27EE0F67
:10950000FF1FEF5AF84F80915F069927851B91093D
:10951000208131818217930714F41092BA02EC2D46
:10952000FF27EE0FFF1FEF5AF84F40915E06242FE2
:109530003327808191812817390744F480918A0666
:1095400080FF04C081E08093B80217C08091B80208
:10955000882399F0EC2DFF27EE0FFF1FEF5AF84FED
:10956000842F992720915F06821B910920813181E8
:109570002817390714F41092B80240912306E42FFB
:10958000FF27EE0FFF1FEF5AF84F50915E06852F11
:10959000992722273327281B390B80819181821735
:1095A000930744F480918A0681FF04C081E0809390
:1095B000B90216C08091B902882391F0E42FFF27E9
:1095C000EE0FFF1FEF5AF84F80915F069927851B1A
:1095D0009109208131818217930714F41092B90206
:1095E0008091BB02882319F48091BA02811181E035
:1095F0008093BC028091B802882321F48091B90243
:10960000882351F081E08093BD021092BC02109239
:10961000BB021092BA0202C08093BD028091BC02CC
:10962000882321F48091BD02882369F080915D0632
:10963000992729813A818217930714F49A838983A1
:1096400081E08093EE028091A10299279C01247011
:10965000307082FF2DC08091A5039091A603909554
:1096600081959F4F9093E9028093E8028091A30334
:109670009091A403909581959F4F9093E7028093DA
:10968000E60280918201909183019093E30280939E
:10969000E202809109088B778B668093090880919C
:1096A000ED078C7B8093ED0788EC80937B011EC0D7
:1096B0008091A20284FF1AC03093E5022093E40255
:1096C0003093E9022093E8023093E7022093E60208
:1096D0009AE59093170888E78093EF079093C9075E
:1096E0008093DE071092BC021092BD028091E107C8
:1096F0009091E207A091E307B091E4072091320333
:10970000309133034091340350913503820F931FFE
:10971000A41FB51F8093E1079093E207A093E3078E
:10972000B093E4078091E9079091EA07A091EB07D5
:10973000B091EC07E0902A03F0902B0300912C03EA
:1097400010912D03EB82FC820D831E838E0D9F1DD5
:10975000A01FB11F8093E9079093EA07A093EB073E
:10976000B093EC078091D8079091D907A091DA07C0
:10977000B091DB07E0902E03F0902F0300913003AF
:1097800010913103EF82F88609871A878E0D9F1D8D
:10979000A01FB11F8093D8079093D907A093DA0731
:1097A000B093DB078091CA079091CB07A091CC07BB
:1097B000B091CD07E0902603F09027030091280395
:1097C00010912903EB86FC860D871E878E0D9F1D49
:1097D000A01FB11F8093CA079093CB07A093CC071B
:1097E000B093CD07F090BD02FF86FF2029F4809151
:1097F000BC02882309F460C0109222031092230354
:10980000109224031092250310921E0310921F033E
:1098100010922003109221031092E1071092E207A8
:109820001092E3071092E4071092E9071092EA07FA
:109830001092EB071092EC071092D8071092D907FC
:109840001092DA071092DB071092CA071092CB072A
:109850001092CC071092CD078091120390911303C0
:10986000A0911403B091150380930E0390930F03FE
:10987000A0931003B093110380910A0390910B03FE
:10988000A0910C03B0910D038093060390930703FE
:10989000A0930803B09309031092EC011092EB011E
:1098A0001092C1021092C0021092C3021092C20222
:1098B0000F85002309F0F8C18091BC02882309F0CC
:1098C000F3C18091C4059091C505815092402CF45C
:1098D0008091D702882309F4E7C190909908A0905D
:1098E0003E0620900D0830900E0840901D085090C4
:1098F0001E0819140CF0E3C0BB24CC24DD24CA01DB
:10990000B901A60195010E94877A79018A018091A7
:10991000620890916308281A390AC101AA2797FDA5
:10992000A095BA2FE81AF90A0A0B1B0B6B817C81F0
:109930008D819E81A60195010E94877A59016A0155
:109940008091640890916508481A590AC201AA27B3
:1099500097FDA095BA2FA81AB90ACA0ADB0A292CC2
:10996000332427FC3094432C532CC801B701A201A7
:1099700091010E94137A97FF04C061507E4F8F4F70
:109980009F4F3B014C0109E095948794779467942D
:109990000A95D1F7C601B501A20191010E94137A7F
:1099A00097FF04C061507E4F8F4F9F4F5B016C014A
:1099B00019E0D594C794B794A7941A95D1F78091DC
:1099C000A7029091A802813491053CF48091A502F0
:1099D0009091A60281349105D4F0D401C30197FE81
:1099E00003C00196A11DB11D3C014D0195948794C2
:1099F00077946794D601C501D7FE03C00196A11DD7
:109A0000B11D5C016D01D594C794B794A794809162
:109A10002606E82FFF27EE0FFF1FEF5AF84F808131
:109A200091810190F081E02DF7FF03C0F095E19561
:109A3000FF4F7A97A4F0C401B30123E030E040E087
:109A400050E00E94877A39014A01C601B50123E03E
:109A500030E040E050E00E94877A59016A0180912D
:109A60009B08282F332727FD3095432F532F26158A
:109A700037054805590514F439014A01992787FD2E
:109A80009095909581959F4FAA2797FDA095BA2F05
:109A9000681679068A069B0614F43C014D012A15C6
:109AA0003B054C055D0514F459016A01A816B90679
:109AB000CA06DB060CF0D0C05C016D01CDC0EA2CFB
:109AC000FF2400271127CA01B901A80197010E94AC
:109AD000877A39014A01C101AA2797FDA095BA2FBB
:109AE000681A790A8A0A9B0A6B817C818D819E8122
:109AF000A80197010E94877A59016A01C201AA2729
:109B000097FDA095BA2FA81AB90ACA0ADB0AD40190
:109B1000C30197FE03C00F96A11DB11D3C014D016D
:109B2000F4E09594879477946794FA95D1F7D601E9
:109B3000C501D7FE03C00F96A11DB11D5C016D01CB
:109B4000E4E0D594C794B794A794EA95D1F78091AF
:109B5000A7029091A802813491053CF48091A5025E
:109B60009091A60281349105A4F0C401B30123E0D1
:109B700030E040E050E00E94877A39014A01C60196
:109B8000B50123E030E040E050E00E94877A5901BF
:109B90006A0180912606E82FFF27EE0FFF1FEF5A7C
:109BA000F84F808191810190F081E02DF7FF03C093
:109BB000F095E195FF4F7A97A4F0C401B30123E03B
:109BC00030E040E050E00E94877A39014A01C60146
:109BD000B50123E030E040E050E00E94877A59016F
:109BE0006A0189E180938E0121E262167104810489
:109BF00091042CF070E2672E712C812C912C30EEA8
:109C000063163FEF73063FEF83063FEF930644F47E
:109C100060EE662E6FEF762E6FEF862E6FEF962E2C
:109C200041E2A416B104C104D1042CF050E2A52EE7
:109C3000B12CC12CD12C50EEA5165FEFB5065FEF0D
:109C4000C5065FEFD50644F440EEA42E4FEFB42EC8
:109C50004FEFC42E4FEFD42E809112039091130337
:109C6000A0911403B091150386199709A809B909A1
:109C70008093120390931303A0931403B0931503DE
:109C800080910A0390910B03A0910C03B0910D03F6
:109C90008A199B09AC09BD0980930A0390930B03B1
:109CA000A0930C03B0930D038091EB019091EC0114
:109CB0008F3F910509F008F4C4C56F85662309F04C
:109CC0004EC58091BC02882309F049C58091EE02FF
:109CD000882309F044C570916606788B772309F4D0
:109CE0003EC58091E1079091E207A091E307B09112
:109CF000E407B7FF04C081509F4FAF4FBF4FE92E1D
:109D0000FA2E0B2F112707FD1A95E092E107F0922A
:109D1000E2070093E3071093E4078091E90790912D
:109D2000EA07A091EB07B091EC07B7FF04C08150A0
:109D30009F4FAF4FBF4F892F9A2FAB2FBB27A7FD48
:109D4000BA95898B9A8BAB8BBC8B8093E9079093E8
:109D5000EA07A093EB07B093EC0780913E06A82E8C
:109D6000BB24CC24DD242091220330912303409195
:109D7000240350912503C601B5010E94137A97FF71
:109D800004C061507F4F8F4F9F4F672E782E892ED2
:109D9000992487FC9A946092220370922303809204
:109DA00024039092250320911E0330911F034091BC
:109DB000200350912103C601B5010E94137A97FF39
:109DC00004C061507F4F8F4F9F4F272E382E492E52
:109DD000552447FC5A9420921E0330921F03409250
:109DE00020035092210380911A0390911B03A091AC
:109DF0001C03B0911D03B7FF04C081509F4FAF4FAC
:109E0000BF4F892F9A2FAB2FBB27A7FDBA95809301
:109E10001A0390931B03A0931C03B0931D03D80156
:109E2000C70186199709A809B90980936F03909310
:109E30007003A0937103B093720320916506E22E24
:109E4000FF2400271127BC01CD01A80197010E9422
:109E5000877A59016A0120937E0330937F034093F0
:109E600080035093810389899A89AB89BC898219BF
:109E70009309A409B5098093730390937403A09385
:109E80007503B0937603BC01CD01A80197010E9430
:109E9000877A209382033093830340938403509303
:109EA0008503D601C501D7FE04C081509F4FAF4F37
:109EB000BF4F892F9A2FAB2FBB27A7FDBA95909341
:109EC000C1028093C00257FF04C021503F4F4F4F43
:109ED0005F4FBB2757FDBA95A52F942F832F9093E3
:109EE000C3028093C2028091A7029091A80281349C
:109EF0009105DCF48091A5029091A6028134910530
:109F0000A4F480912606E82FFF27EE0FFF1FEF5ADB
:109F1000F84F808191810190F081E02DF7FF03C01F
:109F2000F095E195FF4F7A97E4F0809199088F3F83
:109F3000C1F48091C0029091C10297FD0196959560
:109F400087959093C1028093C0028091C202909144
:109F5000C30297FD0196959587959093C3028093D0
:109F6000C2028091D8079091D907A091DA07B091E9
:109F7000DB07B7FF04C081509F4FAF4FBF4F892F02
:109F80009A2FAB2FBB27A7FDBA958093D807909344
:109F9000D907A093DA07B093DB078091CA079091A5
:109FA000CB07A091CC07B091CD07B7FF04C081507B
:109FB0009F4FAF4FBF4F892F9A2FAB2FBB27A7FDC6
:109FC000BA958093CA079093CB07A093CC07B09320
:109FD000CD078091320390913303A0913403B09167
:109FE00035032F81388549855A85281B390B4A0B43
:109FF0005B0B20936703309368034093690350938E
:10A000006A0380912A0390912B03A0912C03B091B5
:10A010002D03EB84FC840D851E85E81AF90A0A0BD2
:10A020001B0BE0926B03F0926C0300936D03109393
:10A030006E0320936F03309370034093710350932A
:10A040007203E0927303F09274030093750310930C
:10A05000760380910E0390910F03A0911003B091AD
:10A060001103821B930BA40BB50B80930E039093EB
:10A070000F03A0931003B0931103809106039091F6
:10A080000703A0910803B09109038E199F09A00B43
:10A09000B10B8093060390930703A0930803B0933A
:10A0A000090388898823E1F02091EC023091ED02C8
:10A0B000213831054CF0809143039091440301967F
:10A0C000909344038093430320583F4F4CF4809176
:10A0D0004303909144030197909344038093430377
:10A0E0001092ED021092EC0281E090E090938B03CD
:10A0F00080938A03E0906F03F090700300917103E6
:10A1000010917203D801C70117FF07C0882799274C
:10A11000DC018E199F09A00BB10B81509240A04029
:10A12000B04034F084E090E090938B0380938A03F6
:10A130008091900390919103A0919203B091930329
:10A140002091E1073091E2074091E3075091E40745
:10A15000821B930BA40BB50B815E914BAF4FBF4F8E
:10A160008F539C49A040B04028F080919A088931D3
:10A170000CF4FFC021E0E21620E1F20620E0020725
:10A1800020E012070CF473C080918C03882309F43B
:10A190006AC0D801C70117FF07C088279927DC01CB
:10A1A0008E199F09A00BB10B9C01AD01B7FF04C034
:10A1B00021503E4F4F4F5F4FF9E0559547953795EA
:10A1C0002795FA95D1F780918A0390918B03820F9E
:10A1D000931F90938B0380938A03D801C70117FFC5
:10A1E00003C00796A11DB11DE3E0B595A79597950E
:10A1F0008795EA95D1F780937E0390937F03A09390
:10A200008003B093810389589341A040B04064F02B
:10A2100088E893E1A0E0B0E080937E0390937F0311
:10A22000A0938003B093810320917E0330917F033C
:10A23000409180035091810357FF04C021503F4F4C
:10A240004F4F5F4F232F342F452F552747FD5A95EA
:10A250008091C0029091C102820F931F9093C1021E
:10A260008093C00206C081E080938C0302C01092EC
:10A270008C0340E0E41640EFF4064FEF04074FEF85
:10A2800014070CF073C080918D03882309F46AC011
:10A29000D801C70117FF07C088279927DC018E194D
:10A2A0009F09A00BB10B9C01AD01B7FF04C0215069
:10A2B0003E4F4F4F5F4F69E055954795379527952E
:10A2C0006A95D1F780918A0390918B03820F931F37
:10A2D00090938B0380938A03D801C70117FF03C0B3
:10A2E0000796A11DB11D23E0B595A7959795879574
:10A2F0002A95D1F780937E0390937F03A0938003E8
:10A30000B093810388579C4EAF4FBF4F64F488E7EA
:10A310009CEEAFEFBFEF80937E0390937F03A093FB
:10A320008003B093810320917E0330917F0340919D
:10A3300080035091810357FF04C021503F4F4F4F7E
:10A340005F4F232F342F452F552747FD5A95809176
:10A35000C0029091C102820F931F9093C10280931B
:10A36000C00211C081E080938D030DC010928D0357
:10A370000AC010928B0310928A0384E690E09093B7
:10A380008D0180938C016889262F332780918A0361
:10A3900090918B032817390724F430938B03209373
:10A3A0008A0310919A08112379F0212F332727FD72
:10A3B000309580918A0390918B032817390724F4F4
:10A3C00030938B0320938A0340916F035091700365
:10A3D00060917103709172034138510561057105F7
:10A3E00074F0809147039091480320918A03309143
:10A3F0008B03820F931F9093480380934703405829
:10A400005F4F6F4F7F4F74F48091470390914803E3
:10A4100020918A0330918B03821B930B9093480306
:10A420008093470381E090E090938B0380938A03AD
:10A43000C0907303D0907403E0907503F09076039E
:10A44000D701C601F7FE07C088279927DC018C19C0
:10A450009D09AE09BF0981509240A040B04034F040
:10A4600084E090E090938B0380938A03809194031F
:10A4700090919503A0919603B09197032091E907DD
:10A480003091EA074091EB075091EC07821B930B48
:10A49000A40BB50B815E914BAF4FBF4F8F539C49BF
:10A4A000A040B04018F019310CF4FFC001E0C01614
:10A4B00000E1D00600E0E00600E0F0060CF473C016
:10A4C00080918E03882309F46AC0D701C601F7FE84
:10A4D00007C088279927DC018C199D09AE09BF099F
:10A4E0009C01AD01B7FF04C021503E4F4F4F5F4F5D
:10A4F00009E055954795379527950A95D1F78091AD
:10A500008A0390918B03820F931F90938B03809308
:10A510008A03D701C601F7FE03C00796A11DB11D2E
:10A5200013E0B595A795979587951A95D1F78093E0
:10A53000820390938303A0938403B0938503895887
:10A540009341A040B04064F088E893E1A0E0B0E01F
:10A550008093820390938303A0938403B093850335
:10A5600020918203309183034091840350918503AD
:10A5700057FF04C021503F4F4F4F5F4F232F342FC1
:10A58000452F552747FD5A958091C2029091C302ED
:10A59000820F931F9093C3028093C20206C081E092
:10A5A00080938E0302C010928E0320E0C21620EF2B
:10A5B000D2062FEFE2062FEFF2060CF073C0809167
:10A5C0008F03882309F46AC0D701C601F7FE07C0CC
:10A5D00088279927DC018C199D09AE09BF099C01C8
:10A5E000AD01B7FF04C021503E4F4F4F5F4FE9E030
:10A5F0005595479537952795EA95D1F780918A0328
:10A6000090918B03820F931F90938B0380938A0307
:10A61000D701C601F7FE03C00796A11DB11D73E067
:10A62000B595A795979587957A95D1F780938203ED
:10A6300090938303A0938403B093850388579C4E23
:10A64000AF4FBF4F64F488E79CEEAFEFBFEF80934E
:10A65000820390938303A0938403B0938503209196
:10A66000820330918303409184035091850357FF07
:10A6700004C021503F4F4F4F5F4F232F342F452FA2
:10A68000552747FD5A958091C2029091C302820FCF
:10A69000931F9093C3028093C20211C081E0809304
:10A6A0008F030DC010928F030AC010928B0310927B
:10A6B0008A0384E690E090938D0180938C01488911
:10A6C000242F332780918A0390918B032817390711
:10A6D00024F430938B0320938A0380919A08882373
:10A6E00079F0282F332727FD309580918A039091A8
:10A6F0008B032817390724F430938B0320938A03A4
:10A7000040917303509174036091750370917603C7
:10A71000413851056105710574F0809145039091B0
:10A72000460320918A0330918B03820F931F9093ED
:10A7300046038093450340585F4F6F4F7F4FCCF4E3
:10A74000809145039091460320918A0330918B03B9
:10A75000821B930B90934603809345030AC010928B
:10A76000C3021092C2021092C1021092C002109253
:10A77000EE028091EF07882341F41092C3021092F9
:10A78000C2021092C1021092C0028091E107909122
:10A79000E207A091E307B091E407809390039093C0
:10A7A0009103A0939203B09393038091E907909152
:10A7B000EA07A091EB07B091EC0780939403909384
:10A7C0009503A0939603B0939703109222031092DF
:10A7D0002303109224031092250310921E0310925B
:10A7E0001F03109220031092210310921A0310925B
:10A7F0001B0310921C0310921D031092E10710928C
:10A80000E2071092E3071092E4071092E907109212
:10A81000EA071092EB071092EC071092D8071092FB
:10A82000D9071092DA071092DB071092CA0710922C
:10A83000CB071092CC071092CD071092EC0110922A
:10A84000EB01E090E402F090E502C701F7FE04C0DE
:10A85000882799278E199F0904973CF08091090851
:10A8600084FD03C082E380937D0310913B06A12EFB
:10A87000BB24CC24DD24B701882777FD8095982F51
:10A880009701F7FE04C0222733272E193F094427DA
:10A8900037FD4095542F0E94137A9B01AC01C601ED
:10A8A000B5010E94137A97FF04C061507E4F8F4F0D
:10A8B0009F4F59E095958795779567955A95D1F76C
:10A8C0009B01812F99278E9DD0018F9DB00D9E9D5C
:10A8D000B00D1124CD01B7FD0396959587959595FB
:10A8E0008795280F391F8091C4029091C502280FC7
:10A8F000391F442737FD4095542F2093630330932D
:10A900006403409365035093660380910203909122
:10A910000303A0910403B0910503821B930BA40BC6
:10A92000B50B8093020390930303A0930403B093A9
:10A9300005038155934CA040B04064F080E593EC52
:10A94000A0E0B0E08093020390930303A09304037C
:10A95000B09305038091020390910303A091040337
:10A96000B0910503805B9C43AF4FBF4F64F480EB15
:10A970009CE3AFEFBFEF8093020390930303A09398
:10A980000403B0930503009190011091910117FD0C
:10A99000FAC08091090883FFF6C080918F01815031
:10A9A00080938F01882309F0F2C08DE080938F019E
:10A9B0008091320390913303A0913403B091350319
:10A9C000B7FF04C081509E4FAF4FBF4F39E0B595E0
:10A9D000A795979587953A95D1F77C0197FF04C085
:10A9E000F094E194F108F39480912A0390912B0361
:10A9F000A0912C03B0912D03B7FF04C081509E4F4E
:10AA0000AF4FBF4F29E0B595A795979587952A95A4
:10AA1000D1F79C0197FF03C0309521953F4FE21677
:10AA2000F3060CF47901B701F7FE02C06D5F7F4FAA
:10AA30002B0155944794559447940894411C511CFC
:10AA40006090190870901A0880901B0890901C085C
:10AA500020914301309144014091450150914601BC
:10AA6000C401B3010E94877A59016A013093C80773
:10AA70002093C707021B130BC801845E9D4F68E635
:10AA800071E00E94527A9C01245B304080918C01DD
:10AA900090918D01009731F0019790938D018093F3
:10AAA0008C011BC009E1E016F104BCF48091EC02BA
:10AAB0009091ED02820F931F9093ED028093EC0230
:10AAC00080917D03882349F0815080937D03882302
:10AAD00021F4B092F102A092F00280918C01909149
:10AAE0008D01892BF9F480918E019927289FA0016F
:10AAF000299F500D389F500D1124CA01B2010E94A8
:10AB0000527ACB01AA2797FDA095BA2F680E791E1D
:10AB10008A1E9B1E6092190870921A0880921B0868
:10AB200090921C0880917D03882369F58091F00242
:10AB30009091F1022091C7073091C807821B930BB7
:10AB4000845E9D4F68E671E00E94527A9C01245B0E
:10AB500030408091780186959927289FB001299FE0
:10AB6000700D389F700D11249B0177FF02C0215F8B
:10AB70003F4FF4E035952795FA95E1F73093C502FC
:10AB80002093C40204C01092C5021092C4028091A6
:10AB9000EE02882381F01092F6021092F7021092D2
:10ABA000F8021092F9021092FA021092FB0210922F
:10ABB000FC021092FD02F090BD02FF20F1F48091A2
:10ABC000EF07282F33274427552780913203909190
:10ABD0003303A0913403B0913503BC01CD010E9431
:10ABE000137ADC01CB01BC01CD0128EF3AE240E051
:10ABF00050E00E94877A390102C066247724E090F1
:10AC0000BC02EE20F1F48091EF07282F3327442770
:10AC1000552780912A0390912B03A0912C03B0918A
:10AC20002D03BC01CD010E94137ADC01CB01BC01D4
:10AC3000CD0128EF3AE240E050E00E94877A2901F6
:10AC400002C0442455248091C4079091C507893CD3
:10AC500091051CF088EC90E005C088539F4F34F4B8
:10AC600088E39FEF9093C5078093C4078091CF0737
:10AC70009091D007893C91051CF088EC90E005C0CC
:10AC800088539F4F34F488E39FEF9093D0078093CD
:10AC9000CF078091D1079091D207AA2797FDA09561
:10ACA000BA2F20911708A22EBB24CC24DD24BC018E
:10ACB000CD01A60195010E94137A9B01AC01809100
:10ACC000C4079091C507AA2797FDA095BA2FE7E082
:10ACD000880F991FAA1FBB1FEA95D1F7280F391FAC
:10ACE0004A1F5B1F57FF04C0215C3F4F4F4F5F4F10
:10ACF00076E055954795379527957A95D1F7830155
:10AD0000020F131F1093D2070093D1078091C2073F
:10AD10009091C307AA2797FDA095BA2FBC01CD013A
:10AD2000A60195010E94137A9B01AC018091CF0787
:10AD30009091D007AA2797FDA095BA2F67E0880FBA
:10AD4000991FAA1FBB1F6A95D1F7280F391F4A1FE9
:10AD50005B1F57FF04C0215C3F4F4F4F5F4F96E092
:10AD600055954795379527959A95D1F74201820ECB
:10AD7000931E9092C3078092C2078091120890910F
:10AD80001308880F991FAA2797FDA095BA2F209125
:10AD9000C907332744275527BC01CD010E94137AE8
:10ADA0005B016C0197FF08C02FE330E040E050E00A
:10ADB000A20EB31EC41ED51E86E0D594C794B794C8
:10ADC000A7948A95D1F78091DE07282F332744274F
:10ADD00055278091160390911703A0911803B09105
:10ADE0001903BC01CD010E94137ADC01CB01BC0127
:10ADF000CD0120EF35E540E050E00E94877AB501B3
:10AE0000620F731F70931308609312080150104172
:10AE100034F080E090E19093D2078093D107809145
:10AE2000D1079091D2078050904F34F480E090EF9A
:10AE30009093D2078093D10751E0851650E1950693
:10AE400034F080E090E19093C3078093C207809133
:10AE5000C2079091C3078050904F34F480E090EF88
:10AE60009093C3078093C2076150704134F080E033
:10AE700090E19093130880931208809112089091AA
:10AE800013088050904F34F480E090EF90931308B3
:10AE90008093120880910001482F552780911E0150
:10AEA00090911F014817590794F420911E01309189
:10AEB0001F0109811A81049FC001059F900D149FF5
:10AEC000900D1124B9010E943E7A7A836983298109
:10AED0003A81220F331F220F331F3A832983409177
:10AEE000090840FFC5C7EE2009F0C2C7FF2009F0DE
:10AEF000BFC7AA24BB2445018091BE029091BF0226
:10AF00009093A8058093A7052091490330914A03A7
:10AF10002115310509F03FC0809114019091150170
:10AF20008959934058F087B5853F20F48091EF010F
:10AF3000815011C081E08093A1034EC08091140123
:10AF4000909115018436910508F587B58B30D0F0C6
:10AF50008091EF018F5F8093EF019AE08902900169
:10AF600011248091CE05821B87BD8CE291E09093E5
:10AF7000DD018093DC018EE591E090934A0380939C
:10AF800049032AC081E08093A00326C0F092A00369
:10AF9000F092A10321C08091D2029091D302A0919E
:10AFA000D402B091D50214E0880F991FAA1FBB1FCD
:10AFB0001A95D1F78093F0019093F101A093F201DB
:10AFC000B093F301B092EE01A092ED012150304018
:10AFD00030934A032093490320917B0141FF24C011
:10AFE0002233D8F4809192018150809392018F3F57
:10AFF000D9F51092EF028091D2029091D302A091E4
:10B00000D402B091D5028093CE029093CF02A09348
:10B01000D002B093D10281E004C081E08093EF02BE
:10B0200088EC8093920120C0809147019091480163
:10B03000820F911D209134063327829FA001839FA8
:10B04000500D929F500D1124CA01AA2797FDA0957B
:10B05000BA2F8093CE029093CF02A093D002B093E8
:10B06000D10281E08093EF0280913203909133030B
:10B07000A0913403B0913503E0904301F090440176
:10B080000091450110914601BC01CD01A801970135
:10B090000E94877A59016A0180912A0390912B03BB
:10B0A000A0912C03B0912D03BC01CD01A801970103
:10B0B0000E94877AB901C5010E94C16F8C01CC97AB
:10B0C00014F00CE310E0C8010E94BB6B8C0180E21D
:10B0D000809342011092CD021092CC028091EF0237
:10B0E000882309F437C58091A20299279C01207119
:10B0F000307084FD2FC58091A10282608093A102EF
:10B100007091ED0770FD04C08091090881FD10C0A9
:10B11000C980DA8030939903209398033093CD024D
:10B120002093CC028091A202806C8093A20280C204
:10B130008091A20281FF52C240918201509183010D
:10B14000CA010F962091E2023091E3028217930721
:10B150008CF56091A003662369F58091A20287FFB8
:10B1600015C08091A2028F778093A2028091D202B3
:10B170009091D302A091D402B091D5028093CE02D7
:10B180009093CF02A093D002B093D1028091A202FB
:10B1900080648093A202C901841B950B0F9797FFCF
:10B1A00003C0909581959F4F9093CD028093CC02E0
:10B1B0008BE238C0CA010F9728173907C4F5609190
:10B1C000A1036623A1F58091A20286FF15C080919C
:10B1D000A2028F7B8093A2028091D2029091D3022F
:10B1E000A091D402B091D5028093CE029093CF0269
:10B1F000A093D002B093D1028091A2028068809384
:10B20000A202C901841B950B0F9697FF03C090956E
:10B2100081959F4F909581959F4F9093CD028093FC
:10B22000CC028DE2809342016093C602D9C08DE3C7
:10B23000809342016091C702662371F12091C80298
:10B240003091C9024091CA025091CB028091CE0246
:10B250009091CF02A091D002B091D10282179307B2
:10B26000A407B507CCF48091A20280648093A20267
:10B27000862F99279093CD028093CC028AE0809309
:10B28000C6028EE5809342018091A20287FFA8C08A
:10B290008091A2028F7733C0662309F443C02091C6
:10B2A000C8023091C9024091CA025091CB028091EC
:10B2B000CE029091CF02A091D002B091D102281776
:10B2C00039074A075B0774F58091A2028068809372
:10B2D000A202862F9927909581959F4F9093CD023A
:10B2E0008093CC0286EF8093C60286E7809342016A
:10B2F0008091A20286FF74C08091A2028F7B80930E
:10B30000A2028091D2029091D302A091D402B09176
:10B31000D5028093CE029093CF02A093D002B09337
:10B32000D1025EC08091A202807C09F459C0809154
:10B33000C602882379F5C090D202D090D302E09063
:10B34000D402F090D502D701C60180589040A040A9
:10B35000B0402091CE023091CF024091D002509166
:10B36000D10282179307A407B5075CF4D701C60181
:10B3700080589F4FAF4FBF4F281739074A075B07C9
:10B380005CF08093CE029093CF02A093D002B09352
:10B39000D10202C01092C6028091A2028F738093E4
:10B3A000A202109299031092980371FF06C084EFD5
:10B3B00091E09093DD018093DC018091D602882397
:10B3C00079F48091D2029091D302A091D402B091ED
:10B3D000D502C397A105B1051CF081E08093D60288
:10B3E00060919803709199038091CC029091CD0265
:10B3F000680F791F7093990360939803CB0177FFCF
:10B4000004C088279927861B970B855F91400CF411
:10B41000CEC04091C602442389F18091C802909128
:10B42000C9022091CE023091CF02821B930B099664
:10B43000439748F48091C8029091C902A091CA0232
:10B44000B091CB0212C0242F332727FD3095432F14
:10B45000532F8091CE029091CF02A091D002B09153
:10B46000D102820F931FA41FB51F8093CE02909329
:10B47000CF02A093D002B093D10224C080913406B1
:10B480002091CE023091CF024091D0025091D10252
:10B490001616170644F463E00E94327A280F311D15
:10B4A000411D511D07C063E00E94327A281B3109FB
:10B4B000410951092093CE023093CF024093D0022C
:10B4C0005093D1021092990310929803C090D20227
:10B4D000D090D302E090D402F090D502D701C601FB
:10B4E00080509440A040B0402091CE023091CF02D5
:10B4F0004091D0025091D10282179307A407B5075B
:10B500005CF4D701C60180509C4FAF4FBF4F281746
:10B5100039074A075B0744F08093CE029093CF022D
:10B52000A093D002B093D1028091ED0781FF06C0B5
:10B5300084E690E09093DD018093DC0180913806F1
:10B540008823A9F58091C702882389F54091BE021E
:10B550005091BF0257FF02C04D5F5F4F5595479511
:10B560005595479580911E0190911F0120910001F2
:10B570003327489FB001499F700D589F700D1124CB
:10B58000CB01B9010E94527A7093830160938201CA
:10B59000663471051CF486E490E005C067397105D6
:10B5A00034F086E990E0909383018093820180914A
:10B5B000490390914A03892BB9F18091D20290916D
:10B5C000D302A091D402B091D5028093CE02909381
:10B5D000CF02A093D002B093D10226C08091D202B4
:10B5E0009091D302A091D402B091D502805991409C
:10B5F000A040B0408093CE029093CF02A093D0029F
:10B60000B093D10280913806882311F0992702C0A7
:10B6100088E790E0909383018093820189819A81E9
:10B620009093BF028093BE02C090BE02D090BF0232
:10B630002091D2023091D3024091D4025091D50290
:10B640002E8B3F8B488F598F2091CE023091CF02A5
:10B650004091D0025091D1026E897F89888D998D59
:10B66000261737074807590724F08091ED0780FD1A
:10B67000BDC28091490390914A03892B39F0C09053
:10B68000BE02D090BF02AA24BB24D9C08E899F8954
:10B69000A88DB98D821B930BA40BB50B8093670308
:10B6A00090936803A0936903B0936A03823070E8B3
:10B6B00097077FEFA7077FEFB7072CF481E090E8AB
:10B6C000AFEFBFEF09C08F5F9F47A040B04064F06D
:10B6D0008FEF9FE7A0E0B0E080936703909368034B
:10B6E000A0936903B0936A03A0906703B0906803C6
:10B6F00080917A01282F33274427552780916703AB
:10B7000090916803A0916903B0916A03BC01CD01D7
:10B710000E94137A97FF04C0615E7F4F8F4F9F4F47
:10B72000A5E09595879577956795AA95D1F760934C
:10B730006703709368038093690390936A0365308D
:10B74000FEEF7F07FFEF8F07FFEF9F072CF484E0EA
:10B750009EEFAFEFBFEF09C0605074408040904053
:10B7600064F080E094E0A0E0B0E080936703909301
:10B770006803A0936903B0936A0380906703909075
:10B7800068032091ED013091EE0137FF02C0295F7F
:10B790003F4FF3E035952795FA95E1F74FEF2238C3
:10B7A00034071CF421E83FEF05C02038310514F0C0
:10B7B00020E830E0C901AA2797FDA095BA2F209173
:10B7C0007C01332744275527BC01CD010E94137A01
:10B7D00097FF04C06D5F7F4F8F4F9F4FE2E09595BD
:10B7E000879577956795EA95D1F79B015FEF613073
:10B7F00075071CF420E03FEF06C06F3F710519F09C
:10B8000014F020E031E08091A202807C49F0C9016F
:10B8100037FD03969C0135952795359527950DC0E5
:10B820008091ED0780FF09C0C90137FD07969C0193
:10B8300043E0359527954A95E1F7820E931E2091B6
:10B840007901222309F454C06091F2027091F3024D
:10B850008091F4029091F50297FF04C061587F4FE8
:10B860008F4F9F4F37E095958795779567953A95D8
:10B87000D1F73327442755270E94137A97FF04C036
:10B88000615E7F4F8F4F9F4FB5E095958795779578
:10B890006795BA95D1F760936703709368038093B7
:10B8A000690390936A036138AFEF7A07AFEF8A07B5
:10B8B000AFEF9A072CF480E89FEFAFEFBFEF0AC01D
:10B8C0006F3F71058105910569F064F080E091E0BA
:10B8D000A0E0B0E08093670390936803A0936903AE
:10B8E000B0936A038091670390916803880E991E54
:10B8F00080917701282F332780919D08992787FD14
:10B900009095289FF001299FF00D389FF00D11248C
:10B910009F01F7FF02C021583F4F220F232F221F04
:10B92000330BFFEF21383F071CF420E83FEF06C040
:10B930002F3F310519F014F020E031E0820E931E04
:10B94000C401AA2797FDA095BA2FE090BE02F090FF
:10B95000BF029701442737FD4095542FBC01CD010C
:10B960000E94137A97FF04C061507E4F8F4F9F4F04
:10B97000F9E09595879577956795FA95D1F7C61A69
:10B98000D70A8091CC029091CD02892B09F060C03A
:10B990001E141F040CF05CC09501B7FE03C0309567
:10B9A00021953F4F2D33310540F48091EA0290916B
:10B9B000EB028C159D0574F526C02C533040E5E054
:10B9C00036952795EA95E1F72031310510F02FE003
:10B9D00030E04091EA025091EB021A141B04E4F4A7
:10B9E00080E190E0821B930B489F9001499F300DAE
:10B9F000589F300D112474E0369527957A95E1F71C
:10BA00002C153D0520F58091800190918101C8168B
:10BA1000D906F4F06C011CC0205F3F4F809180017B
:10BA200090918101829FB001839F700D929F700D54
:10BA300011249B0164E0369527956A95E1F74C1532
:10BA40005D0514F06A0104C0C216D30608F069014E
:10BA5000C601AA2797FDA095BA2F2DE0880F991F40
:10BA6000AA1FBB1F2A95D1F79801442737FD40959F
:10BA7000542FBC01CD010E94877A20936B03309331
:10BA80006C0340936D0350936E03C0906B03D09092
:10BA90006C0380919A0390919B039C01220F331FAA
:10BAA000280F391F2C0D3D1D37FF02C02D5F3F4F62
:10BAB000A901559547955595479550939B034093FC
:10BAC0009A0380913006282F3327220F331F220F2D
:10BAD000331F241735076CF480911108282F332762
:10BAE000220F331F220F331F2055304042175307B8
:10BAF00024F030939B0320939A038091ED0780FFFD
:10BB000014C080919A0390919B03A981BA818A17EE
:10BB10009B0724F0B0939B03A0939A03E0919A03B0
:10BB2000F0919B03FA83E98361C029813A812E1940
:10BB30003F0937FF02C02D5F3F4F3595279535955B
:10BB40002795E0909A03F0909B03E20EF31EFA8291
:10BB5000E9824CC080913806882301F56091BE02CD
:10BB60007091BF0277FF02C06D5F7F4F759567953B
:10BB70007595679540911E0150911F0180910001BC
:10BB8000282F3327649FC001659F900D749F900DEF
:10BB90001124B9010E94527ACB0101C099279093D8
:10BBA0008301809382018091820190918301873487
:10BBB00091051CF486E490E005C08639910534F0C7
:10BBC00086E990E0909383018093820129813A81F4
:10BBD00030939B0320939A038091A202806C809300
:10BBE000A2028091A1028D7F8093A1028091A20286
:10BBF00099279C012270307081FF2BC180919C039A
:10BC000090919D03A0919E03B0919F030097A10581
:10BC1000B10521F08091D6028130B1F449815A8179
:10BC2000CA01AA2797FDA095BA2F2EE0880F991F69
:10BC3000AA1FBB1F2A95D1F780939C0390939D0365
:10BC4000A0939E03B0939F038091D602813019F494
:10BC500082E08093D60269817A81CB01AA2797FD81
:10BC6000A095BA2F9801442737FD4095542FBC0169
:10BC7000CD010E94137ADC01CB0180936B0390937A
:10BC80006C03A0936D03B0936E03B7FF04C08150A3
:10BC9000904EAF4FBF4F7C018D01FDE0159507958C
:10BCA000F794E794FA95D1F7E0926B03F0926C0366
:10BCB00000936D0310936E036091A3027091A40230
:10BCC0008FE0603A780750F580919C0390919D0336
:10BCD000A0919E03B0919F039C01AD01EAE05695AF
:10BCE000479537952795EA95D1F7821B930BA40BBF
:10BCF000B50BA8019701F4E0220F331F441F551F15
:10BD0000FA95D1F7820F931FA41FB51F80939C0350
:10BD100090939D03A0939E03B0939F0360547F4133
:10BD200018F580919C0390919D03A0919E03B09182
:10BD30009F039C01AD01ECE05695479537952795FB
:10BD4000EA95D1F7821B930BA40BB50BA8019701C1
:10BD500072E0220F331F441F551F7A95D1F7820FCF
:10BD6000931FA41FB51F38C08091ED019091EE0183
:10BD70008091ED019091EE0197FF03C09095819520
:10BD80009F4F8436910584F58091D2029091D30221
:10BD90002091CE023091CF02821B930B81509F4F96
:10BDA0008F5F914008F580919C0390919D03A09135
:10BDB0009E03B0919F039C01AD016EE0569547959F
:10BDC000379527956A95D1F7821B930BA40BB50B7A
:10BDD0008E0D9F1DA01FB11F80939C0390939D0308
:10BDE000A0939E03B0939F0380919C0390919D0329
:10BDF000A0919E03B0919F030EE0B695A7959795ED
:10BE000087950A95D1F79093BF028093BE02409127
:10BE10003606442399F055279C01BA010E94527AB4
:10BE2000C901861B970B9093EB028093EA02260FC1
:10BE3000371F30938101209380011FC01092EB02C5
:10BE40001092EA028FEF93E090938101809380013A
:10BE500014C01092D60210929C0310929D0310926F
:10BE60009E0310929F033093BF022093BE0205C031
:10BE70008091A202806C8093A2022091D607822F2B
:10BE80009927880F991F880F991F8896E981FA8151
:10BE90008E179F0714F09A838983F0911108FD8B08
:10BEA0008F2F9927880F991F880F991F80559040D1
:10BEB000E980FA808E159F0514F49A838983809116
:10BEC0002502882341F48091AF088F3F21F48091AF
:10BED000AF038823E1F08091A3029091A40202971E
:10BEE000C097A8F409811A811016110684F481E024
:10BEF00090E09093A4028093A302422F5527440F11
:10BF0000551F440F551F485D5F4F5A834983698110
:10BF10007A8170938C0560938B0580916303909177
:10BF20006403A0916503B0916603F2E0880F991F46
:10BF3000AA1FBB1FFA95D1F70091120810911308A0
:10BF4000081B190B613A71058CF0CB0177FD019646
:10BF500095958795801791070CF48C0190958195A4
:10BF60009F4F081719076CF48C010BC001351105A0
:10BF700014F000E510E07FEF003B170714F400EB2E
:10BF80001FEF8D89282F3327220F331F220F331FD6
:10BF9000C901A981BA818A1B9B0B801791070CF4F8
:10BFA0008C01E981FA81E21BF30B0E171F070CF4D9
:10BFB0008F018091D1079091D2076091E802709132
:10BFC000E902861B970B9093E0078093DF07D090E0
:10BFD000EF072091FA023091FB024091FC02509150
:10BFE000FD02DD2041F0661A770AC301AA2797FDFA
:10BFF000A095BA2F04C0AA2797FDA095BA2F280FA5
:10C00000391F4A1F5B1F2093FA023093FB024093B3
:10C01000FC025093FD028091FA029091FB02A091E4
:10C02000FC02B091FD0281509A4FA040B04064F0F4
:10C0300080E09AEFA0E0B0E08093FA029093FB02D8
:10C04000A093FC02B093FD028091FA029091FB0252
:10C05000A091FC02B091FD0280509640AF4FBF4FBF
:10C0600064F480E096E0AFEFBFEF8093FA02909324
:10C07000FB02A093FC02B093FD02C0904506209104
:10C08000DF073091E00748E04C1598F08C2D992798
:10C09000829FB001839F700D929F700D1124CB0180
:10C0A00077FD07967C0163E0F594E7946A95E1F7E4
:10C0B00012C08C2D86959927829FD001839FB00D49
:10C0C000929FB00D1124CD01B7FD03967C01F5942C
:10C0D000E794F594E794A0907D01B0907E019501DE
:10C0E000442737FD4095542F8091FA029091FB022E
:10C0F000A091FC02B091FD02BC01CD010E94877AA3
:10C10000E20EF31E90906901692D77278827992701
:10C11000980117FF04C022273327201B310B37FF5C
:10C1200002C02F5F3F4F35952795E981FA812E0F89
:10C130003F1F442737FD4095542F0E94137A97FFE5
:10C1400004C0615C7F4F8F4F9F4F26E09595879588
:10C15000779567952A95D1F79B016E157F050CF4AD
:10C160007B01309521953F4FE216F3060CF47901DF
:10C170008091C2079091C3076091E6027091E70237
:10C18000861B970B9093C1078093C0072091F602FE
:10C190003091F7024091F8025091F902DD2041F010
:10C1A000461A570AC201AA2797FDA095BA2F04C0C4
:10C1B000AA2797FDA095BA2F280F391F4A1F5B1F8A
:10C1C0002093F6023093F7024093F8025093F9025D
:10C1D0008091F6029091F702A091F802B091F902D5
:10C1E00081509A4FA040B04064F080E09AEFA0E008
:10C1F000B0E08093F6029093F702A093F802B09318
:10C20000F9028091F6029091F702A091F802B091A4
:10C21000F90280509640AF4FBF4F64F480E096E043
:10C22000AFEFBFEF8093F6029093F702A093F8026E
:10C23000B093F9022091C0073091C10748E04C1536
:10C2400098F08C2D9927829FB001839F700D929F4B
:10C25000700D1124CB0177FD07966C01B3E0D594E6
:10C26000C794BA95E1F712C0C6948C2D9927829F86
:10C27000D001839FB00D929FB00D1124CD01B7FD69
:10C2800003966C01D594C794D594C794950144271F
:10C2900037FD4095542F8091F6029091F702A091BE
:10C2A000F802B091F902BC01CD010E94877AC20E5A
:10C2B000D31E692D772788279927980117FF04C077
:10C2C00022273327201B310B37FF02C02F5F3F4F40
:10C2D00035952795E981FA812E0F3F1F442737FDB9
:10C2E0004095542F0E94137A97FF04C0615C7F4FE2
:10C2F0008F4F9F4FE6E09595879577956795EA95DF
:10C30000D1F79B016C157D050CF46B0130952195DF
:10C310003F4FC216D3060CF469018091D607282E30
:10C3200033245090860660EF862E66E0962E57EAFC
:10C33000A52E56E0B52E4BE0442E30EF632E37E0AD
:10C34000732ED5012C9112160CF029C1203429F43A
:10C35000E981FA81FB8FEA8F1FC049815A81CA01A6
:10C36000AA2797FDA095BA2F332727FD3095432F95
:10C37000532FBC01CD010E94137A97FF04C0615C6A
:10C380007F4F8F4F9F4F26E09595879577956795BF
:10C390002A95D1F77B8F6A8FF5012181203439F4FA
:10C3A0002A8D3B8D2E0D3F1D3B8F2A8F2AC0203CAE
:10C3B00039F44A8D5B8D4E195F095B8F4A8F21C01E
:10C3C000C701AA2797FDA095BA2F332727FD3095DF
:10C3D000432F532FBC01CD010E94137A97FF04C055
:10C3E000615C7F4F8F4F9F4FB6E09595879577950E
:10C3F0006795BA95D1F7AA8DBB8DA60FB71FBB8FD6
:10C40000AA8FF5012281203439F42A8D3B8D2C0D21
:10C410003D1D3B8F2A8F2AC0203C39F44A8D5B8D0D
:10C420004C195D095B8F4A8F21C0C601AA2797FD71
:10C43000A095BA2F332727FD3095432F532FBC01EA
:10C44000CD010E94137A97FF04C0615C7F4F8F4F2C
:10C450009F4FA6E09595879577956795AA95D1F713
:10C46000AA8DBB8DA60FB71FBB8FAA8FF5012381A5
:10C47000203439F42A8D3B8D200F311F3B8F2A8FBA
:10C480002AC0203C39F44A8D5B8D401B510B5B8FD9
:10C490004A8F21C0C801AA2797FDA095BA2F33273C
:10C4A00027FD3095432F532FBC01CD010E94137AF5
:10C4B00097FF04C0615C7F4F8F4F9F4FF6E09595CB
:10C4C000879577956795FA95D1F7AA8DBB8DA60FBD
:10C4D000B71FBB8FAA8FF301808191812A8D3B8D7D
:10C4E0008217930764F4B901680F791F77FF02C0C0
:10C4F0006F5F7F4F759567957B8F6A8F1DC0552045
:10C5000049F44A8D5B8D440F551F481B590B5B8FB7
:10C510004A8F12C051E0551578F4252D33276A8DC6
:10C520007B8D861B970BB9010E94527AAA8DBB8D19
:10C53000A60FB71FBB8FAA8FC101880F991F880F45
:10C54000991FEA8DFB8D8E179F0764F4FD898F2F4D
:10C550009927880F991F880F991F2A8D3B8D2817BF
:10C56000390714F09B8F8A8F8A8D9B8D97FD0396D8
:10C570009595879595958795F4018183880F991FE7
:10C58000880F991F2A8D3B8D281B390BC901880FF5
:10C590008283EA8DFB8DD301ED93FC9303C0F401FC
:10C5A000118212824A9422E030E0620E731E44E04F
:10C5B00050E0A40EB51E68E070E0860E971E47FEA0
:10C5C000C0CEE2E1C55E0C94BE7A84B1806A84B9C3
:10C5D0003D9A82E58CBD1DBC459A81E0809323087D
:10C5E0008AEA8093340883E8809335088AE0809350
:10C5F0003608109238081092370810923A081092B4
:10C60000390810929C081092580808953091230818
:10C61000332309F085C00DB407FE82C084E0809307
:10C62000DB01459A2EB58091B2039927813091059F
:10C6300089F0823091051CF4892B21F03EC00297CD
:10C64000B9F03BC0309357082093B3032138A9F5C4
:10C6500081E008C0253549F48091B303820F8093AF
:10C66000B30382E08093B20328C03093B20325C0A5
:10C6700080915708E82FFF27E758F74F20838F5FF7
:10C68000809357089091B3038032A0F0291769F482
:10C6900080E2A9E7B8E0E9E5F8E00D9001928A951B
:10C6A000E1F781E08093580802C030935808109257
:10C6B000B20303C0920F9093B30320913308223248
:10C6C00008F028C0459800000000000000000000AD
:10C6D000000000000000000000000000000000005A
:10C6E000000000000000000000000000000000004A
:10C6F000000000000000E0912C08F0912D08E20FEE
:10C70000F11D80818EBD809155089081890F8093A5
:10C71000550803C081E0809323082F5F20933308DE
:10C720000895EF92FF920F931F9380913E069927F1
:10C73000880F991F880F991F7C010027F7FC00952F
:10C74000102F8091320390913303A0913403B09164
:10C750003503BC01CD01A80197010E94877A30936F
:10C7600038082093370880912A0390912B03A091D9
:10C770002C03B0912D03BC01CD01A80197010E94AB
:10C78000877A30933A08209339082091190830911C
:10C790001A0840911B0850911C08DA01C90163E096
:10C7A000880F991FAA1FBB1F6A95D1F7820F931F8D
:10C7B000A41FB51F820F931FA41FB51F2091430113
:10C7C000309144014091450150914601BC01CD0199
:10C7D0000E94877A3093400820933F08809143035A
:10C7E000909144032091FB013091FC01821B930B3B
:10C7F0009093460880934508E0913903F0913A03FD
:10C800008091E6079091E707BF010E94527A9B0151
:10C81000220F331F220F331F260F371F260F371FFC
:10C8200037FF02C02D5F3F4F3595279535952795EA
:10C8300030933C0820933B0880911508909116088E
:10C84000BF010E94527A9B01220F331F220F331F18
:10C85000260F371F260F371F37FF02C02D5F3F4FB0
:10C86000359527953595279530933E0820933D08BB
:10C8700010923A03109239031092E7071092E607DC
:10C8800010921608109215088091360899278D305D
:10C89000910509F48EC08E3091055CF48B309105C2
:10C8A00009F4B6C08C3091050CF037C10A9761F0DD
:10C8B000E6C18F30910509F4B2C18F3091050CF4B7
:10C8C00082C14097A9F1DBC18091B70280934908EA
:10C8D0008091B60280934A088091B50280934B08FC
:10C8E0008091B40280934C088091B30280934D08EC
:10C8F0008091B20280934E088091B10280934F08DC
:10C900008091B002809350088091A20280935108D8
:10C910008091A202837F8093A2020E94322C809396
:10C92000520880918706809353088091A102A5C187
:10C930008091A9089091AA0890934A088093490889
:10C940008091AD089091AE0890934C0880934B086D
:10C9500080911E0190911F0180934D0880910001EC
:10C9600080934E088091420180934F08809109087E
:10C97000809350088091ED07809351089091B40303
:10C9800090935208E92FFF27A3E0EE0FFF1FAA950F
:10C99000E1F7E051F94F87818093530885818093B7
:10C9A0005408892F8F5F6CE00E94327A9093B40311
:10C9B00066C18091720680934908809173068093C6
:10C9C0004A088091740680934B0880917506809385
:10C9D0004C088091760680934D0880917A0680936A
:10C9E0004E0880917B0680934F0880917C0680934F
:10C9F000500880917F068093510880917D06809336
:10CA0000520880917E06809353088091800635C13C
:10CA1000F89480912506E82FFF27EE0FFF1FEF5AAD
:10CA2000F84F0190F081E02DE038F1051CF0EFE7C0
:10CA3000F0E006C02FEFE138F20714F4E1E8FFEF71
:10CA4000E093490880912606E82FFF27EE0FFF1F8D
:10CA5000EF5AF84F0190F081E02DE038F1051CF01D
:10CA6000EFE7F0E006C06FEFE138F60714F4E1E815
:10CA7000FFEFE0934A0880912406E82FFF27EE0F8E
:10CA8000FF1FEF5AF84F0190F081E02DE038F105DB
:10CA90001CF0EFE7F0E006C08FEFE138F80714F480
:10CAA000E1E8FFEFE0934B0880912306E82FFF2792
:10CAB000EE0FFF1FEF5AF84F0190F081E02DE038A4
:10CAC000F1051CF0EFE7F0E006C02FEFE138F207C8
:10CAD00014F4E1E8FFEF7894E0934C088091D902D8
:10CAE00080934D088091DA0280934E088091DB029A
:10CAF00080934F088091DC02809350088091DD0282
:10CB0000809351088091DE02809352088091DF0269
:10CB1000809353088091E002B0C080911604863063
:10CB200018F01092160485E08093490880918106E0
:10CB300080934A088091D2029091D302A091D402AE
:10CB4000B091D502BC01CD0125E030E040E050E0DD
:10CB50000E94877A30934C0820934B088091CE0234
:10CB60009091CF02A091D002B091D102BC01CD0131
:10CB700025E030E040E050E00E94877A30934E0894
:10CB800020934D088091770680934F088091780616
:10CB90008093500880917906809351088091D80243
:10CBA00080935208809151079091520780935308C7
:10CBB00080918B0590918C0597FD039695958795AF
:10CBC000959587955AC01092490886E580934A0842
:10CBD00010924B088AE180934C0880910201809367
:10CBE0004D088091FB0380934E088091FC03809355
:10CBF0004F081092FB0380718093FC038091FD032A
:10CC0000809350088091FE03809351088091FF0328
:10CC100080935208809183068093530830C080919E
:10CC200057068093490880918B0680934A0880912B
:10CC30006F0180934B088091500680934C0880913F
:10CC4000510680934D088091520680934E08809142
:10CC50006E0180934F088091540680935008809114
:10CC60005506809351088091560680935208809112
:10CC7000AF08809353088091B50580935408809144
:10CC80005808882309F42DC18AEF80939D0181E023
:10CC900080938F0140915A0850915B08CA018150DE
:10CCA0009E4F8F5F9340B0F420915C0830915D08F7
:10CCB000C90181509E4F8F5F934060F480912F0691
:10CCC00085FF08C05093A6034093A5033093A403A7
:10CCD0002093A303809160089091610821E0893638
:10CCE000920724F4909391018093900120916A0817
:10CCF00030916B088091DC019091DD0182179307E0
:10CD000020F43093DD012093DC01809159089927AC
:10CD10008836910509F464C08936910524F4873674
:10CD2000910531F0E6C08936910509F48AC0E1C069
:10CD300080916C088093990880916D0880939B087E
:10CD400080916E0880939A0880916F0880938E017D
:10CD50008091700880939D088091710880939E0156
:10CD6000809172088093B103809173088093A2032D
:10CD70008091AF028823F9F02091740830917508F2
:10CD800037FD19C03093F1022093F00290915906BB
:10CD9000992389F08FE0989FC0011124281B390B3B
:10CDA000C90188599E4F68E671E00E94527A9093BB
:10CDB000F1028093F0022091AD033091AE03809197
:10CDC000760890917708280F391F37FF02C02F5F30
:10CDD0003F4F359527953093AE032093AD0389C01F
:10CDE00080916C0880932E0880916D0880932F08A5
:10CDF00080916E088093300880916F08809331088D
:10CE0000809170088093320880917B059091710821
:10CE1000892B80937B0590917C059370809172089B
:10CE20008C70982B90937C05809173088093AF034E
:10CE300080917408809393018091750880939C0879
:10CE400058C080916C088093240880916D0880936D
:10CE5000250880916E088093260880916F08809342
:10CE60002708809170089091710890932908809309
:10CE70002808809172089091730890932B088093F2
:10CE80002A0880917408992787FD909590938407CC
:10CE900080938307809175088093C70280917608FC
:10CEA000909177089C01442737FD4095542FDA0173
:10CEB000C90163E0880F991FAA1FBB1F6A95D1F7AC
:10CEC000820F931FA41FB51F820F931FA41FB51FAE
:10CED0008093C8029093C902A093CA02B093CB0278
:10CEE00008C01092A6031092A5031092A4031092FA
:10CEF000A3031F910F91FF90EF9008958091230855
:10CF0000882309F43BC0459884E398E090932D086A
:10CF100080932C089091B003E92FFF27EC56FE4F29
:10CF20009F5F9093B003808180933608993010F012
:10CF30001092B003109223080E94916381E08093C5
:10CF400033080000000000000000000000000000A6
:10CF500000000000000000000000000000000000D1
:10CF600000000000000000000000000000000000C1
:10CF7000000080913408809355088EBD089587B1D4
:10CF80008C6087B9429843981092B60380E88093EA
:10CF9000A0011092B50380939F0108958091BB0377
:10CFA00081508093BB038F3F09F0FAC089E08093E2
:10CFB000BB038091A202992780739070892B21F482
:10CFC0008091FC0380FF1DC080917006882351F082
:10CFD0008091BE03882319F484E08093B60381E036
:10CFE0008093BE03809171068823B9F08091BF03BE
:10CFF000882319F484E08093B50381E08093BF0314
:10D000000CC01092BE031092BF0380916C068093F7
:10D01000BC0380916E068093BD038091BE0388237C
:10D0200009F040C080918A06282F332724FF07C0CB
:10D030008091D702882319F425FD4DC04EC09091F0
:10D040006D06983F50F08091E8078D3D30F080915B
:10D05000BC0388230CF43FC040C0983F48F0809147
:10D06000E807853029F48091BC038823B4F133C0EC
:10D070008091B60381508093B6038F3F79F58091FC
:10D08000E80786958093B6038091A001813011F462
:10D0900080E801C086958093A0018091A0019091C5
:10D0A000BC0317C08091B60381508093B6038F3FB5
:10D0B000A9F489E08093B6038091A001813011F436
:10D0C00080E801C086958093A0018091A001909195
:10D0D0007006892311F0429A01C042988091BF03E3
:10D0E000882309F041C090918A0697FF07C080917C
:10D0F000D702882319F496FD50C034C090916F0672
:10D10000983F50F0809110088D3D30F08091BD0324
:10D1100088230CF442C026C0983F48F08091100844
:10D12000853029F48091BD038823E4F036C08091D6
:10D13000B50381508093B5038F3F91F5809110081E
:10D1400086958093B50380919F01813011F480E82A
:10D1500001C0869580939F0180919F019091BD03AE
:10D160008923D9F4439808958091B5038150809321
:10D17000B5038F3FA9F489E08093B50380919F01A7
:10D18000813011F480E801C0869580939F018091E1
:10D190009F0190917106892311F0439A0895439855
:10D1A00008954FB724E130E0F8948091C9008F775B
:10D1B0008093C9008091C9008F7B8093C9008091C2
:10D1C000C9008F7D8093C9005A9A52985B9A539AEE
:10D1D000832F99278093CD002093CC008091C800A5
:10D1E00082608093C80080E18093C9008091CA006A
:10D1F0008F778093CA008091CA008F7B8093CA008A
:10D200008091CA008F7D8093CA008091CA008F7E72
:10D210008093CA008091CA00877F8093CA00809162
:10D22000C9008B7F8093C9008091CA00846080937D
:10D23000CA008091CA0082608093CA008091C800B1
:10D2400087FF03C08091CE00F9CF8091C90080682C
:10D250008093C9004FBF0895A0E0B0E0E2E3F9E693
:10D260000C94AC7A482F00E010E08091A10181304D
:10D2700061F41092A10184E48093C2031092C4036C
:10D280001092C3031092C50325C28091C203882364
:10D2900019F421E030E001C098019091C303992373
:10D2A00071F4232B11F081E010C084E48093C20359
:10D2B0009093C4039093C3039093C503F4C191303A
:10D2C00069F4232B09F0E5C182E08093C3038091C8
:10D2D000C4038F5F8093C40383E0E3C19230D1F431
:10D2E000232B09F0D6C183E08093C2034093C5038A
:10D2F0009091C403923039F41092C60347FF03C0E3
:10D3000081E08093C60383E08093C3039F5F909383
:10D31000C403C9C1933009F0BCC1232B09F0B9C1C2
:10D320009093C20382E08093C3038091C4038F5F14
:10D330008093C4032091C503822F9927782F6627F5
:10D34000842F9927682B792B80914906813051F4DD
:10D350007370CB018050924063E070E00E94527A7B
:10D36000EB0119C0823069F47770CB018050944092
:10D3700066E070E00E94527AEB012695269526958C
:10D380000CC0EB01D370C856D140CE01D7FD019639
:10D39000EC01D595C79526952695022F11270F707C
:10D3A00010700F5F1F4F0D30110508F06BC1023078
:10D3B000110519F404E010E005C00430110511F462
:10D3C00002E010E06801C00ED11EF601EF5AF84FDE
:10D3D000808191819E01281B390BC90137FF03C051
:10D3E000909581959F4F069794F48091D802883C40
:10D3F00030F48091D802865F8093D80208C088EC10
:10D400008093D80280916F008F7D80936F00F6012A
:10D41000EF5AF84F808191819C01220F331F280F12
:10D42000391F2C0F3D1F37FF02C02D5F3F4F790181
:10D43000F594E794F594E794CE0101968E159F0537
:10D4400024F40894E108F10808C0CE010197E81619
:10D45000F9061CF40894E11CF11C0630110509F0D2
:10D46000D1C0C536D1050CF4A8C09091C103E92FF5
:10D47000FF27E256F74FE081ED3729F48091C00392
:10D4800080958093C003963061F48091C003882317
:10D4900011F0E338B9F0882309F08BC0ED3791F033
:10D4A00088C0993009F085C08091C003882329F491
:10D4B0008091A708833831F07CC08091A7088D3710
:10D4C00009F077C080919F088D3739F48091A008CA
:10D4D0008338B1F483E89FEF0FC0833889F48091DB
:10D4E000A008833829F410925C0710925B0708C0EB
:10D4F0008D3731F48DE790E090935C0780935B0764
:10D500008091A108992787FD909590935E0780935D
:10D510005D078091A208992787FD909590936807F1
:10D52000809367078091A308992787FD9095909332
:10D530006A07809369078091C1038930D1F5809192
:10D54000A5088D3749F4809161079091620705968F
:10D5500090936207809361078091A6088D3749F404
:10D56000809161079091620705979093620780937D
:10D570006107809161079091620783589F4F1CF467
:10D5800083E89FEF09C080916107909162078E3711
:10D59000910534F08DE790E09093620780936107E6
:10D5A0008091A408992787FD9095909366078093B2
:10D5B00065071092C1031092C003CA30D1055CF414
:10D5C0008091C1038F5F8093C103E82FFF27E2564C
:10D5D000F74F83E880838091C1038A3011F4109261
:10D5E000C1038FEFCC39D8076CF48091C103E82FC9
:10D5F000FF27E256F74F8DE780838091C003809527
:10D600008093C0038091D802843BD0F0F601EF5A9A
:10D61000F84F80819181F701E81BF90BCF0163E09E
:10D6200070E00E94527ACB01880F991F860F971FD6
:10D6300025E837E0C20ED31EF6019183808307C030
:10D6400025E837E0C20ED31EF601118210820530A4
:10D65000110540F4000F111F0F5A184FF801F18205
:10D66000E08221C00530110529F4D0936007C093F2
:10D670005F0719C007301105B1F4D0936407C09358
:10D68000630711C00231110570F081E08093A101A0
:10D690000AC081E08093A1011092C4031092C603D6
:10D6A00084E48093C2038091C403803198F0809118
:10D6B000C603882331F48091A101882311F480935B
:10D6C00041011092C4031092C6031092C30384E474
:10D6D0008093C203E8E0CDB7DEB70C94C87ACF934D
:10D6E000FC0197FF05C0CFEFF095E195FF4F01C01A
:10D6F000C1E028E631E0CF01B9010E94527AFC0175
:10D700008B35910554F08B5590408A35910538F44E
:10D7100084EB90E08E1B9F0BFC0141E00DC0CF011C
:10D72000855B90408A35910518F4E45BF04003C0B6
:10D730002E1B3F0BF9014FEFEE0FFF1FE25DF64F7F
:10D74000259134918C2F992787FD9095289FB001C2
:10D75000299F700D389F700D1124842F992787FD04
:10D760009095689FA001699F500D789F500D1124DE
:10D77000CA01CF9108952AE530E0281B390BC90171
:10D780000E946F6B0895CF93DF9380E00E94A77192
:10D7900080911E0190911F016AE070E00E94527A10
:10D7A0009F938F9380911E0190911F016AE070E01A
:10D7B0000E94527A7F936F938CEF99E09F938F939F
:10D7C000CAE9D1E7DF93CF93E091E203F091E3035D
:10D7D00009952DB73EB7285F3F4F2DBF80919D0122
:10D7E000882361F186E00E94A771809193019927B7
:10D7F0009F938F9380912808909129086AE070E0A8
:10D800000E943E7A7F936F938FED90E09F938F936A
:10D810008091C7079091C8079F938F9385E09AE006
:10D820009F938F93DF93CF93E091E203F091E30313
:10D8300009958DB79EB70C968DBF12C086E00E94E9
:10D84000A77183E19AE09F938F93DF93CF93E09149
:10D85000E203F091E30309950F900F900F900F9062
:10D860008091AF038823F9F086E00E94A771809130
:10D87000AF0399279F938F938AE19AE09F938F93A9
:10D88000DF93CF93E091E203F091E30309952DB785
:10D890003EB72A5F3F4F2DBF8091D702882319F0F2
:10D8A0008FE48093A80180E10E94A7718091AA0172
:10D8B0009091AB016CE370E00E943E7A9F938F934E
:10D8C0008091AA019091AB016CE370E00E943E7AD6
:10D8D0007F936F938091AD089091AE089F938F9343
:10D8E00086E29AE09F938F93CAE9D1E7DF93CF93C3
:10D8F000E091E203F091E3030995809109082DB7C7
:10D900003EB7265F3F4F2DBF80FF29C08AE10E94AE
:10D91000A7718091420199279F938F938091D202A2
:10D920009091D302A091D402B091D502BC01CD0157
:10D9300024E630E040E050E00E94877A3F932F9346
:10D9400083E39AE09F938F93DF93CF93E091E20379
:10D95000F091E30309958DB79EB708968DBFDF91CF
:10D96000CF910895CF93DF9380E00E94A7718091BB
:10D970000F07992787FD90959F938F9380910707B5
:10D98000992787FD90959F938F938091FF06992704
:10D9900087FD90959F938F938091F706992787FD38
:10D9A00090959F938F938AE39AE09F938F93CAE910
:10D9B000D1E7DF93CF93E091E203F091E303099580
:10D9C00080E10E94A7712DB73EB7245F3F4F2DBF66
:10D9D00080912F07992787FD90959F938F93809132
:10D9E0002707992787FD90959F938F9380911F0715
:10D9F000992787FD90959F938F938091170799277B
:10DA000087FD90959F938F938AE49AE09F938F93DD
:10DA1000DF93CF93E091E203F091E30309958091C6
:10DA200021062DB73EB7245F3F4F2DBF853098F4B8
:10DA300080E10E94A7718AE59AE09F938F93DF931C
:10DA4000CF93E091E203F091E30309950F900F90DB
:10DA50000F900F9018C08730B0F488E10E94A77132
:10DA60008FED90E09F938F938BE69AE09F938F9337
:10DA7000DF93CF93E091E203F091E30309958DB733
:10DA80009EB706968DBFDF91CF9108950F931F9398
:10DA900080E00E94A7712AE030E08091A90890916F
:10DAA000AA08B9010E943E7A9F938F938091A9089A
:10DAB0009091AA08B9010E943E7A7F936F9380915A
:10DAC0001E0190911F01B9010E94527A9F938F937A
:10DAD00080911E0190911F01B9010E94527A7F939B
:10DAE0006F9384E79AE09F938F930AE911E71F935E
:10DAF0000F93E091E203F091E303099580E10E9426
:10DB0000A7718DB79EB70C968DBF8091AD0890918F
:10DB1000AE089F938F938091AB089091AC089F9330
:10DB20008F9387E89AE09F938F931F930F93E091D1
:10DB3000E203F091E30309958DB79EB708968DBF78
:10DB40001F910F9108950F931F93CF93DF938091AF
:10DB50009D01CAE9D1E7882309F47DC080E00E94D5
:10DB6000A7718091250899279F938F93809127080B
:10DB700099279F938F9383E99AE09F938F938E01C8
:10DB8000DF93CF93E091E203F091E30309958DB722
:10DB90009EB708968DBF80912608833031F48CE0C3
:10DBA0000E94A77182EA9AE005C08CE00E94A771EA
:10DBB00087EA9AE09F938F93DF93CF93E091E203FC
:10DBC000F091E30309950F900F900F900F908091C3
:10DBD000240881FF12C08CE00E94A7718CEA9AE0B1
:10DBE0009F938F931F930F93E091E203F091E303D0
:10DBF00009950F900F900F900F9080E10E94A771F0
:10DC00008091930199279F938F938FED90E09F933D
:10DC10008F9380912A0890912B089F938F938091E6
:10DC20002808909129086AE070E00E943E7A7F936C
:10DC30006F9381EB9AE09F938F938AE991E79F938B
:10DC40008F93E091E203F091E30309958DB79EB7BE
:10DC50000C968DBF12C082E00E94A77184EC9AE0FE
:10DC60009F938F93DF93CF93E091E203F091E303CF
:10DC700009950F900F900F900F90DF91CF911F910A
:10DC80000F910895CF93C82F2091C7032093C80305
:10DC900099278F32910509F1803391051CF44F9734
:10DCA000A1F02CC08F34910501F18F38910531F529
:10DCB000222319F481E090E038C086E0289FF0012B
:10DCC0001124EC51F64F849117C086E0289FF00193
:10DCD0001124EB51F64F84910FC086E0289FF0018C
:10DCE0001124EA51F64F849107C086E0289FF00185
:10DCF0001124E951F64F84918093C7039091C70393
:10DD00008091C8039813C0E00E94AD719091C70341
:10DD100086E0989FF0011124E851F64F2591349147
:10DD20008C2FF901099580E090E0CF910895109231
:10DD3000AA081092A9081092AE081092AD0810928D
:10DD4000AC081092AB081092AF088AE090E00E94F5
:10DD50008F169093CA038093C9030895CF93DF93DE
:10DD60008091C9039091CA030E949816882309F4F0
:10DD7000AFC08091C9039091CA030A969093CA03D9
:10DD80008093C903E0E0F0E09F0190E05FEFA0EF37
:10DD9000B6E04BE0ED018B8187FF0BC09F5F8D816B
:10DDA000E80FF11D8981280F311D8E81851708F438
:10DDB000582F4150189647FFEDCF5093AF08232BB3
:10DDC00041F52091CF033091D0034091D103509180
:10DDD000D203BB27A52F942F832F9093CE0380933C
:10DDE000CD03AA27BB27281B390B4A0B5B0BCF019E
:10DDF000AA27BB27280F391F4A1F5B1F2093CF0379
:10DE00003093D0034093D1035093D203E5E0F0E088
:10DE100013C02091CD033091CE032E173F0718F485
:10DE2000E21BF30B02C0E0E0F0E0892F9927880F96
:10DE3000991FE80FF91F3596F093AA08E093A908F7
:10DE4000EF3FF10578F480911E0190911F018E9FA4
:10DE500090018F9F300D9E9F300D1124C90164E603
:10DE600070E013C0CF019695879596958795209180
:10DE70001E0130911F01289FA001299F500D389F3E
:10DE8000500D1124CA0169E170E00E943E7A70933E
:10DE9000AC086093AB082091CB033091CC032E0FDC
:10DEA0003F1F3093CC032093CB035EE02131350735
:10DEB00078F08091AD089091AE0801969093AE08ED
:10DEC0008093AD0820513E403093CC032093CB0388
:10DED000DF91CF910895002422273327442751E072
:10DEE000BB27EE27FF27A0E1660F771F881F991F2A
:10DEF000001C221F331F441F660F771F881F991FA6
:10DF0000001C221F331F441F2AF4050E2B1F3E1F27
:10DF10004F1F04C0051A2B0B3E0B4F0B550FBB1F99
:10DF2000EE1F587F556047FD5250AA95E9F6E695D9
:10DF3000B7955795E695B7955795852F9B2F0895DB
:10DF40002227332741E0552768E0880F991F221FB9
:10DF5000331F880F991F221F331F1AF4240F351FF8
:10DF600002C0241B350B440F551F487F456037FD09
:10DF700042506A9551F75695479556954795842F87
:10DF80000895AA2797FF04C0809590958A1F9A1F2D
:10DF900077FF04C0609570956A1F7A1F669F900195
:10DFA000779FA001679F300D411D5A1F300D411D05
:10DFB0005A1F889FF001999F2E0F3F1F401D511D32
:10DFC000899F300D411D5A1F300D411D5A1FCA0136
:10DFD000B901112480CF4FB720E430E0F89480914C
:10DFE000C9008F778093C9008091C9008F7B80938F
:10DFF000C9008091C9008F7D8093C9005A9A5298B8
:10E000005B9A539A832F99278093CD002093CC005D
:10E010008091C80082608093C80088E18093C90025
:10E020008091CA008F778093CA008091CA008F7B4D
:10E030008093CA008091CA008F7D8093CA0080912E
:10E04000CA008F7E8093CA008091CA00877F809328
:10E05000CA008091C9008B7F8093C9008091CA005B
:10E0600084608093CA008091CA0082608093CA0055
:10E070008091C80087FF03C08091CE00F9CF8091C6
:10E08000C90080688093C9004FBF08950F931F9304
:10E09000CF93DF93482F4F5F893108F08BC0809179
:10E0A0005007841720F44F5F409350074150CB0135
:10E0B00083539B4268E170E00E94527AA42FBB27F1
:10E0C000FD01EA0FFB1FEF5AF84F808191819B0100
:10E0D000281B390BC90137FF03C0909581959F4FCD
:10E0E000069794F48091D802883C30F48091D8024D
:10E0F000865F8093D80208C088EC8093D802809114
:10E100006F008F7D80936F00FD01EA0FFB1FEF5AB8
:10E11000F84F808191819C01220F331F280F391FF6
:10E12000260F371F37FF02C02D5F3F4FE901D595FE
:10E13000C795D595C795CB0101968C179D0714F40B
:10E14000219706C061507040C617D7070CF421967E
:10E150008091D802843BD8F08D010A0F1B1FF80173
:10E16000EF5AF84F80819181FE01E81BF90BCF0136
:10E1700063E070E00E94527ACB01880F991F860FEE
:10E18000971F0B57184FF8019183808307C0AA0F80
:10E19000BB1FAB57B84F11961C921E92E42FFF275E
:10E1A000EE0FFF1FEF5AF84FD183C083443011F4B4
:10E1B00010924101DF91CF911F910F910895CF935C
:10E1C000DF932091B008822F9927807F907040972D
:10E1D00009F06CC02F3109F046C08091B1088093DE
:10E1E000D7032091B3082093D9038091B40880937A
:10E1F000D803822F992790935207809351072223A7
:10E2000009F054C080912306282F3327220F331F93
:10E21000F901EB57F84F1182108280912406A82F44
:10E22000BB27AA0FBB1FFD01EB57F84F11821082CD
:10E2300080912606E82FFF27EE0FFF1FCF018B5797
:10E24000984FEC01198218822F5A384FE901198230
:10E250001882AF5AB84F11961C921E92EF5AF84F7F
:10E260001182108223C0C22FCF70CA30F8F480917F
:10E27000B1088093DA088091B2088093D908809120
:10E28000B3088093DC088091B4088093DB08609128
:10E29000D9087091DA088C2F0E9446706091DB08D3
:10E2A0007091DC088C2F8F5F0E944670DF91CF91B8
:10E2B0000895CF93C82F8F3F49F48091DA038F3FA1
:10E2C00029F41092DC031092DB0332C02091DC03AE
:10E2D000222339F4CF3111F485E001C084E080932A
:10E2E000DD038091DD039091DB038217A0F4892F79
:10E2F00080958093DB038F3F19F48EEF8093DB03CF
:10E300008091DB03C81711F40E94DF701092DC03C8
:10E310001092DB030BC0E22FFF27E055F74FC083BD
:10E320002F5F2093DC039C0F9093DB03C093DA03F1
:10E33000CF9108959091D603933240F4E92FFF27AF
:10E34000EA54F74F80839F5F9093D60308958332FA
:10E3500018F48D5F8093D603089590E2E9EBF8E01E
:10E360008FE19193815087FFFCCF0895CF93CFB772
:10E3700023E031E0F8948091C9008F778093C90041
:10E380008091C9008F7B8093C9008091C9008F7DE7
:10E390008093C9005A9A52985B9A539A832F99276F
:10E3A0008093CD002093CC008091C8008260809340
:10E3B000C80088E18093C9008091CA008F7780935C
:10E3C000CA008091CA008F7B8093CA008091CA00E6
:10E3D00080628093CA008091CA0080618093CA00E5
:10E3E0008091CA0088608093CA008091C9008460CF
:10E3F0008093C9008091CA0084608093CA00809194
:10E40000CA0082608093CA008091C80087FF03C061
:10E410008091CE00F9CF8091C90080688093C900B7
:10E420008091C90080648093C9000E94AD71CFBF04
:10E43000CF910895282F99278F709070892B31F4F0
:10E4400020958091D503822B8093D50308958091E8
:10E45000A401882309F44BC08091A20285FD04C069
:10E460008091A801882381F082E98093B60883E235
:10E470008093B7088091A801882309F485E58093EB
:10E48000B8081092A80102C08093B6088091A50137
:10E490008F3071F48091D5030E94426E882341F041
:10E4A00081E98093B6088093B70881E38093B80828
:10E4B0001092A4018091C80085FFFCCF8091C90013
:10E4C0008F7E8093C9008091C9008E7F8093C900A0
:10E4D0008091B608882311F48EEF01C08EE78093F7
:10E4E000CE008091D5038093A5011092D5030895A5
:10E4F0001F920F920FB60F9211248F939F93EF9359
:10E50000FF939091A401992309F040C08091DE030C
:10E51000882361F48091B608882311F483E003C056
:10E52000813999F481E08093DE030FC0833099F440
:10E530008091B608882349F09093B6088091C9006D
:10E540008E7F8093C9008EEF1EC08091C9008160CC
:10E550008093C9000EC0833261F48091C9008E7F20
:10E560008093C9008FEF8093CE0081E08093A40157
:10E5700014C08091DE03E82FFF27EA54F74F8F5F26
:10E580008093DE0380818093CE0007C01092DE036B
:10E590008091C90080618093C900FF91EF919F91A4
:10E5A0008F910F900FBE0F901F901895EF92FF92D2
:10E5B0000F931F93CF93DF937C018B01EA01452BCF
:10E5C00039F0F80181918F01F70109952197C9F779
:10E5D000E6E0CDB7DEB70C94CA7AEF92FF920F93C4
:10E5E0001F93CF93DF937C018B01EA01452B41F010
:10E5F000F8010F5F1F4F8491F70109952197C1F72B
:10E60000E6E0CDB7DEB70C94CA7A0F931F93CF9391
:10E610008C01C62F161634F480E2F8010995C1501A
:10E620001C16D4F3CF911F910F9108950F931F9350
:10E63000CF938C01C62F161634F480E3F8010995A8
:10E64000C1501C16D4F3CF911F910F910895A5E3EB
:10E65000B0E0EDE2F3E70C94A27A2E96EEADFFADBA
:10E660002E978824992454018091D403882321F47F
:10E670002C961FAE1EAE2C975EE4452E512C4C0EF0
:10E680005D1E6F01B60105C0153239F00894C11C3A
:10E69000D11CF60114911123B9F7A601461B570BA3
:10E6A00031F02C968EAD9FAD2C970E94ED72112308
:10E6B00009F46AC20894C11CD11CFF24FDA6FCA663
:10E6C0004FEFE42EF9A6F6010894C11CD11C149159
:10E6D000153721F0812F80628837B1F4F0FE0AC02F
:10E6E000F20124E030E0420E531E80809180A2802F
:10E6F000B3800AC0F20142E050E0440E551E808112
:10E7000091814C01AA24BB24103221F489A58823CD
:10E71000D1F61DC0133219F458E0F52AD4CF1A32BD
:10E7200011F01D3291F41A3259F4F20182E090E0B6
:10E73000480E591EE081ECA7EE232CF6E195ECA7DC
:10E7400090E1F92AAFEDFA22BECF1B3211F419A7DE
:10E75000BACF1E32C1F5F6010894C11CD11C149128
:10E760001A3279F4F20122E030E0420E531E408169
:10E7700051813FEF4F3F530714F44FEF5FEFE42E0B
:10E78000A2CF40E050E0812F80538A30A0F4CA012C
:10E7900033E0880F991F3A95E1F7840F951F480FD2
:10E7A000591F410F511D40535040F6010894C11CA0
:10E7B000D11C1491E8CF8FEF4F3F580714F44FEF5F
:10E7C0005FEFE42E85CF103329F4F4FC7CCF90E288
:10E7D000F92A79CF812F81538930D8F440E050E075
:10E7E000CA0123E0880F991F2A95E1F7840F951F2E
:10E7F000480F591F410F511D40535040F6010894D6
:10E80000C11CD11C1491812F80538A3048F34CA72E
:10E810005FCF183619F4A4E0FA2A55CF1C3619F444
:10E82000B1E0FB2A50CF133661F43E010894611C1D
:10E83000711CF20122E030E0420E531E8081898378
:10E840003CC1143421F0143611F0193651F514344A
:10E8500011F431E0F32AF0FE0AC0F20144E050E086
:10E86000440E551E80809180A280B3800CC0F201BE
:10E8700082E090E0480E591E808191814C01AA24CB
:10E8800097FCA094BA2CB7FE0AC0B094A0949094C0
:10E890008094811C911CA11CB11C8DE289A70AE007
:10E8A0006FC01F3411F01F3631F41F3411F491E0A2
:10E8B000F92A08E064C0103779F4F201A2E0B0E070
:10E8C0004A0E5B1E808191814C01AA24BB2400E189
:10E8D000B0E4FB2A18E753C01337C1F5F20122E078
:10E8E00030E0420E531E608071806114710489F41F
:10E8F0003E010894611C711C88E289838EE6F30155
:10E90000818385E78B838CE68C838D8389E28E837C
:10E910001F82E7FC13C08E2D992787FD9095AC01CF
:10E9200060E070E0C3010E946F78009729F0382EF4
:10E930003618E3140CF0C3C03E2CC1C0F3010190A3
:10E940000020E9F731973E2E3618B9C0153511F081
:10E95000153731F4153511F4F1E0FF2A0AE00FC044
:10E96000183519F0183709F0A0C000E1F3FE07C010
:10E9700081149104A104B10411F020E4F22A19A633
:10E98000EDA6E7FC02C03FEDF32289E2682E712C70
:10E990006C0E7D1E81149104A104B10421F44DA5D7
:10E9A000442309F47BC0802F9927AA27BB278EA771
:10E9B0009FA7A8ABB9AB202E332490E0891690E036
:10E9C000990691E0A90690E0B90648F0C501B401A6
:10E9D0002EA53FA548A959A90E94657A17C0AFEF97
:10E9E0008A169104A104B10449F040F0C401B101B8
:10E9F0000E943E7A9B014427552708C0882D602F2E
:10EA00000E94327A282F3327442755272AAB3BAB65
:10EA10004CAB5DAB0A3059F48AA9880F880F880F78
:10EA20009AA9990F890F382D381B832F10C00031F8
:10EA300039F48AA98295807F482D481B842F07C00E
:10EA40008AA9880F880F880F582D581B852F90E0B2
:10EA50002EA53FA548A959A982169306A406B50676
:10EA600008F091E08AA89BA8ACA8BDA88A3010F451
:10EA7000805D04C0895A183509F48F7DD3018E93C7
:10EA80003D01992309F099CF083041F4F3FE06C007
:10EA9000803321F080E3FD0182933F01CE01019696
:10EAA000382E3618F8E23F0E0BC0112309F46CC063
:10EAB0003E010894611C711C1983B1E03B2E19A61C
:10EAC000032D2DA4231827FC222489A5882311F0C7
:10EAD0000F5F02C0F6FC0E5F020DEF2CFF24C70192
:10EAE00080739070892B49F48CA5801B682F2C961D
:10EAF0008EAD9FAD2C970E94057389A5882331F0B8
:10EB000041E050E0BE01675D7F4F0AC0E6FE0EC0E7
:10EB100080E38AA71BA742E050E0BE01665D7F4FFD
:10EB20002C968EAD9FAD2C970E94D672C701807334
:10EB30009070809749F48CA5801B682F2C968EAD21
:10EB40009FAD2C970E941673622D2C968EAD9FADB3
:10EB50002C970E941673832D992787FD9095AC0101
:10EB6000B3012C968EAD9FAD2C970E94D672E4FE19
:10EB700089CD2CA5201B2CA7622F2C968EAD9FAD86
:10EB80002C970E9405737ECDE2E1CB5C0C94BE7A9B
:10EB90002FB740E0F894E0E0F0E081E28093570086
:10EBA0009491E2E0F0E0809357003491E4E0F0E0EB
:10EBB0008093570084912FBF9E3199F4363941F4E8
:10EBC000893011F441E00DC08A3059F442E009C0A7
:10EBD000373939F4863011F443E003C0853009F445
:10EBE00044E0842F992708959FB7F8948091C90035
:10EBF000877F8093C9008091C9008F7E8093C90070
:10EC00008091C9008F778093C9008091C9008F7B64
:10EC10008093C9008091C9008F7D8093C90052986C
:10EC20005A9A53985B9A9FBF08951F93CF93DF938F
:10EC3000182F8091D403882309F4A9C08091A301DF
:10EC4000181709F4A4C08091D303882321F40E94EB
:10EC5000C8758093D30382ED91E090934001809337
:10EC60003F018BEC9BE09F938F93C1E8D2E1DF9350
:10EC7000CF93E091E203F091E30309950F900F9099
:10EC80000F900F90812F99278330910539F18430AF
:10EC900091054CF48130910591F082309105DCF4BE
:10ECA000892B51F036C085309105F1F08530910502
:10ECB000C4F00697E1F02DC08BEB9BE002C089EA1F
:10ECC0009BE09F938F93DF93CF93E091E203F091CA
:10ECD000E30309952AC080E99BE0F3CF8DE69BE032
:10ECE000F0CF8FE59BE0EDCF87E59BE0EACF89E4AD
:10ECF0009BE09F938F93DF93CF93E091E203F0919A
:10ED0000E303099588ED91E09093400180933F01E2
:10ED10000CC088ED9BE09F938F93DF93CF93E0919E
:10ED2000E203F091E303099510E00F900F900F902C
:10ED30000F908091D303843011F0823099F40E94B7
:10ED4000F475812F8150833018F40E94D1681DC062
:10ED5000143019F40E94B67118C01530B1F40E9435
:10ED6000EB6F13C0112389F08EEE9BE09F938F937E
:10ED700081E892E19F938F93E091E203F091E303A6
:10ED800009950F900F900F900F901093A301DF91B2
:10ED9000CF911F9108950F931F9381E08093D40327
:10EDA0004091A201E9EFFAE020E030E05FE48491D5
:10EDB00099272F5F3F4F829FB001839F700D929FD5
:10EDC000700D112446275150319657FFF0CF4093D4
:10EDD000A201E1EDFAE020E030E057E284919927CA
:10EDE0002F5F3F4F829FB001839F700D929F700DE8
:10EDF000112446275150319657FFF0CF4093A2017E
:10EE00008091D303882321F40E94C8758093D30393
:10EE10008091A201833459F088E190E029E20FB695
:10EE2000F894A895809360000FBE2093600087E25D
:10EE300093E79093E3038093E20389E09CE09F9340
:10EE40008F9301E812E11F930F93E091E203F09199
:10EE5000E30309950F900F900F900F9081E690E0DB
:10EE60009F938F9386E590E09F938F931F921F92BD
:10EE7000809102016AE00E94327A892F99279F933C
:10EE80008F93809102010E94327A99279F938F93EA
:10EE90008FE29CE09F938F931F930F93E091E20387
:10EEA000F091E303099589EF9AE09F938F931F9365
:10EEB0000F93E091E203F091E303099581ED9AE06D
:10EEC0009F938F931F930F93E091E203F091E303DD
:10EED00009958DB79EB746968DBF83E69CE09F93BC
:10EEE0008F931F930F93E091E203F091E303099551
:10EEF00083EC8093810080916F00806280936F002B
:10EF00000F900F900F900F901F910F910895809187
:10EF100088068F3138F08091240887FD03C08EE188
:10EF20008093880680913806882331F08055853695
:10EF300018F08FE7809338060895CF938091D4031B
:10EF4000882309F46EC08091DF0381508093DF0332
:10EF5000882309F04FC089E18093DF038091880600
:10EF6000803238F08091240887FD03C08FE18093C0
:10EF700088068091D802823800F58091A302909192
:10EF8000A402885E934020F41092E1031092E00303
:10EF90008091E0039091E103009739F101979093FC
:10EFA000E1038093E003419728F18091240884FFD6
:10EFB00021C08091A10284601BC08091D802853B52
:10EFC000C8F09091880684E1989FC0011124409672
:10EFD0002091E0033091E1032817390730F42F5FC7
:10EFE0003F4F3093E1032093E0038091A1028B7F98
:10EFF0008093A102C091A601CC2321F0C150C093FF
:10F00000A6010FC086E98093A6018091A3018430F8
:10F0100011F40E9427728091A201833411F0C093F1
:10F02000D403CF9108951F920F920FB60F9211241F
:10F030002F933F934F935F936F937F938F939F9300
:10F04000AF93BF93EF93FF932091CE008091B201D5
:10F050008823B1F02093C6008091B201823029F557
:10F060002F3F19F58FEF94E3ACE0B0E0C297A10910
:10F07000B109B7FFFBCF809125048093CE0015C066
:10F080009091A301892F8150833020F4822F0E9418
:10F090002C690BC0943021F4822F0E941A7205C093
:10F0A000953019F4822F0E945971FF91EF91BF9111
:10F0B000AF919F918F917F916F915F914F913F9110
:10F0C0002F910F900FBE0F901F901895FB01DC0140
:10F0D00002C005900D9241505040D8F70895FC01B0
:10F0E0004150504030F001900616D1F73197CF01D2
:10F0F0000895882799270895A0E0B0E0E2E8F8E7AE
:10F100000C94AA7A6C017B01EA01590121978FEFD7
:10F11000CF3FD80789F086010894C11CD11CC701D4
:10F120000894E11CF11CF5010995F80180832197F1
:10F13000FFEFCF3FDF0779F7EAE0CDB7DEB70C94FA
:10F14000C67ACF92DF92EF92FF920F931F937C01CA
:10F150006B01FB010995082FC7010196F60109957E
:10F16000182FC8011F910F91FF90EF90DF90CF9063
:10F170000895A0E0B0E0EFEBF8E70C94AC7A8C01D6
:10F180007B01EA01690121978FEFCF3FD80771F02A
:10F19000F70121917F01C8010F5F1F4F622FF60118
:10F1A00009952197FFEFCF3FDF0791F7E8E0CDB753
:10F1B000DEB70C94C87ACF92DF92EF92FF920F9352
:10F1C0001F936C018B017A01FA010995812F992710
:10F1D000682FC6010196F70109951F910F91FF90C5
:10F1E000EF90DF90CF9008955058BB27AA270ED0FC
:10F1F000E0C0D1D030F0D6D020F031F49F3F11F4F0
:10F200001EF4C6C00EF4E095E7FBBCC0E92FE2D0C7
:10F2100080F3BA17620773078407950718F071F433
:10F220009EF5FAC00EF4E0950B2EBA2FA02D0B011F
:10F23000B90190010C01CA01A0011124FF27591B3B
:10F2400099F0593F50F4503E68F11A16F040A22F41
:10F25000232F342F4427585FF3CF469537952795B2
:10F26000A795F0405395C9F77EF41F16BA0B620BB1
:10F27000730B840BBAF09150A1F0FF0FBB1F661FF8
:10F28000771F881FC2F70EC0BA0F621F731F841F3B
:10F2900048F4879577956795B795F7959E3F08F061
:10F2A000B3CF9395880F08F09927EE0F9795879520
:10F2B000089598D088F09F5790F0B92F9927B751AB
:10F2C000A0F0D1F0660F771F881F991F1AF0BA952A
:10F2D000C9F712C0B13081F09FD0B1E008959CC051
:10F2E000672F782F8827B85F39F0B93FCCF3869520
:10F2F00077956795B395D9F73EF49095809570957D
:10F3000061957F4F8F4F9F4F0895E89409C097FBF9
:10F310003EF490958095709561957F4F8F4F9F4FEC
:10F320009923A9F0F92F96E9BB279395F695879530
:10F3300077956795B795F111F8CFFAF4BB0F11F4F3
:10F3400060FF1BC06F5F7F4F8F4F9F4F16C088239A
:10F3500011F096E911C0772321F09EE8872F762FD0
:10F3600005C0662371F096E8862F70E060E02AF011
:10F370009A95660F771F881FDAF7880F96958795FD
:10F3800097F9089597F99F6780E870E060E0089525
:10F390009FEF80EC089500240A94161617061806AD
:10F3A0000906089500240A94121613061406050689
:10F3B0000895092E0394000C11F4882352F0BB0F1A
:10F3C00040F4BF2B11F460FF04C06F5F7F4F8F4F7D
:10F3D0009F4F089557FD9058440F551F59F05F3FB8
:10F3E00071F04795880F97FB991F61F09F3F79F067
:10F3F00087950895121613061406551FF2CF4695E9
:10F40000F1DF08C0161617061806991FF1CF86956A
:10F410007105610508940895E894BB27662777274E
:10F42000CB0197F90895629FD001739FF001829FED
:10F43000E00DF11D649FE00DF11D929FF00D839F83
:10F44000F00D749FF00D659FF00D9927729FB00D20
:10F45000E11DF91F639FB00DE11DF91FBD01CF0133
:10F4600011240895991B79E004C0991F961708F09C
:10F47000961B881F7A95C9F780950895AA1BBB1B18
:10F4800051E107C0AA1FBB1FA617B70710F0A61BA4
:10F49000B70B881F991F5A95A9F780959095BC01C5
:10F4A000CD01089597FB092E07260AD077FD04D0D9
:10F4B000E5DF06D000201AF4709561957F4F08951E
:10F4C000F6F7909581959F4F0895A1E21A2EAA1BF9
:10F4D000BB1BFD010DC0AA1FBB1FEE1FFF1FA21704
:10F4E000B307E407F50720F0A21BB30BE40BF50B01
:10F4F000661F771F881F991F1A9469F7609570958A
:10F50000809590959B01AC01BD01CF01089597FBBB
:10F51000092E05260ED057FD04D0D7DF0AD0001CD7
:10F5200038F450954095309521953F4F4F4F5F4FA0
:10F530000895F6F790958095709561957F4F8F4F60
:10F540009F4F08952F923F924F925F926F927F92BA
:10F550008F929F92AF92BF92CF92DF92EF92FF92E3
:10F560000F931F93CF93DF93CDB7DEB7CA1BDB0B8F
:10F570000FB6F894DEBF0FBECDBF09942A88398834
:10F5800048885F846E847D848C849B84AA84B9843B
:10F59000C884DF80EE80FD800C811B81AA81B98147
:10F5A000CE0FD11D0FB6F894DEBF0FBECDBFED015B
:10F5B0000895EE0FFF1F0590F491E02D0994FFCF01
:10F5C0005E010A010164FF01FFFFC01FC01F0101AE
:10F5D00001737373FF03007D0000C409C409640054
:10F5E000104661737400004E6F726D616C000045CF
:10F5F000617379000051756164726F00006400D21C
:10F600000101200B050000ECFF00020406070808BA
:10F61000080706040200FEFCFAF9F8F8F8F9FAFC0B
:10F62000FE00020406070808286440415A46646444
:10F630000A02969696960840403A10FB30380132FE
:10F64000FF03780090D0030090D0030032002064C4
:10F65000FFFF64200B0A0D0B0C0E0B0F10FA20019C
:08F66000010170FF010F6400BD
:00000001FF
